 SWDialParserG

 Timestamp is 548ff518 (Tue Dec 16 17:02:16 2014)

 Preferred load address is 00100000

 Start         Length     Name                   Class
 0001:00000000 0001ba50H .text                   CODE
 0001:0001ba50 00000774H .text$yc                CODE
 0001:0001c1c4 000001dcH .text$yd                CODE
 0002:00000000 0000ccb4H .rdata                  DATA
 0002:0000ccb4 0000007aH .rdata$debug            DATA
 0002:0000cd30 000001bcH .rdata$r                DATA
 0002:0000ceec 000000f8H .xdata                  DATA
 0002:0000cfe4 00000158H .xdata$x                DATA
 0002:0000d13c 00000004H ATL$__a                 DATA
 0002:0000d140 00000004H ATL$__z                 DATA
 0002:0000d144 0000008cH .idata$2                DATA
 0002:0000d1d0 00000014H .idata$3                DATA
 0002:0000d1e4 00000204H .idata$4                DATA
 0002:0000d3e8 000001a0H .idata$6                DATA
 0002:0000d590 0000014cH .edata                  DATA
 0003:00000000 00000204H .idata$5                DATA
 0003:00000204 00000004H .CRT$XCA                DATA
 0003:00000208 00000004H .CRT$XCAA               DATA
 0003:0000020c 00000010H .CRT$XCC                DATA
 0003:0000021c 0000005cH .CRT$XCL                DATA
 0003:00000278 0000000cH .CRT$XCU                DATA
 0003:00000284 00000004H .CRT$XCZ                DATA
 0003:00000288 00000004H .CRT$XIA                DATA
 0003:0000028c 00000004H .CRT$XIZ                DATA
 0003:00000290 00000004H .CRT$XPA                DATA
 0003:00000294 00000004H .CRT$XPZ                DATA
 0003:00000298 00000004H .CRT$XTA                DATA
 0003:0000029c 00000004H .CRT$XTZ                DATA
 0003:000002a0 000002a8H .data                   DATA
 0003:00000548 000007acH .bss                    DATA
 0004:00000000 000013e8H .pdata                  DATA
 0005:00000000 000000a0H .rsrc$01                DATA
 0005:000000a0 00000504H .rsrc$02                DATA

  Address         Publics by Value              Rva+Base       Lib:Object

 0000:00000000       ___safe_se_handler_count   00000000     <absolute>
 0000:00000000       ___safe_se_handler_table   00000000     <absolute>
 0001:00000000       ??0CSWContextMenuClassFactory@@QAA@XZ 00101000 f   clsfact.obj
 0001:00000064       ??1CSWContextMenuClassFactory@@QAA@XZ 00101064 f   clsfact.obj
 0001:000000f0       ?AddRef@CSWContextMenuClassFactory@@UAAKXZ 001010f0 f   clsfact.obj
 0001:00000138       ?Release@CSWContextMenuClassFactory@@UAAKXZ 00101138 f   clsfact.obj
 0001:000001e0       ?QueryInterface@CSWContextMenuClassFactory@@UAAJABU_GUID@@PAPAX@Z 001011e0 f   clsfact.obj
 0001:000002f8       ?CreateInstance@CSWContextMenuClassFactory@@UAAJPAUIUnknown@@ABU_GUID@@PAPAX@Z 001012f8 f   clsfact.obj
 0001:00000400       ?LockServer@CSWContextMenuClassFactory@@UAAJH@Z 00101400 f   clsfact.obj
 0001:00000424       ??0IClassFactory@@QAA@XZ   00101424 f i clsfact.obj
 0001:00000450       ??0IUnknown@@QAA@XZ        00101450 f i clsfact.obj
 0001:00000474       ??_GCSWContextMenuClassFactory@@QAAPAXI@Z 00101474 f i clsfact.obj
 0001:000004b4       ??8@YAHABU_GUID@@0@Z       001014b4 f i clsfact.obj
 0001:0000050c       ?GetCarrier@@YAXXZ         0010150c f   DialParsExtOEM.obj
 0001:00000544       ?SWDialParserWndProc@@YAJPAUHWND__@@IIJ@Z 00101544 f   DialParsExtOEM.obj
 0001:000007e0       ?LaunchRiltest@@YAXXZ      001017e0 f   DialParsExtOEM.obj
 0001:000008c0       ?LaunchRegEdit@@YAXXZ      001018c0 f   DialParsExtOEM.obj
 0001:000009a0       ?LaunchPhoneUtility@@YAKPBG@Z 001019a0 f   DialParsExtOEM.obj
 0001:00000a9c       ?CreateMessageWindow@@YAJPAPAUHWND__@@PAUHINSTANCE__@@@Z 00101a9c f   DialParsExtOEM.obj
 0001:00000ca8       DllMain                    00101ca8 f   DialParsExtOEM.obj
 0001:00000e0c       ?PhExtFormatPhoneNumber@@YAHPBG00K@Z 00101e0c f   DialParsExtOEM.obj
 0001:00000e98       ?IsImmediateDialRequestRequired@@YAHPBG@Z 00101e98 f   DialParsExtOEM.obj
 0001:00000fe4       ?PreprocessDialRequest@@YAKPAUHWND__@@PBGH@Z 00101fe4 f   DialParsExtOEM.obj
 0001:000010a0       ?SW_PhExtFormatPhoneNumber@@YAHPBG00K@Z 001020a0 f   DialParsExtOEM.obj
 0001:000010cc       ?SW_IsImmediateDialRequestRequired@@YAHPBG@Z 001020cc f   DialParsExtOEM.obj
 0001:0000147c       ?SW_PreprocessDialRequest@@YAKPAUHWND__@@PBGH@Z 0010247c f   DialParsExtOEM.obj
 0001:0000191c       ?CheckifEmergencyNumber@@YAHPAG@Z 0010291c f   DialParsExtOEM.obj
 0001:00001be0       ?CheckIfSpecialNumber@@YAHPAG@Z 00102be0 f   DialParsExtOEM.obj
 0001:00001c5c       ?CheckSpecialProcess@@YAHPAG@Z 00102c5c f   DialParsExtOEM.obj
 0001:00001d7c       ?CheckforRoamGuard@@YAHPAUHWND__@@@Z 00102d7c f   DialParsExtOEM.obj
 0001:00001f50       ?MakeTapiVoiceCall@@YAKPAGI@Z 00102f50 f   DialParsExtOEM.obj
 0001:000020ec       ?CheckPowerState@@YAXXZ    001030ec f   DialParsExtOEM.obj
 0001:0000214c       DllCanUnloadNow            0010314c f   DialParsExtOEM.obj
 0001:000021dc       DllGetClassObject          001031dc f   DialParsExtOEM.obj
 0001:00002310       ??0Csw_ctxMenu@@QAA@XZ     00103310 f   DialParsExtOEM.obj
 0001:00002480       ??1Csw_ctxMenu@@QAA@XZ     00103480 f   DialParsExtOEM.obj
 0001:00002568       ?AddRef@Csw_ctxMenu@@UAAKXZ 00103568 f   DialParsExtOEM.obj
 0001:000025f4       ?Release@Csw_ctxMenu@@UAAKXZ 001035f4 f   DialParsExtOEM.obj
 0001:000026e0       ?QueryInterface@Csw_ctxMenu@@UAAJABU_GUID@@PAPAX@Z 001036e0 f   DialParsExtOEM.obj
 0001:000028ac       ?GetCommandString@Csw_ctxMenu@@UAAJIIPAIPADI@Z 001038ac f   DialParsExtOEM.obj
 0001:000029e0       ?InvokeCommand@Csw_ctxMenu@@UAAJPAU_CMInvokeCommandInfo@@@Z 001039e0 f   DialParsExtOEM.obj
 0001:00002b30       ?QueryContextMenu@Csw_ctxMenu@@UAAJPAUHMENU__@@IIII@Z 00103b30 f   DialParsExtOEM.obj
 0001:00002c0c       ?GetSite@Csw_ctxMenu@@UAAJABU_GUID@@PAPAX@Z 00103c0c f   DialParsExtOEM.obj
 0001:00002d10       ?SetSite@Csw_ctxMenu@@UAAJPAUIUnknown@@@Z 00103d10 f   DialParsExtOEM.obj
 0001:00002e24       ?LaunchActWiz@@YAXXZ       00103e24 f   DialParsExtOEM.obj
 0001:00002f28       ?wcsrchr@@YAPAGPAGG@Z      00103f28 f i DialParsExtOEM.obj
 0001:00002f5c       ?IsEqualGUID@@YAHABU_GUID@@0@Z 00103f5c f i DialParsExtOEM.obj
 0001:00002fb4       ??0IContextMenu@@QAA@XZ    00103fb4 f i DialParsExtOEM.obj
 0001:00002ff0       ??0IObjectWithSite@@QAA@XZ 00103ff0 f i DialParsExtOEM.obj
 0001:0000302c       ??_GCsw_ctxMenu@@QAAPAXI@Z 0010402c f i DialParsExtOEM.obj
 0001:0000306c       ?AddRef@Csw_ctxMenu@@W3AAKXZ 0010406c f i DialParsExtOEM.obj
 0001:00003074       ?QueryInterface@Csw_ctxMenu@@W3AAJABU_GUID@@PAPAX@Z 00104074 f i DialParsExtOEM.obj
 0001:0000307c       ?Release@Csw_ctxMenu@@W3AAKXZ 0010407c f i DialParsExtOEM.obj
 0001:00003084       ??0CResultListElement@@QAA@XZ 00104084 f   resultelement.obj
 0001:000030c8       ??1CResultListElement@@UAA@XZ 001040c8 f   resultelement.obj
 0001:000030e8       ?SetCallBackId@CResultListElement@@QAAXJ@Z 001040e8 f   resultelement.obj
 0001:00003108       ?GetCallBackId@CResultListElement@@QAAJXZ 00104108 f   resultelement.obj
 0001:00003134       ?SetFuncId@CResultListElement@@QAAXW4eFuncId@1@@Z 00104134 f   resultelement.obj
 0001:00003154       ?GetFuncId@CResultListElement@@QAA?AW4eFuncId@1@XZ 00104154 f   resultelement.obj
 0001:00003180       ??_GCResultListElement@@UAAPAXI@Z 00104180 f i resultelement.obj
 0001:00003180       ??_ECResultListElement@@UAAPAXI@Z 00104180 f i resultelement.obj
 0001:000031c0       ??0CAtlWinModule@ATL@@QAA@XZ 001041c0 f i resultelement.obj
 0001:0000327c       ??0_ATL_WIN_MODULE70@ATL@@QAA@XZ 0010427c f i resultelement.obj
 0001:000032e0       ??0CComCriticalSection@ATL@@QAA@XZ 001042e0 f i resultelement.obj
 0001:00003314       ??1CComCriticalSection@ATL@@QAA@XZ 00104314 f i resultelement.obj
 0001:00003324       ??0?$CSimpleArray@GV?$CSimpleArrayEqualHelper@G@ATL@@@ATL@@QAA@XZ 00104324 f i resultelement.obj
 0001:0000337c       ??1CAtlWinModule@ATL@@QAA@XZ 0010437c f i resultelement.obj
 0001:000033bc       ?Term@CAtlWinModule@ATL@@QAAXXZ 001043bc f i resultelement.obj
 0001:000033f0       ?GetModuleInstance@CAtlBaseModule@ATL@@QAAPAUHINSTANCE__@@XZ 001043f0 f i resultelement.obj
 0001:00003424       ??1_ATL_WIN_MODULE70@ATL@@QAA@XZ 00104424 f i resultelement.obj
 0001:00003470       ?AtlWinModuleTerm@ATL@@YAJPAU_ATL_WIN_MODULE70@1@PAUHINSTANCE__@@@Z 00104470 f i resultelement.obj
 0001:00003570       ?Term@CComCriticalSection@ATL@@QAAJXZ 00104570 f i resultelement.obj
 0001:0000359c       ?GetSize@?$CSimpleArray@GV?$CSimpleArrayEqualHelper@G@ATL@@@ATL@@QBAHXZ 0010459c f i resultelement.obj
 0001:000035c8       ?RemoveAll@?$CSimpleArray@GV?$CSimpleArrayEqualHelper@G@ATL@@@ATL@@QAAXXZ 001045c8 f i resultelement.obj
 0001:0000365c       ??A?$CSimpleArray@GV?$CSimpleArrayEqualHelper@G@ATL@@@ATL@@QAAAAGH@Z 0010465c f i resultelement.obj
 0001:00003724       ?_AtlRaiseException@ATL@@YAXKK@Z 00104724 f i resultelement.obj
 0001:00003748       ??1?$CSimpleArray@GV?$CSimpleArrayEqualHelper@G@ATL@@@ATL@@QAA@XZ 00104748 f i resultelement.obj
 0001:00003760       ??0CModemStatus@@QAA@XZ    00104760 f   winmodemstat.obj
 0001:000037f0       ??1CModemStatus@@UAA@XZ    001047f0 f   winmodemstat.obj
 0001:0000381c       ?AddResultItem@CModemStatus@@KAXJW4eFuncId@CResultListElement@@K@Z 0010481c f   winmodemstat.obj
 0001:00003954       ?Init@CModemStatus@@QAAJPAUHWND__@@@Z 00104954 f   winmodemstat.obj
 0001:00003a9c       ?Deregister@CModemStatus@@SAXXZ 00104a9c f   winmodemstat.obj
 0001:00003af4       ?PrepareRilDevSpecificInfo@CModemStatus@@KAPAUtagDEVSPECIFICDATA@@KKAAK@Z 00104af4 f   winmodemstat.obj
 0001:00003c98       ?ModGetSubscriberNumber@CModemStatus@@SAJXZ 00104c98 f   winmodemstat.obj
 0001:00003e58       ?ModReadPDP@CModemStatus@@SAJK@Z 00104e58 f   winmodemstat.obj
 0001:00003e84       ?SendSupServiceData@CModemStatus@@SAJPAGK@Z 00104e84 f   winmodemstat.obj
 0001:00003ef0       ?CancelSupServiceDataSession@CModemStatus@@SAJXZ 00104ef0 f   winmodemstat.obj
 0001:00003f44       ?ModGetOpState@CModemStatus@@SAJXZ 00104f44 f   winmodemstat.obj
 0001:00003fa0       ?ModGetCallList@CModemStatus@@SAJXZ 00104fa0 f   winmodemstat.obj
 0001:00004178       ?ModGetRegistrationStatus@CModemStatus@@SAJXZ 00105178 f   winmodemstat.obj
 0001:0000435c       ?RilResultCallback@CModemStatus@@KAXKJPBXKK@Z 0010535c f   winmodemstat.obj
 0001:00004bf0       ?RilNotifyCallback@CModemStatus@@KAXKPBXKK@Z 00105bf0 f   winmodemstat.obj
 0001:00005348       ?Read@CModemStatus@@SAJK@Z 00106348 f   winmodemstat.obj
 0001:00005498       ?AddrStrToDW@CModemStatus@@KAKPBG@Z 00106498 f   winmodemstat.obj
 0001:000055b0       ?SetSlotInfo@CModemStatus@@SAHH@Z 001065b0 f   winmodemstat.obj
 0001:0000574c       ?ExecNoParamDevSpecific@CModemStatus@@SAJK@Z 0010674c f   winmodemstat.obj
 0001:000059e8       ?Send2UI@CModemStatus@@SAJIIJ@Z 001069e8 f   winmodemstat.obj
 0001:00005b7c       ?MessageBoxOnSeparateThread@CModemStatus@@QAAXPBG0I@Z 00106b7c f   winmodemstat.obj
 0001:00005c68       ?MessageBoxFunction@CModemStatus@@KAIPAX@Z 00106c68 f   winmodemstat.obj
 0001:00005ce8       ?UpdateCallTypeAndStatus@CModemStatus@@KAKKKG@Z 00106ce8 f   winmodemstat.obj
 0001:0000682c       ?ParseDetailErrorCode@CModemStatus@@SAHPAUtagRLE_RILDEVSPECIFIC_ErrorCode@@KG@Z 0010782c f   winmodemstat.obj
 0001:000068ec       ?GetTestModeSettings@CModemStatus@@SAXXZ 001078ec f   winmodemstat.obj
 0001:00006994       ?GetPowerSaveMode@CModemStatus@@SAXXZ 00107994 f   winmodemstat.obj
 0001:00006a3c       ?PowerSaveExit@CModemStatus@@SAXXZ 00107a3c f   winmodemstat.obj
 0001:00006ae4       ?GetModemTime@CModemStatus@@SAHXZ 00107ae4 f   winmodemstat.obj
 0001:00006b48       ?StartDMMode@CModemStatus@@SAHK@Z 00107b48 f   winmodemstat.obj
 0001:00006c38       ?StopDMMode@CModemStatus@@SAHXZ 00107c38 f   winmodemstat.obj
 0001:00006c80       ?IsDMMode@CModemStatus@@SAHXZ 00107c80 f   winmodemstat.obj
 0001:00006ca8       ?StopEmergencyMode@CModemStatus@@SAJXZ 00107ca8 f   winmodemstat.obj
 0001:00006e84       ?ModSetEquipmentState@CModemStatus@@SAJK@Z 00107e84 f   winmodemstat.obj
 0001:000070bc       ?HangUp@CModemStatus@@SAJXZ 001080bc f   winmodemstat.obj
 0001:00007260       ??_GCModemStatus@@UAAPAXI@Z 00108260 f i winmodemstat.obj
 0001:00007260       ??_ECModemStatus@@UAAPAXI@Z 00108260 f i winmodemstat.obj
 0001:000072a0       ??1?$_Iterator@$00@?$list@VCResultListElement@@V?$allocator@VCResultListElement@@@std@@@std@@QAA@XZ 001082a0 f i winmodemstat.obj
 0001:000072b8       ??0CResultListElement@@QAA@ABV0@@Z 001082b8 f i winmodemstat.obj
 0001:00007334       ??1?$_Const_iterator@$00@?$list@VCResultListElement@@V?$allocator@VCResultListElement@@@std@@@std@@QAA@XZ 00108334 f i winmodemstat.obj
 0001:0000734c       ??1?$_Bidit@VCResultListElement@@HPBV1@ABV1@@std@@QAA@XZ 0010834c f i winmodemstat.obj
 0001:0000736c       ??1_Iterator_base@std@@QAA@XZ 0010836c f i winmodemstat.obj
 0001:000073c0       ?_Orphan_me@_Iterator_base@std@@QAAXXZ 001083c0 f i winmodemstat.obj
 0001:00007488       GetCurrentProcess          00108488 f i winmodemstat.obj
 0001:000074a0       ResetEvent                 001084a0 f i winmodemstat.obj
 0001:000074d4       SetEvent                   001084d4 f i winmodemstat.obj
 0001:00007508       ?_AtlGetConversionACP@ATL@@YAIXZ 00108508 f i winmodemstat.obj
 0001:00007520       ?W2T@@YAPAGPAG@Z           00108520 f i winmodemstat.obj
 0001:00007544       ??4?$_Iterator@$00@?$list@VCResultListElement@@V?$allocator@VCResultListElement@@@std@@@std@@QAAAAV012@ABV012@@Z 00108544 f i winmodemstat.obj
 0001:00007574       ??4CResultListElement@@QAAAAV0@ABV0@@Z 00108574 f i winmodemstat.obj
 0001:000075e0       ??0?$_Iterator@$00@?$list@VCResultListElement@@V?$allocator@VCResultListElement@@@std@@@std@@QAA@ABV012@@Z 001085e0 f i winmodemstat.obj
 0001:00007614       ??4?$_Const_iterator@$00@?$list@VCResultListElement@@V?$allocator@VCResultListElement@@@std@@@std@@QAAAAV012@ABV012@@Z 00108614 f i winmodemstat.obj
 0001:0000765c       ??0?$_Const_iterator@$00@?$list@VCResultListElement@@V?$allocator@VCResultListElement@@@std@@@std@@QAA@ABV012@@Z 0010865c f i winmodemstat.obj
 0001:000076a8       ??4?$_Bidit@VCResultListElement@@HPBV1@ABV1@@std@@QAAAAU01@ABU01@@Z 001086a8 f i winmodemstat.obj
 0001:000076e0       ??4_Iterator_base@std@@QAAAAV01@ABV01@@Z 001086e0 f i winmodemstat.obj
 0001:00007770       ?_Adopt@_Iterator_base@std@@QAAXPBV_Container_base@2@@Z 00108770 f i winmodemstat.obj
 0001:00007820       ??0?$_Bidit@VCResultListElement@@HPBV1@ABV1@@std@@QAA@ABU01@@Z 00108820 f i winmodemstat.obj
 0001:00007854       ??0_Iterator_base@std@@QAA@ABV01@@Z 00108854 f i winmodemstat.obj
 0001:000078a0       ?begin@?$list@VCResultListElement@@V?$allocator@VCResultListElement@@@std@@@std@@QAA?AV?$_Iterator@$00@12@XZ 001088a0 f i winmodemstat.obj
 0001:00007904       ?end@?$list@VCResultListElement@@V?$allocator@VCResultListElement@@@std@@@std@@QAA?AV?$_Iterator@$00@12@XZ 00108904 f i winmodemstat.obj
 0001:00007960       ?insert@?$list@VCResultListElement@@V?$allocator@VCResultListElement@@@std@@@std@@QAA?AV?$_Iterator@$00@12@V312@ABVCResultListElement@@@Z 00108960 f i winmodemstat.obj
 0001:00007a44       ?erase@?$list@VCResultListElement@@V?$allocator@VCResultListElement@@@std@@@std@@QAA?AV?$_Iterator@$00@12@V312@@Z 00108a44 f i winmodemstat.obj
 0001:00007c58       ??0?$_Iterator@$00@?$list@VCResultListElement@@V?$allocator@VCResultListElement@@@std@@@std@@QAA@XZ 00108c58 f i winmodemstat.obj
 0001:00007c88       ??D?$_Iterator@$00@?$list@VCResultListElement@@V?$allocator@VCResultListElement@@@std@@@std@@QBAAAVCResultListElement@@XZ 00108c88 f i winmodemstat.obj
 0001:00007cc0       ??E?$_Iterator@$00@?$list@VCResultListElement@@V?$allocator@VCResultListElement@@@std@@@std@@QAA?AV012@H@Z 00108cc0 f i winmodemstat.obj
 0001:00007d78       ??9?$_Const_iterator@$00@?$list@VCResultListElement@@V?$allocator@VCResultListElement@@@std@@@std@@QBA_NABV012@@Z 00108d78 f i winmodemstat.obj
 0001:00007dd0       ?_Nextnode@?$list@VCResultListElement@@V?$allocator@VCResultListElement@@@std@@@std@@KAAAPAU_Node@?$_List_nod@VCResultListElement@@V?$allocator@VCResultListElement@@@std@@@2@PAU342@@Z 00108dd0 f i winmodemstat.obj
 0001:00007df4       ?_Prevnode@?$list@VCResultListElement@@V?$allocator@VCResultListElement@@@std@@@std@@KAAAPAU_Node@?$_List_nod@VCResultListElement@@V?$allocator@VCResultListElement@@@std@@@2@PAU342@@Z 00108df4 f i winmodemstat.obj
 0001:00007e24       ?_Insert@?$list@VCResultListElement@@V?$allocator@VCResultListElement@@@std@@@std@@QAAXV?$_Iterator@$00@12@ABVCResultListElement@@@Z 00108e24 f i winmodemstat.obj
 0001:00007f20       ?_Orphan_ptr@?$list@VCResultListElement@@V?$allocator@VCResultListElement@@@std@@@std@@IBAXAAV12@PAU_Node@?$_List_nod@VCResultListElement@@V?$allocator@VCResultListElement@@@std@@@2@@Z 00108f20 f i winmodemstat.obj
 0001:00007ff4       ?deallocate@?$allocator@U_Node@?$_List_nod@VCResultListElement@@V?$allocator@VCResultListElement@@@std@@@std@@@std@@QAAXPAU_Node@?$_List_nod@VCResultListElement@@V?$allocator@VCResultListElement@@@std@@@2@I@Z 00108ff4 f i winmodemstat.obj
 0001:0000800c       ?destroy@?$allocator@U_Node@?$_List_nod@VCResultListElement@@V?$allocator@VCResultListElement@@@std@@@std@@@std@@QAAXPAU_Node@?$_List_nod@VCResultListElement@@V?$allocator@VCResultListElement@@@std@@@2@@Z 0010900c f i winmodemstat.obj
 0001:00008024       ??0?$_Iterator@$00@?$list@VCResultListElement@@V?$allocator@VCResultListElement@@@std@@@std@@QAA@PAU_Node@?$_List_nod@VCResultListElement@@V?$allocator@VCResultListElement@@@std@@@2@PBV12@@Z 00109024 f i winmodemstat.obj
 0001:0000805c       ??E?$_Iterator@$00@?$list@VCResultListElement@@V?$allocator@VCResultListElement@@@std@@@std@@QAAAAV012@XZ 0010905c f i winmodemstat.obj
 0001:00008088       ??F?$_Iterator@$00@?$list@VCResultListElement@@V?$allocator@VCResultListElement@@@std@@@std@@QAAAAV012@XZ 00109088 f i winmodemstat.obj
 0001:000080b4       ??0?$_Const_iterator@$00@?$list@VCResultListElement@@V?$allocator@VCResultListElement@@@std@@@std@@QAA@XZ 001090b4 f i winmodemstat.obj
 0001:000080f4       ??D?$_Const_iterator@$00@?$list@VCResultListElement@@V?$allocator@VCResultListElement@@@std@@@std@@QBAABVCResultListElement@@XZ 001090f4 f i winmodemstat.obj
 0001:000081d0       ??8?$_Const_iterator@$00@?$list@VCResultListElement@@V?$allocator@VCResultListElement@@@std@@@std@@QBA_NABV012@@Z 001091d0 f i winmodemstat.obj
 0001:00008238       ?_Mynode@?$_Const_iterator@$00@?$list@VCResultListElement@@V?$allocator@VCResultListElement@@@std@@@std@@QBAPAU_Node@?$_List_nod@VCResultListElement@@V?$allocator@VCResultListElement@@@std@@@3@XZ 00109238 f i winmodemstat.obj
 0001:00008264       ??0?$_Bidit@VCResultListElement@@HPBV1@ABV1@@std@@QAA@XZ 00109264 f i winmodemstat.obj
 0001:00008294       ??0_Iterator_base@std@@QAA@XZ 00109294 f i winmodemstat.obj
 0001:000082d4       ?_Myval@?$list@VCResultListElement@@V?$allocator@VCResultListElement@@@std@@@std@@KAAAVCResultListElement@@PAU_Node@?$_List_nod@VCResultListElement@@V?$allocator@VCResultListElement@@@std@@@2@@Z 001092d4 f i winmodemstat.obj
 0001:00008304       ?_Buynode@?$list@VCResultListElement@@V?$allocator@VCResultListElement@@@std@@@std@@IAAPAU_Node@?$_List_nod@VCResultListElement@@V?$allocator@VCResultListElement@@@std@@@2@PAU342@0ABVCResultListElement@@@Z 00109304 f i winmodemstat.obj
 0001:00008464       ?_Incsize@?$list@VCResultListElement@@V?$allocator@VCResultListElement@@@std@@@std@@IAAXI@Z 00109464 f i winmodemstat.obj
 0001:00008534       ??0length_error@std@@QAA@ABV?$basic_string@DU?$char_traits@D@std@@V?$allocator@D@2@@1@@Z 00109534 f i winmodemstat.obj
 0001:00008580       ??0logic_error@std@@QAA@ABV?$basic_string@DU?$char_traits@D@std@@V?$allocator@D@2@@1@@Z 00109580 f i winmodemstat.obj
 0001:000085f0       ?what@logic_error@std@@UBAPBDXZ 001095f0 f i winmodemstat.obj
 0001:00008624       ??_Glogic_error@std@@UAAPAXI@Z 00109624 f i winmodemstat.obj
 0001:00008624       ??_Elogic_error@std@@UAAPAXI@Z 00109624 f i winmodemstat.obj
 0001:00008664       ??1logic_error@std@@UAA@XZ 00109664 f i winmodemstat.obj
 0001:00008698       ??1length_error@std@@UAA@XZ 00109698 f i winmodemstat.obj
 0001:000086c0       ??_Glength_error@std@@UAAPAXI@Z 001096c0 f i winmodemstat.obj
 0001:000086c0       ??_Elength_error@std@@UAAPAXI@Z 001096c0 f i winmodemstat.obj
 0001:00008708       ??0?$basic_string@DU?$char_traits@D@std@@V?$allocator@D@2@@std@@QAA@ABV01@@Z 00109708 f i winmodemstat.obj
 0001:000087a8       ??1?$basic_string@DU?$char_traits@D@std@@V?$allocator@D@2@@std@@QAA@XZ 001097a8 f i winmodemstat.obj
 0001:000087f0       ?c_str@?$basic_string@DU?$char_traits@D@std@@V?$allocator@D@2@@std@@QBAPBDXZ 001097f0 f i winmodemstat.obj
 0001:00008820       ??1?$_String_val@DV?$allocator@D@std@@@std@@QAA@XZ 00109820 f i winmodemstat.obj
 0001:00008838       ??1_String_base@std@@QAA@XZ 00109838 f i winmodemstat.obj
 0001:00008850       ??1_Container_base@std@@QAA@XZ 00109850 f i winmodemstat.obj
 0001:00008868       ?_Orphan_all@_Container_base@std@@QBAXXZ 00109868 f i winmodemstat.obj
 0001:000088fc       ?assign@?$basic_string@DU?$char_traits@D@std@@V?$allocator@D@2@@std@@QAAAAV12@ABV12@II@Z 001098fc f i winmodemstat.obj
 0001:00008a20       ?_Tidy@?$basic_string@DU?$char_traits@D@std@@V?$allocator@D@2@@std@@IAAX_NI@Z 00109a20 f i winmodemstat.obj
 0001:00008acc       ?_Myptr@?$basic_string@DU?$char_traits@D@std@@V?$allocator@D@2@@std@@IBAPBDXZ 00109acc f i winmodemstat.obj
 0001:00008b24       ??0?$_String_val@DV?$allocator@D@std@@@std@@IAA@V?$allocator@D@1@@Z 00109b24 f i winmodemstat.obj
 0001:00008b64       ??0?$allocator@D@std@@QAA@ABV01@@Z 00109b64 f i winmodemstat.obj
 0001:00008b88       ??0_String_base@std@@QAA@XZ 00109b88 f i winmodemstat.obj
 0001:00008bb8       ??0_Container_base@std@@QAA@XZ 00109bb8 f i winmodemstat.obj
 0001:00008be8       ?erase@?$basic_string@DU?$char_traits@D@std@@V?$allocator@D@2@@std@@QAAAAV12@II@Z 00109be8 f i winmodemstat.obj
 0001:00008cfc       ?size@?$basic_string@DU?$char_traits@D@std@@V?$allocator@D@2@@std@@QBAIXZ 00109cfc f i winmodemstat.obj
 0001:00008d28       ?_Eos@?$basic_string@DU?$char_traits@D@std@@V?$allocator@D@2@@std@@IAAXI@Z 00109d28 f i winmodemstat.obj
 0001:00008d78       ?assign@?$char_traits@D@std@@SAXAADABD@Z 00109d78 f i winmodemstat.obj
 0001:00008d98       ?_Grow@?$basic_string@DU?$char_traits@D@std@@V?$allocator@D@2@@std@@IAA_NI_N@Z 00109d98 f i winmodemstat.obj
 0001:00008eac       ?_Myptr@?$basic_string@DU?$char_traits@D@std@@V?$allocator@D@2@@std@@IAAPADXZ 00109eac f i winmodemstat.obj
 0001:00008f04       ?deallocate@?$allocator@D@std@@QAAXPADI@Z 00109f04 f i winmodemstat.obj
 0001:00008f1c       ?allocate@?$allocator@U_Node@?$_List_nod@VCResultListElement@@V?$allocator@VCResultListElement@@@std@@@std@@@std@@QAAPAU_Node@?$_List_nod@VCResultListElement@@V?$allocator@VCResultListElement@@@std@@@2@I@Z 00109f1c f i winmodemstat.obj
 0001:00008f50       ?construct@?$allocator@PAU_Node@?$_List_nod@VCResultListElement@@V?$allocator@VCResultListElement@@@std@@@std@@@std@@QAAXPAPAU_Node@?$_List_nod@VCResultListElement@@V?$allocator@VCResultListElement@@@std@@@2@ABQAU342@@Z 00109f50 f i winmodemstat.obj
 0001:00008f6c       ?destroy@?$allocator@PAU_Node@?$_List_nod@VCResultListElement@@V?$allocator@VCResultListElement@@@std@@@std@@@std@@QAAXPAPAU_Node@?$_List_nod@VCResultListElement@@V?$allocator@VCResultListElement@@@std@@@2@@Z 00109f6c f i winmodemstat.obj
 0001:00008f8c       ??0?$_Const_iterator@$00@?$list@VCResultListElement@@V?$allocator@VCResultListElement@@@std@@@std@@QAA@PAU_Node@?$_List_nod@VCResultListElement@@V?$allocator@VCResultListElement@@@std@@@2@PBV12@@Z 00109f8c f i winmodemstat.obj
 0001:00008ff4       ??E?$_Const_iterator@$00@?$list@VCResultListElement@@V?$allocator@VCResultListElement@@@std@@@std@@QAAAAV012@XZ 00109ff4 f i winmodemstat.obj
 0001:000090e4       ??F?$_Const_iterator@$00@?$list@VCResultListElement@@V?$allocator@VCResultListElement@@@std@@@std@@QAAAAV012@XZ 0010a0e4 f i winmodemstat.obj
 0001:000091e0       ?_Compat@?$_Const_iterator@$00@?$list@VCResultListElement@@V?$allocator@VCResultListElement@@@std@@@std@@QBAXABV123@@Z 0010a1e0 f i winmodemstat.obj
 0001:0000929c       ??0length_error@std@@QAA@ABV01@@Z 0010a29c f i winmodemstat.obj
 0001:000092e8       ??0logic_error@std@@QAA@ABV01@@Z 0010a2e8 f i winmodemstat.obj
 0001:00009368       ??0?$basic_string@DU?$char_traits@D@std@@V?$allocator@D@2@@std@@QAA@PBD@Z 0010a368 f i winmodemstat.obj
 0001:000093e8       ?max_size@?$basic_string@DU?$char_traits@D@std@@V?$allocator@D@2@@std@@QBAIXZ 0010a3e8 f i winmodemstat.obj
 0001:00009450       ?_Copy@?$basic_string@DU?$char_traits@D@std@@V?$allocator@D@2@@std@@IAAXII@Z 0010a450 f i winmodemstat.obj
 0001:00009684       ?max_size@?$list@VCResultListElement@@V?$allocator@VCResultListElement@@@std@@@std@@QBAIXZ 0010a684 f i winmodemstat.obj
 0001:000096b8       ?construct@?$allocator@VCResultListElement@@@std@@QAAXPAVCResultListElement@@ABV3@@Z 0010a6b8 f i winmodemstat.obj
 0001:000096d4       ?assign@?$basic_string@DU?$char_traits@D@std@@V?$allocator@D@2@@std@@QAAAAV12@PBD@Z 0010a6d4 f i winmodemstat.obj
 0001:00009718       ?length@?$char_traits@D@std@@SAIPBD@Z 0010a718 f i winmodemstat.obj
 0001:00009748       ??0?$allocator@D@std@@QAA@XZ 0010a748 f i winmodemstat.obj
 0001:0000976c       ?allocate@?$allocator@D@std@@QAAPADI@Z 0010a76c f i winmodemstat.obj
 0001:000097a0       ?max_size@?$allocator@D@std@@QBAIXZ 0010a7a0 f i winmodemstat.obj
 0001:000097ec       ?max_size@?$allocator@VCResultListElement@@@std@@QBAIXZ 0010a7ec f i winmodemstat.obj
 0001:00009838       ?assign@?$basic_string@DU?$char_traits@D@std@@V?$allocator@D@2@@std@@QAAAAV12@PBDI@Z 0010a838 f i winmodemstat.obj
 0001:00009904       ?_Inside@?$basic_string@DU?$char_traits@D@std@@V?$allocator@D@2@@std@@IAA_NPBD@Z 0010a904 f i winmodemstat.obj
 0001:00009998       ??$_Debug_pointer@D@std@@YAXPBDPBGI@Z 0010a998 f i winmodemstat.obj
 0001:000099c8       ??$copy_s@U?$char_traits@D@std@@@_Traits_helper@std@@YAPADPADIPBDI@Z 0010a9c8 f i winmodemstat.obj
 0001:00009a30       ??$_Destroy@U_Node@?$_List_nod@VCResultListElement@@V?$allocator@VCResultListElement@@@std@@@std@@@std@@YAXPAU_Node@?$_List_nod@VCResultListElement@@V?$allocator@VCResultListElement@@@std@@@0@@Z 0010aa30 f i winmodemstat.obj
 0001:00009a4c       ??$move_s@U?$char_traits@D@std@@@_Traits_helper@std@@YAPADPADIPBDI@Z 0010aa4c f i winmodemstat.obj
 0001:00009ab4       ??$_Allocate@U_Node@?$_List_nod@VCResultListElement@@V?$allocator@VCResultListElement@@@std@@@std@@@std@@YAPAU_Node@?$_List_nod@VCResultListElement@@V?$allocator@VCResultListElement@@@std@@@0@IPAU120@@Z 0010aab4 f i winmodemstat.obj
 0001:00009b44       ??0bad_alloc@std@@QAA@PBD@Z 0010ab44 f i winmodemstat.obj
 0001:00009b88       ??1bad_alloc@std@@UAA@XZ   0010ab88 f i winmodemstat.obj
 0001:00009bb0       ??_Ebad_alloc@std@@UAAPAXI@Z 0010abb0 f i winmodemstat.obj
 0001:00009bb0       ??_Gbad_alloc@std@@UAAPAXI@Z 0010abb0 f i winmodemstat.obj
 0001:00009bf0       ??$_Construct@PAU_Node@?$_List_nod@VCResultListElement@@V?$allocator@VCResultListElement@@@std@@@std@@PAU123@@std@@YAXPAPAU_Node@?$_List_nod@VCResultListElement@@V?$allocator@VCResultListElement@@@std@@@0@ABQAU120@@Z 0010abf0 f i winmodemstat.obj
 0001:00009c58       ??2@YAPAXIPAX@Z            0010ac58 f i winmodemstat.obj
 0001:00009c7c       ??$_Destroy@PAU_Node@?$_List_nod@VCResultListElement@@V?$allocator@VCResultListElement@@@std@@@std@@@std@@YAXPAPAU_Node@?$_List_nod@VCResultListElement@@V?$allocator@VCResultListElement@@@std@@@0@@Z 0010ac7c f i winmodemstat.obj
 0001:00009c8c       ??$_Construct@VCResultListElement@@V1@@std@@YAXPAVCResultListElement@@ABV1@@Z 0010ac8c f i winmodemstat.obj
 0001:00009cf4       ??$_Allocate@D@std@@YAPADIPAD@Z 0010acf4 f i winmodemstat.obj
 0001:00009d7c       ??_G_Node@?$_List_nod@VCResultListElement@@V?$allocator@VCResultListElement@@@std@@@std@@QAAPAXI@Z 0010ad7c f i winmodemstat.obj
 0001:00009dbc       ??0bad_alloc@std@@QAA@ABV01@@Z 0010adbc f i winmodemstat.obj
 0001:00009e00       ??1_Node@?$_List_nod@VCResultListElement@@V?$allocator@VCResultListElement@@@std@@@std@@QAA@XZ 0010ae00 f i winmodemstat.obj
 0001:00009e1c       ??$_Char_traits_cat@U?$char_traits@D@std@@@std@@YA?AU_Secure_char_traits_tag@0@XZ 0010ae1c f i winmodemstat.obj
 0001:00009e50       ??$copy_s@U?$char_traits@D@std@@@_Traits_helper@std@@YAPADPADIPBDIU_Secure_char_traits_tag@1@@Z 0010ae50 f i winmodemstat.obj
 0001:00009e8c       ?_Copy_s@?$char_traits@D@std@@SAPADPADIPBDI@Z 0010ae8c f i winmodemstat.obj
 0001:00009ec4       ??$move_s@U?$char_traits@D@std@@@_Traits_helper@std@@YAPADPADIPBDIU_Secure_char_traits_tag@1@@Z 0010aec4 f i winmodemstat.obj
 0001:00009f00       ?_Move_s@?$char_traits@D@std@@SAPADPADIPBDI@Z 0010af00 f i winmodemstat.obj
 0001:00009f40       ??0?$list@VCResultListElement@@V?$allocator@VCResultListElement@@@std@@@std@@QAA@XZ 0010af40 f i winmodemstat.obj
 0001:00009fd0       ??1?$_List_val@VCResultListElement@@V?$allocator@VCResultListElement@@@std@@@std@@QAA@XZ 0010afd0 f i winmodemstat.obj
 0001:00009fe8       ??1?$_List_ptr@VCResultListElement@@V?$allocator@VCResultListElement@@@std@@@std@@QAA@XZ 0010afe8 f i winmodemstat.obj
 0001:0000a000       ??1?$_List_nod@VCResultListElement@@V?$allocator@VCResultListElement@@@std@@@std@@QAA@XZ 0010b000 f i winmodemstat.obj
 0001:0000a020       ?_Buynode@?$list@VCResultListElement@@V?$allocator@VCResultListElement@@@std@@@std@@IAAPAU_Node@?$_List_nod@VCResultListElement@@V?$allocator@VCResultListElement@@@std@@@2@XZ 0010b020 f i winmodemstat.obj
 0001:0000a124       ??0?$_List_val@VCResultListElement@@V?$allocator@VCResultListElement@@@std@@@std@@QAA@V?$allocator@VCResultListElement@@@1@@Z 0010b124 f i winmodemstat.obj
 0001:0000a180       ??0?$allocator@VCResultListElement@@@std@@QAA@XZ 0010b180 f i winmodemstat.obj
 0001:0000a1a4       ??0?$_List_ptr@VCResultListElement@@V?$allocator@VCResultListElement@@@std@@@std@@IAA@V?$allocator@VCResultListElement@@@1@@Z 0010b1a4 f i winmodemstat.obj
 0001:0000a200       ??0?$allocator@VCResultListElement@@@std@@QAA@ABV01@@Z 0010b200 f i winmodemstat.obj
 0001:0000a224       ??0?$_List_nod@VCResultListElement@@V?$allocator@VCResultListElement@@@std@@@std@@IAA@V?$allocator@VCResultListElement@@@1@@Z 0010b224 f i winmodemstat.obj
 0001:0000a264       ??$?0VCResultListElement@@@?$allocator@PAU_Node@?$_List_nod@VCResultListElement@@V?$allocator@VCResultListElement@@@std@@@std@@@std@@QAA@ABV?$allocator@VCResultListElement@@@1@@Z 0010b264 f i winmodemstat.obj
 0001:0000a288       ??$?0VCResultListElement@@@?$allocator@U_Node@?$_List_nod@VCResultListElement@@V?$allocator@VCResultListElement@@@std@@@std@@@std@@QAA@ABV?$allocator@VCResultListElement@@@1@@Z 0010b288 f i winmodemstat.obj
 0001:0000a2b4       ??1?$list@VCResultListElement@@V?$allocator@VCResultListElement@@@std@@@std@@QAA@XZ 0010b2b4 f i winmodemstat.obj
 0001:0000a2f4       ?_Tidy@?$list@VCResultListElement@@V?$allocator@VCResultListElement@@@std@@@std@@IAAXXZ 0010b2f4 f i winmodemstat.obj
 0001:0000a388       ?clear@?$list@VCResultListElement@@V?$allocator@VCResultListElement@@@std@@@std@@QAAXXZ 0010b388 f i winmodemstat.obj
 0001:0000a494       ?GetCarrierIndex@@YAKXZ    0010b494 f   sw_utilityG:sw_utilityG.dll
 0001:0000a4a4       ?WriteLog@@YAXKPBGZZ       0010b4a4 f   sw_utilityG:sw_utilityG.dll
 0001:0000a4b4       ?LogC@@YAXPBGZZ            0010b4b4 f   sw_utilityG:sw_utilityG.dll
 0001:0000a4c4       ?LogV@@YAXPBGZZ            0010b4c4 f   sw_utilityG:sw_utilityG.dll
 0001:0000a4d4       ?LogStoreFileLine@@YAXPAGH@Z 0010b4d4 f   sw_utilityG:sw_utilityG.dll
 0001:0000a4e4       ?GetVerInfo@@YAPAGPAUHINSTANCE__@@@Z 0010b4e4 f   sw_utilityG:sw_utilityG.dll
 0001:0000a4f4       ?InitLog@@YAXPAUHINSTANCE__@@@Z 0010b4f4 f   sw_utilityG:sw_utilityG.dll
 0001:0000a504       ?LogW@@YAXPBGZZ            0010b504 f   sw_utilityG:sw_utilityG.dll
 0001:0000a514       ?SWAI_GetRegValue@@YAJPAUHKEY__@@PBG1AAK@Z 0010b514 f   sw_utilityG:sw_utilityG.dll
 0001:0000a524       RIL_Initialize             0010b524 f   ril:ril.dll
 0001:0000a534       RIL_Deinitialize           0010b534 f   ril:ril.dll
 0001:0000a544       RIL_GetSubscriberNumbers   0010b544 f   ril:ril.dll
 0001:0000a554       RIL_SendSupServiceData     0010b554 f   ril:ril.dll
 0001:0000a564       RIL_CancelSupServiceDataSession 0010b564 f   ril:ril.dll
 0001:0000a574       RIL_GetEquipmentState      0010b574 f   ril:ril.dll
 0001:0000a584       RIL_GetCallList            0010b584 f   ril:ril.dll
 0001:0000a594       RIL_GetRegistrationStatus  0010b594 f   ril:ril.dll
 0001:0000a5a4       RIL_DevSpecific            0010b5a4 f   ril:ril.dll
 0001:0000a5b4       RIL_GetSystemTime          0010b5b4 f   ril:ril.dll
 0001:0000a5c4       RIL_SetEquipmentState      0010b5c4 f   ril:ril.dll
 0001:0000a5d4       RIL_Hangup                 0010b5d4 f   ril:ril.dll
 0001:0000a5e4       tapiRequestMakeCallW       0010b5e4 f   Cellcore:cellcore.dll
 0001:0000a5f4       SHGetEmergencyCallList     0010b5f4 f   aygshell:AYGSHELL.dll
 0001:0000a604       PhoneMakeCall              0010b604 f   phone:PHONE.dll
 0001:0000a614       NKDbgPrintfW               0010b614 f   coredll:COREDLL.dll
 0001:0000a624       ??3@YAXPAX@Z               0010b624 f   coredll:COREDLL.dll
 0001:0000a634       ??2@YAPAXI@Z               0010b634 f   coredll:COREDLL.dll
 0001:0000a644       memcmp                     0010b644 f   coredll:COREDLL.dll
 0001:0000a654       CreateProcessW             0010b654 f   coredll:COREDLL.dll
 0001:0000a664       CreateWindowExW            0010b664 f   coredll:COREDLL.dll
 0001:0000a674       GetLastError               0010b674 f   coredll:COREDLL.dll
 0001:0000a684       RegisterClassW             0010b684 f   coredll:COREDLL.dll
 0001:0000a694       swprintf                   0010b694 f   coredll:COREDLL.dll
 0001:0000a6a4       GetStockObject             0010b6a4 f   coredll:COREDLL.dll
 0001:0000a6b4       memset                     0010b6b4 f   coredll:COREDLL.dll
 0001:0000a6c4       DestroyWindow              0010b6c4 f   coredll:COREDLL.dll
 0001:0000a6d4       wcscmp                     0010b6d4 f   coredll:COREDLL.dll
 0001:0000a6e4       wcslen                     0010b6e4 f   coredll:COREDLL.dll
 0001:0000a6f4       wcscpy                     0010b6f4 f   coredll:COREDLL.dll
 0001:0000a704       wcsrchr                    0010b704 f   coredll:COREDLL.dll
 0001:0000a714       MessageBoxW                0010b714 f   coredll:COREDLL.dll
 0001:0000a724       LoadStringW                0010b724 f   coredll:COREDLL.dll
 0001:0000a734       Sleep                      0010b734 f   coredll:COREDLL.dll
 0001:0000a744       _purecall                  0010b744 f   coredll:COREDLL.dll
 0001:0000a754       InsertMenuW                0010b754 f   coredll:COREDLL.dll
 0001:0000a764       UnregisterClassW           0010b764 f   coredll:COREDLL.dll
 0001:0000a774       DeleteCriticalSection      0010b774 f   coredll:COREDLL.dll
 0001:0000a784       free                       0010b784 f   coredll:COREDLL.dll
 0001:0000a794       RaiseException             0010b794 f   coredll:COREDLL.dll
 0001:0000a7a4       CreateEventW               0010b7a4 f   coredll:COREDLL.dll
 0001:0000a7b4       ??_U@YAPAXI@Z              0010b7b4 f   coredll:COREDLL.dll
 0001:0000a7c4       TerminateProcess           0010b7c4 f   coredll:COREDLL.dll
 0001:0000a7d4       PostMessageW               0010b7d4 f   coredll:COREDLL.dll
 0001:0000a7e4       __rt_udiv                  0010b7e4 f   coredll:COREDLL.dll
 0001:0000a7f4       EventModify                0010b7f4 f   coredll:COREDLL.dll
 0001:0000a804       ??_V@YAXPAX@Z              0010b804 f   coredll:COREDLL.dll
 0001:0000a814       swscanf                    0010b814 f   coredll:COREDLL.dll
 0001:0000a824       SendMessageTimeout         0010b824 f   coredll:COREDLL.dll
 0001:0000a834       CreateThread               0010b834 f   coredll:COREDLL.dll
 0001:0000a844       wcsncpy                    0010b844 f   coredll:COREDLL.dll
 0001:0000a854       memcpy                     0010b854 f   coredll:COREDLL.dll
 0001:0000a864       __CxxThrowException        0010b864 f   coredll:COREDLL.dll
 0001:0000a874       ??_7type_info@@6B@         0010b874 f   coredll:COREDLL.dll
 0001:0000a884       ??0exception@std@@QAA@ABV01@@Z 0010b884 f   coredll:COREDLL.dll
 0001:0000a894       ??1exception@std@@UAA@XZ   0010b894 f   coredll:COREDLL.dll
 0001:0000a8a4       ??0exception@std@@QAA@XZ   0010b8a4 f   coredll:COREDLL.dll
 0001:0000a8b4       strlen                     0010b8b4 f   coredll:COREDLL.dll
 0001:0000a8c4       ??0exception@std@@QAA@PBD@Z 0010b8c4 f   coredll:COREDLL.dll
 0001:0000a8d4       ?what@exception@std@@UBAPBDXZ 0010b8d4 f   coredll:COREDLL.dll
 0001:0000a8e4       _DllMainCRTStartup         0010b8e4 f   corelibc:pegdmain.obj
 0001:0000a97c       __security_check_cookie    0010b97c     corelibc:armsecgs.obj
 0001:0000a990       __gsfailure                0010b990     corelibc:armsecgs.obj
 0001:0000a9d4       _onexit                    0010b9d4 f   corelibc:onexit.obj
 0001:0000aa80       atexit                     0010ba80 f   corelibc:onexit.obj
 0001:0000aad4       _cinit                     0010bad4 f   corelibc:crt0dat.obj
 0001:0000ac44       exit                       0010bc44 f   corelibc:crt0dat.obj
 0001:0000ac5c       _exit                      0010bc5c f   corelibc:crt0dat.obj
 0001:0000ac74       _cexit                     0010bc74 f   corelibc:crt0dat.obj
 0001:0000ac90       _c_exit                    0010bc90 f   corelibc:crt0dat.obj
 0001:0000acdc       __security_init_cookie     0010bcdc f   corelibc:seccinit.obj
 0001:0000ad2c       __InternalCxxFrameHandler  0010bd2c f   LIBCMTD:frame_ce.obj
 0001:0000af08       __CxxFrameHandler3         0010bf08 f   LIBCMTD:frame_ce.obj
 0001:0000b6e4       __FrameUnwindToState       0010c6e4 f   LIBCMTD:frame_ce.obj
 0001:0000c490       ?_DestructExceptionObject@@YAXPAUEHExceptionRecord@@E@Z 0010d490 f   LIBCMTD:frame_ce.obj
 0001:0000c5e0       ?_OffsetToAddress@@YAPAXHPAKK@Z 0010d5e0 f   LIBCMTD:frame_ce.obj
 0001:0000c66c       ?FindFrameInfo@@YAPAU_FrameInfo@@PAK@Z 0010d66c f   LIBCMTD:frame_ce.obj
 0001:0000c6f4       ?FindCatchFrameInfo@@YAPAU_FrameInfo@@PAK@Z 0010d6f4 f   LIBCMTD:frame_ce.obj
 0001:0000c778       ?_GetRangeOfTrysToCheck@@YAPBU_s_TryBlockMapEntry@@PBU_s_FuncInfo@@HHPAI1@Z 0010d778 f   LIBCMTD:frame_ce.obj
 0001:0000c870       __GSHandlerCheckCommon     0010d870 f   LIBCMTD:gshandler.obj
 0001:0000c8b8       __GSHandlerCheck           0010d8b8 f   LIBCMTD:gshandler.obj
 0001:0000c8f0       _CrtSetReportHookT2        0010d8f0 f   LIBCMTD:dbgrpt.obj
 0001:0000cdbc       _CrtDbgReportW             0010ddbc f   LIBCMTD:dbgrpt.obj
 0001:0000ce34       _CrtDbgReportTV            0010de34 f i LIBCMTD:dbgrpt.obj
 0001:0000ce90       __crtMessageWindowW        0010de90 f   LIBCMTD:dbgrpt.obj
 0001:0000d568       _invoke_watson_if_error    0010e568 f i LIBCMTD:dbgrpt.obj
 0001:0000d5bc       _invalid_parameter         0010e5bc f   LIBCMTD:invarginternal.obj
 0001:0000d600       __GSHandlerCheck_EH        0010e600 f   LIBCMTD:gshandlereh.obj
 0001:0000d694       memcpy_s                   0010e694 f   LIBCMTD:memcpy_s.obj
 0001:0000d94c       memmove_s                  0010e94c f   LIBCMTD:memmove_s.obj
 0001:0000dbc0       GetCRTStorage              0010ebc0 f   LIBCMTD:corecrt.obj
 0001:0000dcd0       TlsAlloc                   0010ecd0 f i LIBCMTD:corecrt.obj
 0001:0000dd0c       TlsFree                    0010ed0c f i LIBCMTD:corecrt.obj
 0001:0000dd50       ?FindFrameForUnwind@@YAPAKPAKPBU_s_FuncInfo@@@Z 0010ed50 f   LIBCMTD:mdframe_arm.obj
 0001:0000dde8       ?FindCatchFrame@@YAPAKPAKK@Z 0010ede8 f   LIBCMTD:mdframe_arm.obj
 0001:0000de80       ?AdjustFrameForCatch@@YAPAKPAKPBU_s_FuncInfo@@@Z 0010ee80 f   LIBCMTD:mdframe_arm.obj
 0001:0000df20       ?GetCurrentState@@YAHPAKPAU_DISPATCHER_CONTEXT@@PBU_s_FuncInfo@@@Z 0010ef20 f   LIBCMTD:ehstate_arm_mips.obj
 0001:0000dffc       _CallSettingFrame          0010effc     LIBCMTD:handlers_arm.obj
 0001:0000e040       _mtinitlocks               0010f040 f   LIBCMTD:mlock.obj
 0001:0000e158       _mtdeletelocks             0010f158 f   LIBCMTD:mlock.obj
 0001:0000e2dc       _mtinitlocknum             0010f2dc f   LIBCMTD:mlock.obj
 0001:0000e444       _lock                      0010f444 f   LIBCMTD:mlock.obj
 0001:0000e540       _unlock                    0010f540 f   LIBCMTD:mlock.obj
 0001:0000e580       _lockerr_exit              0010f580 f   LIBCMTD:mlock.obj
 0001:0000e5a8       _CrtDbgBreak               0010f5a8 f   LIBCMTD:dbgrptt.obj
 0001:0000e5b0       _CrtSetReportMode          0010f5b0 f   LIBCMTD:dbgrptt.obj
 0001:0000e7d8       _CrtSetReportFile          0010f7d8 f   LIBCMTD:dbgrptt.obj
 0001:0000e974       _CrtSetReportHook          0010f974 f   LIBCMTD:dbgrptt.obj
 0001:0000e9b8       _CrtGetReportHook          0010f9b8 f   LIBCMTD:dbgrptt.obj
 0001:0000e9e0       _VCrtDbgReportW            0010f9e0 f   LIBCMTD:dbgrptt.obj
 0001:0000f598       __crtMessageBoxW           00110598 f   LIBCMTD:crtmbox.obj
 0001:0000f7fc       wcsncpy_s                  001107fc f   LIBCMTD:wcsncpy_s.obj
 0001:0000fdfc       wcscpy_s                   00110dfc f   LIBCMTD:wcscpy_s.obj
 0001:00010270       _invoke_watson             00111270 f   LIBCMTD:invarg.obj
 0001:000102a4       _initp_misc_initcrit       001112a4 f   LIBCMTD:initcrit.obj
 0001:000102d0       __crtInitCritSecAndSpinCount 001112d0 f   LIBCMTD:initcrit.obj
 0001:00010400       _amsg_exit                 00111400 f   LIBCMTD:crt0dat.obj
 0001:0001042c       __crtExitProcess           0011142c f   LIBCMTD:crt0dat.obj
 0001:00010474       strcpy_s                   00111474 f   LIBCMTD:strcpy_s.obj
 0001:000108c8       wcscat_s                   001118c8 f   LIBCMTD:wcscat_s.obj
 0001:00010eac       _itow_s                    00111eac f   LIBCMTD:xtows.obj
 0001:00011538       _ltow_s                    00112538 f   LIBCMTD:xtows.obj
 0001:000115b8       _ultow_s                   001125b8 f   LIBCMTD:xtows.obj
 0001:0001160c       _encode_pointer            0011260c f   LIBCMTD:tidtable.obj
 0001:00011634       _encoded_null              00112634 f   LIBCMTD:tidtable.obj
 0001:0001166c       _decode_pointer            0011266c f   LIBCMTD:tidtable.obj
 0001:00011694       ??0_Init_locks@std@@QAA@XZ 00112694 f   libcpmtd:xlock.obj
 0001:000116f4       ??1_Init_locks@std@@QAA@XZ 001126f4 f   libcpmtd:xlock.obj
 0001:0001174c       ?_Init_locks_ctor@_Init_locks@std@@CAXPAV12@@Z 0011274c f   libcpmtd:xlock.obj
 0001:000117a4       ?_Init_locks_dtor@_Init_locks@std@@CAXPAV12@@Z 001127a4 f   libcpmtd:xlock.obj
 0001:000117fc       ??0_Lockit@std@@QAA@XZ     001127fc f   libcpmtd:xlock.obj
 0001:00011830       ??0_Lockit@std@@QAA@H@Z    00112830 f   libcpmtd:xlock.obj
 0001:0001186c       ??1_Lockit@std@@QAA@XZ     0011286c f   libcpmtd:xlock.obj
 0001:0001189c       ?_Lockit_ctor@_Lockit@std@@CAXPAV12@@Z 0011289c f   libcpmtd:xlock.obj
 0001:000118c0       ?_Lockit_ctor@_Lockit@std@@CAXPAV12@H@Z 001128c0 f   libcpmtd:xlock.obj
 0001:000118f8       ?_Lockit_dtor@_Lockit@std@@CAXPAV12@@Z 001128f8 f   libcpmtd:xlock.obj
 0001:00011928       ?_Debug_message@std@@YAXPBD0@Z 00112928 f   libcpmtd:stdthrow.obj
 0001:000119e8       ?_Debug_message@std@@YAXPB_W0I@Z 001129e8 f   libcpmtd:stdthrow.obj
 0001:00011a28       ?_Debug_message@std@@YAXPBG0I@Z 00112a28 f   libcpmtd:stdthrow.obj
 0001:00011a44       ?_Throw@std@@YAXABVexception@1@@Z 00112a44 f   libcpmtd:stdthrow.obj
 0001:00011a7c       ??$_Debug_pointer@D@std@@YAXPBDPB_WI@Z 00112a7c f i libcpmtd:string.obj
 0001:00011aa4       ??0invalid_argument@std@@QAA@ABV?$basic_string@DU?$char_traits@D@std@@V?$allocator@D@2@@1@@Z 00112aa4 f i libcpmtd:string.obj
 0001:00011ad4       ??1invalid_argument@std@@UAA@XZ 00112ad4 f i libcpmtd:string.obj
 0001:00011b00       ??_Ginvalid_argument@std@@UAAPAXI@Z 00112b00 f i libcpmtd:string.obj
 0001:00011b00       ??_Einvalid_argument@std@@UAAPAXI@Z 00112b00 f i libcpmtd:string.obj
 0001:00011b4c       ??0out_of_range@std@@QAA@ABV?$basic_string@DU?$char_traits@D@std@@V?$allocator@D@2@@1@@Z 00112b4c f i libcpmtd:string.obj
 0001:00011b7c       ??1out_of_range@std@@UAA@XZ 00112b7c f i libcpmtd:string.obj
 0001:00011ba8       ??_Eout_of_range@std@@UAAPAXI@Z 00112ba8 f i libcpmtd:string.obj
 0001:00011ba8       ??_Gout_of_range@std@@UAAPAXI@Z 00112ba8 f i libcpmtd:string.obj
 0001:00011bfc       ?_Xlen@_String_base@std@@SAXXZ 00112bfc f   libcpmtd:string.obj
 0001:00011c8c       ?_Xran@_String_base@std@@SAXXZ 00112c8c f   libcpmtd:string.obj
 0001:00011d14       ??0out_of_range@std@@QAA@ABV01@@Z 00112d14 f i libcpmtd:string.obj
 0001:00011d4c       ?_Xinvarg@_String_base@std@@SAXXZ 00112d4c f   libcpmtd:string.obj
 0001:00011dd4       ??0invalid_argument@std@@QAA@ABV01@@Z 00112dd4 f i libcpmtd:string.obj
 0001:00011e04       _Once                      00112e04 f   libcpmtd:xmtx.obj
 0001:00011e90       _Mtxinit                   00112e90 f   libcpmtd:xmtx.obj
 0001:00011eac       _Mtxdst                    00112eac f   libcpmtd:xmtx.obj
 0001:00011ec8       _Mtxlock                   00112ec8 f   libcpmtd:xmtx.obj
 0001:00011ee4       _Mtxunlock                 00112ee4 f   libcpmtd:xmtx.obj
 0001:00011f00       ?AtlAdvise@ATL@@YAJPAUIUnknown@@0ABU_GUID@@PAK@Z 00112f00 f   atlsd:atlfuncs.obj
 0001:000120bc       ?AtlUnadvise@ATL@@YAJPAUIUnknown@@ABU_GUID@@K@Z 001130bc f   atlsd:atlfuncs.obj
 0001:00012274       ?AtlFreeMarshalStream@ATL@@YAJPAUIStream@@@Z 00113274 f   atlsd:atlfuncs.obj
 0001:0001232c       ?AtlMarshalPtrInProc@ATL@@YAJPAUIUnknown@@ABU_GUID@@PAPAUIStream@@@Z 0011332c f   atlsd:atlfuncs.obj
 0001:00012470       ?AtlUnmarshalPtr@ATL@@YAJPAUIStream@@ABU_GUID@@PAPAUIUnknown@@@Z 00113470 f   atlsd:atlfuncs.obj
 0001:00012590       ?AtlComModuleGetClassObject@ATL@@YAJPAU_ATL_COM_MODULE70@1@ABU_GUID@@1PAPAX@Z 00113590 f   atlsd:atlfuncs.obj
 0001:00012908       ?AtlComModuleRegisterClassObjects@ATL@@YAJPAU_ATL_COM_MODULE70@1@KK@Z 00113908 f   atlsd:atlfuncs.obj
 0001:00012a28       ?AtlComModuleRevokeClassObjects@ATL@@YAJPAU_ATL_COM_MODULE70@1@@Z 00113a28 f   atlsd:atlfuncs.obj
 0001:00012b40       ?AtlWaitWithMessageLoop@ATL@@YAHPAX@Z 00113b40 f   atlsd:atlfuncs.obj
 0001:00012cd8       ?AtlInternalQueryInterface@ATL@@YAJPAXPBU_ATL_INTMAP_ENTRY@1@ABU_GUID@@PAPAX@Z 00113cd8 f   atlsd:atlfuncs.obj
 0001:00013060       ?AtlGetVersion@ATL@@YAKPAX@Z 00114060 f   atlsd:atlfuncs.obj
 0001:00013088       ?AtlWinModuleAddCreateWndData@ATL@@YAXPAU_ATL_WIN_MODULE70@1@PAU_AtlCreateWndData@1@PAX@Z 00114088 f   atlsd:atlfuncs.obj
 0001:000132c4       ?AtlWinModuleExtractCreateWndData@ATL@@YAPAXPAU_ATL_WIN_MODULE70@1@@Z 001142c4 f   atlsd:atlfuncs.obj
 0001:00013510       ?AtlWinModuleInit@ATL@@YAJPAU_ATL_WIN_MODULE70@1@@Z 00114510 f   atlsd:atlfuncs.obj
 0001:00013660       ?AtlModuleAddTermFunc@ATL@@YAJPAU_ATL_MODULE70@1@P6AXK@ZK@Z 00114660 f   atlsd:atlfuncs.obj
 0001:0001386c       ?AtlCallTermFunc@ATL@@YAXPAU_ATL_MODULE70@1@@Z 0011486c f   atlsd:atlfuncs.obj
 0001:00013934       ??1?$CComPtr@UIConnectionPointContainer@@@ATL@@QAA@XZ 00114934 f i atlsd:atlfuncs.obj
 0001:0001395c       ??1?$CComPtr@UIConnectionPoint@@@ATL@@QAA@XZ 0011495c f i atlsd:atlfuncs.obj
 0001:00013984       GetCurrentThreadId         00114984 f i atlsd:atlfuncs.obj
 0001:000139a4       ?IsWindowUnicode@ATL@@YAHPAUHWND__@@@Z 001149a4 f i atlsd:atlfuncs.obj
 0001:000139cc       ??0?$CComPtr@UIConnectionPointContainer@@@ATL@@QAA@XZ 001149cc f i atlsd:atlfuncs.obj
 0001:00013a0c       ??1?$CComPtrBase@UIConnectionPointContainer@@@ATL@@QAA@XZ 00114a0c f i atlsd:atlfuncs.obj
 0001:00013a54       ??I?$CComPtrBase@UIConnectionPointContainer@@@ATL@@QAAPAPAUIConnectionPointContainer@@XZ 00114a54 f i atlsd:atlfuncs.obj
 0001:00013ad0       ??C?$CComPtrBase@UIConnectionPointContainer@@@ATL@@QBAPAV?$_NoAddRefReleaseOnCComPtr@UIConnectionPointContainer@@@1@XZ 00114ad0 f i atlsd:atlfuncs.obj
 0001:00013b50       ??0?$CComPtr@UIConnectionPoint@@@ATL@@QAA@XZ 00114b50 f i atlsd:atlfuncs.obj
 0001:00013b90       ??1?$CComPtrBase@UIConnectionPoint@@@ATL@@QAA@XZ 00114b90 f i atlsd:atlfuncs.obj
 0001:00013bd8       ??I?$CComPtrBase@UIConnectionPoint@@@ATL@@QAAPAPAUIConnectionPoint@@XZ 00114bd8 f i atlsd:atlfuncs.obj
 0001:00013c54       ??C?$CComPtrBase@UIConnectionPoint@@@ATL@@QBAPAV?$_NoAddRefReleaseOnCComPtr@UIConnectionPoint@@@1@XZ 00114c54 f i atlsd:atlfuncs.obj
 0001:00013cd4       ??0?$CComPtrBase@UIConnectionPointContainer@@@ATL@@IAA@XZ 00114cd4 f i atlsd:atlfuncs.obj
 0001:00013d08       ??0?$CComPtrBase@UIConnectionPoint@@@ATL@@IAA@XZ 00114d08 f i atlsd:atlfuncs.obj
 0001:00013d3c       ?InlineIsEqualGUID@ATL@@YAHABU_GUID@@0@Z 00114d3c f i atlsd:atlfuncs.obj
 0001:00013df0       ??0CTraceFileAndLineInfo@ATL@@QAA@PBDH@Z 00114df0 f i atlsd:atlfuncs.obj
 0001:00013e34       ??RCTraceFileAndLineInfo@ATL@@QBAXKIPB_WZZ 00114e34 f i atlsd:atlfuncs.obj
 0001:00013eac       ?TraceV@CTrace@ATL@@QBAXPBDHKIPB_WPAD@Z 00114eac f i atlsd:atlfuncs.obj
 0001:00013f08       ??BCTraceCategory@ATL@@QBAKXZ 00114f08 f i atlsd:atlfuncs.obj
 0001:00013f3c       ?Init@CComCriticalSection@ATL@@QAAJXZ 00114f3c f i atlsd:atlfuncs.obj
 0001:00013fe0       ?RevokeClassObject@_ATL_OBJMAP_ENTRY30@ATL@@QAAJXZ 00114fe0 f i atlsd:atlfuncs.obj
 0001:00014048       ?RegisterClassObject@_ATL_OBJMAP_ENTRY30@ATL@@QAAJKK@Z 00115048 f i atlsd:atlfuncs.obj
 0001:00014140       ?InlineIsEqualUnknown@ATL@@YAHABU_GUID@@@Z 00115140 f i atlsd:atlfuncs.obj
 0001:000141c8       ??0?$CComCritSecLock@VCComCriticalSection@ATL@@@ATL@@QAA@AAVCComCriticalSection@1@_N@Z 001151c8 f i atlsd:atlfuncs.obj
 0001:00014258       ?AtlThrowImpl@ATL@@YAXJ@Z  00115258 f i atlsd:atlfuncs.obj
 0001:00014368       ??1?$CComCritSecLock@VCComCriticalSection@ATL@@@ATL@@QAA@XZ 00115368 f i atlsd:atlfuncs.obj
 0001:000143a4       ?Unlock@?$CComCritSecLock@VCComCriticalSection@ATL@@@ATL@@QAAXXZ 001153a4 f i atlsd:atlfuncs.obj
 0001:00014444       ?Unlock@CComCriticalSection@ATL@@QAAJXZ 00115444 f i atlsd:atlfuncs.obj
 0001:00014480       ?Lock@?$CComCritSecLock@VCComCriticalSection@ATL@@@ATL@@QAAJXZ 00115480 f i atlsd:atlfuncs.obj
 0001:00014550       ?Lock@CComCriticalSection@ATL@@QAAJXZ 00115550 f i atlsd:atlfuncs.obj
 0001:0001458c       AtlRawDllMain              0011558c f   atlsd:atlbase.obj
 0001:0001468c       ?CoDisconnectObject@ATL@@YAJPAUIUnknown@@K@Z 0011568c f   atlsd:atlbase.obj
 0001:000147e0       ?CoInitialize@ATL@@YAJPAX@Z 001157e0 f   atlsd:atlbase.obj
 0001:00014894       ?CoRevokeClassObject@ATL@@YAJK@Z 00115894 f   atlsd:atlbase.obj
 0001:00014948       ?CoRegisterClassObject@ATL@@YAJABU_GUID@@PAUIUnknown@@KKPAK@Z 00115948 f   atlsd:atlbase.obj
 0001:00014a10       ?CoMarshalInterface@ATL@@YAJPAUIStream@@ABU_GUID@@PAUIUnknown@@KPAXK@Z 00115a10 f   atlsd:atlbase.obj
 0001:00014ae0       ?CoUnmarshalInterface@ATL@@YAJPAUIStream@@ABU_GUID@@PAPAX@Z 00115ae0 f   atlsd:atlbase.obj
 0001:00014b9c       ?CoReleaseMarshalData@ATL@@YAJPAUIStream@@@Z 00115b9c f   atlsd:atlbase.obj
 0001:00014c50       ?OleSaveToStream@ATL@@YAJPAUIPersistStream@@PAUIStream@@@Z 00115c50 f   atlsd:atlbase.obj
 0001:00014e08       ?OleLoadFromStream@ATL@@YAJPAUIStream@@ABU_GUID@@PAPAX@Z 00115e08 f   atlsd:atlbase.obj
 0001:00015134       ??0CAtlBaseModule@ATL@@QAA@XZ 00116134 f   atlsd:atlbase.obj
 0001:000152c0       ??1CAtlBaseModule@ATL@@QAA@XZ 001162c0 f   atlsd:atlbase.obj
 0001:00015300       ?AddResourceInstance@CAtlBaseModule@ATL@@QAA_NPAUHINSTANCE__@@@Z 00116300 f   atlsd:atlbase.obj
 0001:0001549c       ?RemoveResourceInstance@CAtlBaseModule@ATL@@QAA_NPAUHINSTANCE__@@@Z 0011649c f   atlsd:atlbase.obj
 0001:000156b0       ?GetHInstanceAt@CAtlBaseModule@ATL@@QAAPAUHINSTANCE__@@H@Z 001166b0 f   atlsd:atlbase.obj
 0001:000158e4       ??0_ATL_BASE_MODULE70@ATL@@QAA@XZ 001168e4 f i atlsd:atlbase.obj
 0001:00015944       ??1_ATL_BASE_MODULE70@ATL@@QAA@XZ 00116944 f i atlsd:atlbase.obj
 0001:00015988       ?_AtlGetThisModuleHandle@ATL@@YAPAUHINSTANCE__@@XZ 00116988 f i atlsd:atlbase.obj
 0001:000159e8       ??0?$CSimpleArray@PAUHINSTANCE__@@V?$CSimpleArrayEqualHelper@PAUHINSTANCE__@@@ATL@@@ATL@@QAA@XZ 001169e8 f i atlsd:atlbase.obj
 0001:00015a3c       ?GetSize@?$CSimpleArray@PAUHINSTANCE__@@V?$CSimpleArrayEqualHelper@PAUHINSTANCE__@@@ATL@@@ATL@@QBAHXZ 00116a3c f i atlsd:atlbase.obj
 0001:00015a6c       ?Add@?$CSimpleArray@PAUHINSTANCE__@@V?$CSimpleArrayEqualHelper@PAUHINSTANCE__@@@ATL@@@ATL@@QAAHABQAUHINSTANCE__@@@Z 00116a6c f i atlsd:atlbase.obj
 0001:00015bbc       ?RemoveAt@?$CSimpleArray@PAUHINSTANCE__@@V?$CSimpleArrayEqualHelper@PAUHINSTANCE__@@@ATL@@@ATL@@QAAHH@Z 00116bbc f i atlsd:atlbase.obj
 0001:00015d34       ??A?$CSimpleArray@PAUHINSTANCE__@@V?$CSimpleArrayEqualHelper@PAUHINSTANCE__@@@ATL@@@ATL@@QAAAAPAUHINSTANCE__@@H@Z 00116d34 f i atlsd:atlbase.obj
 0001:00015e18       ?InternalSetAtIndex@?$CSimpleArray@PAUHINSTANCE__@@V?$CSimpleArrayEqualHelper@PAUHINSTANCE__@@@ATL@@@ATL@@QAAXHABQAUHINSTANCE__@@@Z 00116e18 f i atlsd:atlbase.obj
 0001:00015ea8       ??0Wrapper@?$CSimpleArray@PAUHINSTANCE__@@V?$CSimpleArrayEqualHelper@PAUHINSTANCE__@@@ATL@@@ATL@@QAA@ABQAUHINSTANCE__@@@Z 00116ea8 f i atlsd:atlbase.obj
 0001:00015ee0       ??1?$CSimpleArray@PAUHINSTANCE__@@V?$CSimpleArrayEqualHelper@PAUHINSTANCE__@@@ATL@@@ATL@@QAA@XZ 00116ee0 f i atlsd:atlbase.obj
 0001:00015f08       ??$?2PAUHINSTANCE__@@@Wrapper@?$CSimpleArray@PAUHINSTANCE__@@V?$CSimpleArrayEqualHelper@PAUHINSTANCE__@@@ATL@@@ATL@@SAPAXIPAPAUHINSTANCE__@@@Z 00116f08 f i atlsd:atlbase.obj
 0001:00015f30       ?RemoveAll@?$CSimpleArray@PAUHINSTANCE__@@V?$CSimpleArrayEqualHelper@PAUHINSTANCE__@@@ATL@@@ATL@@QAAXXZ 00116f30 f i atlsd:atlbase.obj
 0001:00015fd4       ?memmove_s@Checked@ATL@@YAXPAXIPBXI@Z 00116fd4 f i atlsd:atlbase.obj
 0001:00016028       ?AtlCrtErrorCheck@ATL@@YAHH@Z 00117028 f i atlsd:atlbase.obj
 0001:000160f4       ??1?$CComPtr@UIUnknown@@@ATL@@QAA@XZ 001170f4 f i atlsd:atlbase.obj
 0001:0001611c       ??1?$CComPtr@UIPersistStream@@@ATL@@QAA@XZ 0011711c f i atlsd:atlbase.obj
 0001:00016144       ??0?$CComPtr@UIUnknown@@@ATL@@QAA@XZ 00117144 f i atlsd:atlbase.obj
 0001:00016184       ??1?$CComPtrBase@UIUnknown@@@ATL@@QAA@XZ 00117184 f i atlsd:atlbase.obj
 0001:000161cc       ??I?$CComPtrBase@UIUnknown@@@ATL@@QAAPAPAUIUnknown@@XZ 001171cc f i atlsd:atlbase.obj
 0001:00016248       ??C?$CComPtrBase@UIUnknown@@@ATL@@QBAPAV?$_NoAddRefReleaseOnCComPtr@UIUnknown@@@1@XZ 00117248 f i atlsd:atlbase.obj
 0001:000162c8       ??0?$CComPtr@UIPersistStream@@@ATL@@QAA@XZ 001172c8 f i atlsd:atlbase.obj
 0001:00016308       ??1?$CComPtrBase@UIPersistStream@@@ATL@@QAA@XZ 00117308 f i atlsd:atlbase.obj
 0001:00016350       ??I?$CComPtrBase@UIPersistStream@@@ATL@@QAAPAPAUIPersistStream@@XZ 00117350 f i atlsd:atlbase.obj
 0001:000163cc       ??C?$CComPtrBase@UIPersistStream@@@ATL@@QBAPAV?$_NoAddRefReleaseOnCComPtr@UIPersistStream@@@1@XZ 001173cc f i atlsd:atlbase.obj
 0001:0001644c       ??0?$CComPtrBase@UIUnknown@@@ATL@@IAA@XZ 0011744c f i atlsd:atlbase.obj
 0001:00016480       ??0?$CComPtrBase@UIPersistStream@@@ATL@@IAA@XZ 00117480 f i atlsd:atlbase.obj
 0001:000164b4       ??0CTraceCategory@ATL@@QAA@PB_WI@Z 001174b4 f i atlsd:atltrace.obj
 0001:00016538       ?ChangeCategory@CTrace@ATL@@QAA_NKIW4ATLTRACESTATUS@2@@Z 00117538 f i atlsd:atltrace.obj
 0001:000165a8       ?RegisterCategory@CTrace@ATL@@QAAKPB_W@Z 001175a8 f i atlsd:atltrace.obj
 0001:000165f4       ??0CAtlAllocator@@QAA@XZ   001175f4 f i atlsd:Externs.obj
 0001:00016684       ??0CTraceSnapshot@@QAA@XZ  00117684 f i atlsd:Externs.obj
 0001:000166e0       ??0?$CSimpleArray@UCModuleInfo@CTraceSnapshot@@V?$CSimpleArrayEqualHelper@UCModuleInfo@CTraceSnapshot@@@ATL@@@ATL@@QAA@XZ 001176e0 f i atlsd:Externs.obj
 0001:00016734       ??0?$CSimpleArray@KV?$CSimpleArrayEqualHelper@K@ATL@@@ATL@@QAA@XZ 00117734 f i atlsd:Externs.obj
 0001:000168f8       GetCurrentProcessId        001178f8 f i atlsd:Externs.obj
 0001:00016918       ??0CAtlException@ATL@@QAA@J@Z 00117918 f i atlsd:Externs.obj
 0001:0001694c       ??0CTrace@ATL@@AAA@P6AHHPB_WH00ZZ@Z 0011794c f i atlsd:Externs.obj
 0001:000169d4       ??1CAtlAllocator@@QAA@XZ   001179d4 f i atlsd:Externs.obj
 0001:00016a14       ??1CTraceSnapshot@@QAA@XZ  00117a14 f i atlsd:Externs.obj
 0001:00016a54       ??1?$CSimpleArray@UCModuleInfo@CTraceSnapshot@@V?$CSimpleArrayEqualHelper@UCModuleInfo@CTraceSnapshot@@@ATL@@@ATL@@QAA@XZ 00117a54 f i atlsd:Externs.obj
 0001:00016a7c       ??1?$CSimpleArray@KV?$CSimpleArrayEqualHelper@K@ATL@@@ATL@@QAA@XZ 00117a7c f i atlsd:Externs.obj
 0001:00016aa4       ?RemoveAll@?$CSimpleArray@UCModuleInfo@CTraceSnapshot@@V?$CSimpleArrayEqualHelper@UCModuleInfo@CTraceSnapshot@@@ATL@@@ATL@@QAAXXZ 00117aa4 f i atlsd:Externs.obj
 0001:00016b48       ?RemoveAll@?$CSimpleArray@KV?$CSimpleArrayEqualHelper@K@ATL@@@ATL@@QAAXXZ 00117b48 f i atlsd:Externs.obj
 0001:00016bec       ??1CTrace@ATL@@AAA@XZ      00117bec f i atlsd:Externs.obj
 0001:00016c1c       ?NotifyTool@ATL@@YAXXZ     00117c1c f   atlsd:AtlDebugAPI.obj
 0001:00016c94       AtlTraceRegister           00117c94 f   atlsd:AtlDebugAPI.obj
 0001:00016d90       AtlTraceUnregister         00117d90 f   atlsd:AtlDebugAPI.obj
 0001:00016df0       AtlTraceRegisterCategoryU  00117df0 f   atlsd:AtlDebugAPI.obj
 0001:00016e7c       AtlTraceModifyProcess      00117e7c f   atlsd:AtlDebugAPI.obj
 0001:00016ffc       AtlTraceModifyModule       00117ffc f   atlsd:AtlDebugAPI.obj
 0001:0001719c       AtlTraceModifyCategory     0011819c f   atlsd:AtlDebugAPI.obj
 0001:000172dc       AtlTraceGetProcess         001182dc f   atlsd:AtlDebugAPI.obj
 0001:0001747c       AtlTraceGetModule          0011847c f   atlsd:AtlDebugAPI.obj
 0001:0001766c       AtlTraceGetCategory        0011866c f   atlsd:AtlDebugAPI.obj
 0001:00017810       AtlTraceGetUpdateEventNameU 00118810 f   atlsd:AtlDebugAPI.obj
 0001:00017864       AtlTraceGetUpdateEventNameU_s 00118864 f   atlsd:AtlDebugAPI.obj
 0001:000178bc       AtlTraceVU                 001188bc f   atlsd:AtlDebugAPI.obj
 0001:00017bcc       AtlTraceOpenProcess        00118bcc f   atlsd:AtlDebugAPI.obj
 0001:00017c28       AtlTraceCloseProcess       00118c28 f   atlsd:AtlDebugAPI.obj
 0001:00017d64       AtlTraceSnapshotProcess    00118d64 f   atlsd:AtlDebugAPI.obj
 0001:00017e3c       AtlTraceGetProcessInfo     00118e3c f   atlsd:AtlDebugAPI.obj
 0001:0001816c       AtlTraceGetModuleInfo      0011916c f   atlsd:AtlDebugAPI.obj
 0001:00018460       AtlTraceGetCategoryInfo    00119460 f   atlsd:AtlDebugAPI.obj
 0001:00018b18       ?GetProcess@CAtlAllocator@@QBAPAVCAtlTraceProcess@@XZ 00119b18 f i atlsd:AtlDebugAPI.obj
 0001:00018b48       ?Name@CAtlTraceCategory@@QBAPB_WXZ 00119b48 f i atlsd:AtlDebugAPI.obj
 0001:00018b74       ?Path@CAtlTraceModuleInfo@@QBAPB_WXZ 00119b74 f i atlsd:AtlDebugAPI.obj
 0001:00018ba0       ?Name@CAtlTraceModuleInfo@@QBAPB_WXZ 00119ba0 f i atlsd:AtlDebugAPI.obj
 0001:00018bcc       ?Id@CAtlTraceProcess@@QBAKXZ 00119bcc f i atlsd:AtlDebugAPI.obj
 0001:00018c00       ?CrtDbgReport@CAtlTraceModule@@QBAP6AHHPB_WH00ZZXZ 00119c00 f i atlsd:AtlDebugAPI.obj
 0001:00018c34       ?GetSize@?$CSimpleArray@UCModuleInfo@CTraceSnapshot@@V?$CSimpleArrayEqualHelper@UCModuleInfo@CTraceSnapshot@@@ATL@@@ATL@@QBAHXZ 00119c34 f i atlsd:AtlDebugAPI.obj
 0001:00018c64       ??A?$CSimpleArray@UCModuleInfo@CTraceSnapshot@@V?$CSimpleArrayEqualHelper@UCModuleInfo@CTraceSnapshot@@@ATL@@@ATL@@QAAAAUCModuleInfo@CTraceSnapshot@@H@Z 00119c64 f i atlsd:AtlDebugAPI.obj
 0001:00018d48       ?wcscpy_s@Checked@ATL@@YAXPA_WIPB_W@Z 00119d48 f i atlsd:AtlDebugAPI.obj
 0001:00018da0       ?Init@CAtlAllocator@@QAA_NPB_WK@Z 00119da0 f   atlsd:Allocate.obj
 0001:00019278       ?Close@CAtlAllocator@@QAAX_N@Z 0011a278 f   atlsd:Allocate.obj
 0001:00019348       ?GetModule@CAtlAllocator@@QBAPAVCAtlTraceModule@@H@Z 0011a348 f   atlsd:Allocate.obj
 0001:0001945c       ?GetCategory@CAtlAllocator@@QBAPAVCAtlTraceCategory@@H@Z 0011a45c f   atlsd:Allocate.obj
 0001:000195a4       ?GetCategoryCount@CAtlAllocator@@QBAHH@Z 0011a5a4 f   atlsd:Allocate.obj
 0001:0001967c       ?GetCategoryCount@CAtlAllocator@@QBAHABVCAtlTraceModule@@@Z 0011a67c f   atlsd:Allocate.obj
 0001:00019718       ?GetModuleCount@CAtlAllocator@@QBAHXZ 0011a718 f   atlsd:Allocate.obj
 0001:000197b8       ?FindModule@CAtlAllocator@@QBA_NPB_WPAI@Z 0011a7b8 f   atlsd:Allocate.obj
 0001:000198ac       ?AddModule@CAtlAllocator@@QAAHPAUHINSTANCE__@@@Z 0011a8ac f   atlsd:Allocate.obj
 0001:00019bf4       ?AddCategory@CAtlAllocator@@QAAHHPB_W@Z 0011abf4 f   atlsd:Allocate.obj
 0001:00019ffc       ?RemoveModule@CAtlAllocator@@QAA_NH@Z 0011affc f   atlsd:Allocate.obj
 0001:0001a130       ?CleanUp@CAtlAllocator@@QAAXXZ 0011b130 f   atlsd:Allocate.obj
 0001:0001a15c       ?TakeSnapshot@CAtlAllocator@@QAAXXZ 0011b15c f   atlsd:Allocate.obj
 0001:0001a498       ?ReleaseSnapshot@CAtlAllocator@@QAAXXZ 0011b498 f   atlsd:Allocate.obj
 0001:0001a638       ?IncRef@CAtlTraceProcess@@QAAIXZ 0011b638 f i atlsd:Allocate.obj
 0001:0001a690       ?Base@CAtlTraceProcess@@QBAPAXXZ 0011b690 f i atlsd:Allocate.obj
 0001:0001a6c4       ?DecRef@CAtlTraceProcess@@QAAIXZ 0011b6c4 f i atlsd:Allocate.obj
 0001:0001a71c       ?ModuleCount@CAtlTraceProcess@@QBAHXZ 0011b71c f i atlsd:Allocate.obj
 0001:0001a750       ?MaxSize@CAtlTraceProcess@@QBAKXZ 0011b750 f i atlsd:Allocate.obj
 0001:0001a780       ?CategoryCount@CAtlTraceProcess@@QBAHXZ 0011b780 f i atlsd:Allocate.obj
 0001:0001a7b0       ?TryAllocate@CAtlTraceSettings@@QAA_NXZ 0011b7b0 f i atlsd:Allocate.obj
 0001:0001a834       ?MarkValid@CAtlTraceSettings@@QAAXJ@Z 0011b834 f i atlsd:Allocate.obj
 0001:0001a8b0       ?IncModuleCount@CAtlTraceProcess@@QAAXI@Z 0011b8b0 f i atlsd:Allocate.obj
 0001:0001a8ec       ?TryAddRef@CAtlTraceSettings@@QAA_NXZ 0011b8ec f i atlsd:Allocate.obj
 0001:0001a97c       ?Release@CAtlTraceSettings@@QAAXXZ 0011b97c f i atlsd:Allocate.obj
 0001:0001a9d8       ?IncCategoryCount@CAtlTraceProcess@@QAAXI@Z 0011b9d8 f i atlsd:Allocate.obj
 0001:0001aa0c       ?Add@?$CSimpleArray@UCModuleInfo@CTraceSnapshot@@V?$CSimpleArrayEqualHelper@UCModuleInfo@CTraceSnapshot@@@ATL@@@ATL@@QAAHABUCModuleInfo@CTraceSnapshot@@@Z 0011ba0c f i atlsd:Allocate.obj
 0001:0001ab64       ?GetSize@?$CSimpleArray@KV?$CSimpleArrayEqualHelper@K@ATL@@@ATL@@QBAHXZ 0011bb64 f i atlsd:Allocate.obj
 0001:0001ab94       ?Add@?$CSimpleArray@KV?$CSimpleArrayEqualHelper@K@ATL@@@ATL@@QAAHABK@Z 0011bb94 f i atlsd:Allocate.obj
 0001:0001ace4       ?RemoveAt@?$CSimpleArray@KV?$CSimpleArrayEqualHelper@K@ATL@@@ATL@@QAAHH@Z 0011bce4 f i atlsd:Allocate.obj
 0001:0001ae5c       ??A?$CSimpleArray@KV?$CSimpleArrayEqualHelper@K@ATL@@@ATL@@QAAAAKH@Z 0011be5c f i atlsd:Allocate.obj
 0001:0001af40       ?InternalSetAtIndex@?$CSimpleArray@UCModuleInfo@CTraceSnapshot@@V?$CSimpleArrayEqualHelper@UCModuleInfo@CTraceSnapshot@@@ATL@@@ATL@@QAAXHABUCModuleInfo@CTraceSnapshot@@@Z 0011bf40 f i atlsd:Allocate.obj
 0001:0001afd0       ?InternalSetAtIndex@?$CSimpleArray@KV?$CSimpleArrayEqualHelper@K@ATL@@@ATL@@QAAXHABK@Z 0011bfd0 f i atlsd:Allocate.obj
 0001:0001b060       ??0Wrapper@?$CSimpleArray@UCModuleInfo@CTraceSnapshot@@V?$CSimpleArrayEqualHelper@UCModuleInfo@CTraceSnapshot@@@ATL@@@ATL@@QAA@ABUCModuleInfo@CTraceSnapshot@@@Z 0011c060 f i atlsd:Allocate.obj
 0001:0001b098       ??0Wrapper@?$CSimpleArray@KV?$CSimpleArrayEqualHelper@K@ATL@@@ATL@@QAA@ABK@Z 0011c098 f i atlsd:Allocate.obj
 0001:0001b0d0       ??$?2UCModuleInfo@CTraceSnapshot@@@Wrapper@?$CSimpleArray@UCModuleInfo@CTraceSnapshot@@V?$CSimpleArrayEqualHelper@UCModuleInfo@CTraceSnapshot@@@ATL@@@ATL@@SAPAXIPAUCModuleInfo@CTraceSnapshot@@@Z 0011c0d0 f i atlsd:Allocate.obj
 0001:0001b0f8       ??$?2K@Wrapper@?$CSimpleArray@KV?$CSimpleArrayEqualHelper@K@ATL@@@ATL@@SAPAXIPAK@Z 0011c0f8 f i atlsd:Allocate.obj
 0001:0001b120       ??0CAtlTraceModuleInfo@@QAA@XZ 0011c120 f   atlsd:AtlTraceModuleManager.obj
 0001:0001b194       ?Reset@CAtlTraceModuleInfo@@QAAXPAUHINSTANCE__@@@Z 0011c194 f   atlsd:AtlTraceModuleManager.obj
 0001:0001b330       ??0CAtlTraceCategory@@QAA@XZ 0011c330 f   atlsd:AtlTraceModuleManager.obj
 0001:0001b39c       ?Reset@CAtlTraceCategory@@QAAXPB_WJ@Z 0011c39c f   atlsd:AtlTraceModuleManager.obj
 0001:0001b41c       ??0CAtlTraceModule@@QAA@XZ 0011c41c f   atlsd:AtlTraceModuleManager.obj
 0001:0001b488       ?CrtDbgReport@CAtlTraceModule@@QAAXP6AHHPB_WH00ZZ@Z 0011c488 f   atlsd:AtlTraceModuleManager.obj
 0001:0001b4dc       ??0CAtlTraceProcess@@QAA@K@Z 0011c4dc f   atlsd:AtlTraceModuleManager.obj
 0001:0001b654       ?GetNextCookie@CAtlTraceProcess@@QAAJXZ 0011c654 f   atlsd:AtlTraceModuleManager.obj
 0001:0001b69c       ??0CAtlTraceSettings@@QAA@XZ 0011c69c f i atlsd:AtlTraceModuleManager.obj
 0001:0001b700       __report_gsfailure         0011c700 f   coredll:COREDLL.dll
 0001:0001b710       LocalReAlloc               0011c710 f   coredll:COREDLL.dll
 0001:0001b720       LocalAlloc                 0011c720 f   coredll:COREDLL.dll
 0001:0001b730       LocalSize                  0011c730 f   coredll:COREDLL.dll
 0001:0001b740       LocalFree                  0011c740 f   coredll:COREDLL.dll
 0001:0001b750       __security_gen_cookie      0011c750 f   coredll:COREDLL.dll
 0001:0001b760       strcmp                     0011c760 f   coredll:COREDLL.dll
 0001:0001b770       __C_specific_handler       0011c770 f   coredll:COREDLL.dll
 0001:0001b780       ?terminate@std@@YAXXZ      0011c780 f   coredll:COREDLL.dll
 0001:0001b790       memmove                    0011c790 f   coredll:COREDLL.dll
 0001:0001b7a0       malloc                     0011c7a0 f   coredll:COREDLL.dll
 0001:0001b7b0       _snwprintf                 0011c7b0 f   coredll:COREDLL.dll
 0001:0001b7c0       GetModuleFileNameW         0011c7c0 f   coredll:COREDLL.dll
 0001:0001b7d0       TlsSetValue                0011c7d0 f   coredll:COREDLL.dll
 0001:0001b7e0       TlsGetValue                0011c7e0 f   coredll:COREDLL.dll
 0001:0001b7f0       InterlockedCompareExchange 0011c7f0 f   coredll:COREDLL.dll
 0001:0001b800       TlsCall                    0011c800 f   coredll:COREDLL.dll
 0001:0001b810       EnterCriticalSection       0011c810 f   coredll:COREDLL.dll
 0001:0001b820       LeaveCriticalSection       0011c820 f   coredll:COREDLL.dll
 0001:0001b830       InterlockedDecrement       0011c830 f   coredll:COREDLL.dll
 0001:0001b840       WriteFile                  0011c840 f   coredll:COREDLL.dll
 0001:0001b850       wcstombs                   0011c850 f   coredll:COREDLL.dll
 0001:0001b860       _vsnwprintf                0011c860 f   coredll:COREDLL.dll
 0001:0001b870       OutputDebugStringW         0011c870 f   coredll:COREDLL.dll
 0001:0001b880       InterlockedIncrement       0011c880 f   coredll:COREDLL.dll
 0001:0001b890       GetProcAddressW            0011c890 f   coredll:COREDLL.dll
 0001:0001b8a0       LoadLibraryW               0011c8a0 f   coredll:COREDLL.dll
 0001:0001b8b0       SetLastError               0011c8b0 f   coredll:COREDLL.dll
 0001:0001b8c0       InitializeCriticalSection  0011c8c0 f   coredll:COREDLL.dll
 0001:0001b8d0       fputs                      0011c8d0 f   coredll:COREDLL.dll
 0001:0001b8e0       _getstdfilex               0011c8e0 f   coredll:COREDLL.dll
 0001:0001b8f0       fflush                     0011c8f0 f   coredll:COREDLL.dll
 0001:0001b900       InterlockedExchange        0011c900 f   coredll:COREDLL.dll
 0001:0001b910       WaitForSingleObject        0011c910 f   coredll:COREDLL.dll
 0001:0001b920       DispatchMessageW           0011c920 f   coredll:COREDLL.dll
 0001:0001b930       TranslateMessage           0011c930 f   coredll:COREDLL.dll
 0001:0001b940       GetMessageW                0011c940 f   coredll:COREDLL.dll
 0001:0001b950       PeekMessageW               0011c950 f   coredll:COREDLL.dll
 0001:0001b960       MsgWaitForMultipleObjectsEx 0011c960 f   coredll:COREDLL.dll
 0001:0001b970       GetModuleHandleW           0011c970 f   coredll:COREDLL.dll
 0001:0001b980       realloc                    0011c980 f   coredll:COREDLL.dll
 0001:0001b990       CloseHandle                0011c990 f   coredll:COREDLL.dll
 0001:0001b9a0       OpenEventW                 0011c9a0 f   coredll:COREDLL.dll
 0001:0001b9b0       VirtualAlloc               0011c9b0 f   coredll:COREDLL.dll
 0001:0001b9c0       UnmapViewOfFile            0011c9c0 f   coredll:COREDLL.dll
 0001:0001b9d0       GetSystemInfo              0011c9d0 f   coredll:COREDLL.dll
 0001:0001b9e0       MapViewOfFile              0011c9e0 f   coredll:COREDLL.dll
 0001:0001b9f0       CreateFileMappingW         0011c9f0 f   coredll:COREDLL.dll
 0001:0001ba00       _wcsicmp                   0011ca00 f   coredll:COREDLL.dll
 0001:0001ba10       CreateStreamOnHGlobal      0011ca10 f   ole32:ole32.dll
 0001:0001ba20       WriteClassStm              0011ca20 f   ole32:ole32.dll
 0001:0001ba30       CoCreateInstance           0011ca30 f   ole32:ole32.dll
 0001:0001ba40       ReadClassStm               0011ca40 f   ole32:ole32.dll
 0002:000000e8       ??_7CSWContextMenuClassFactory@@6B@ 0011e0e8     clsfact.obj
 0002:00000100       CLSID_ShellDesktop         0011e100     DialParsExtOEM.obj
 0002:00000110       IID_IContextMenu           0011e110     DialParsExtOEM.obj
 0002:00000120       IID_IShellFolder           0011e120     DialParsExtOEM.obj
 0002:00000130       IID_IShellExtInit          0011e130     DialParsExtOEM.obj
 0002:00000140       IID_IShellPropSheetExt     0011e140     DialParsExtOEM.obj
 0002:00000150       IID_IEnumIDList            0011e150     DialParsExtOEM.obj
 0002:00000160       IID_IShellCommandUI        0011e160     DialParsExtOEM.obj
 0002:00000170       IID_IShellListView         0011e170     DialParsExtOEM.obj
 0002:00000180       IID_IShellFind             0011e180     DialParsExtOEM.obj
 0002:00000190       IID_IShellFindItem         0011e190     DialParsExtOEM.obj
 0002:000001a0       IID_IShellFindCallback     0011e1a0     DialParsExtOEM.obj
 0002:000001b0       IID_IShellNotificationCallback 0011e1b0     DialParsExtOEM.obj
 0002:000001c0       IID_INewMenuItemServer     0011e1c0     DialParsExtOEM.obj
 0002:000001d0       IID_IAutoSuggestionGenerator 0011e1d0     DialParsExtOEM.obj
 0002:000001f0       CLSID_CSWContextMenu       0011e1f0     DialParsExtOEM.obj
 0002:00002050       ??_7Csw_ctxMenu@@6BIObjectWithSite@@@ 00120050     DialParsExtOEM.obj
 0002:00002064       ??_7Csw_ctxMenu@@6BIContextMenu@@@ 00120064     DialParsExtOEM.obj
 0002:0000207c       ??_7IContextMenu@@6B@      0012007c     DialParsExtOEM.obj
 0002:00002094       ??_7IObjectWithSite@@6B@   00120094     DialParsExtOEM.obj
 0002:000022b4       ?_Min@?$AtlLimits@H@ATL@@2HB 001202b4     resultelement.obj
 0002:000022b8       ?_Max@?$AtlLimits@H@ATL@@2HB 001202b8     resultelement.obj
 0002:000022bc       ?_Min@?$AtlLimits@I@ATL@@2IB 001202bc     resultelement.obj
 0002:000022c0       ?_Max@?$AtlLimits@I@ATL@@2IB 001202c0     resultelement.obj
 0002:000022c4       ?_Min@?$AtlLimits@J@ATL@@2JB 001202c4     resultelement.obj
 0002:000022c8       ?_Max@?$AtlLimits@J@ATL@@2JB 001202c8     resultelement.obj
 0002:000022cc       ?_Min@?$AtlLimits@K@ATL@@2KB 001202cc     resultelement.obj
 0002:000022d0       ?_Max@?$AtlLimits@K@ATL@@2KB 001202d0     resultelement.obj
 0002:000022d8       ?_Min@?$AtlLimits@_J@ATL@@2_JB 001202d8     resultelement.obj
 0002:000022e0       ?_Max@?$AtlLimits@_J@ATL@@2_JB 001202e0     resultelement.obj
 0002:000022e8       ?_Min@?$AtlLimits@_K@ATL@@2_KB 001202e8     resultelement.obj
 0002:000022f0       ?_Max@?$AtlLimits@_K@ATL@@2_KB 001202f0     resultelement.obj
 0002:000022f8       ?VT@?$CVarTypeInfo@D@ATL@@2GB 001202f8     resultelement.obj
 0002:000022fc       ?pmField@?$CVarTypeInfo@D@ATL@@2QQtagVARIANT@@DQ3@ 001202fc     resultelement.obj
 0002:00002300       ?VT@?$CVarTypeInfo@E@ATL@@2GB 00120300     resultelement.obj
 0002:00002304       ?pmField@?$CVarTypeInfo@E@ATL@@2QQtagVARIANT@@EQ3@ 00120304     resultelement.obj
 0002:00002308       ?VT@?$CVarTypeInfo@PAD@ATL@@2GB 00120308     resultelement.obj
 0002:0000230c       ?pmField@?$CVarTypeInfo@PAD@ATL@@2QQtagVARIANT@@PADQ3@ 0012030c     resultelement.obj
 0002:00002310       ?VT@?$CVarTypeInfo@PAE@ATL@@2GB 00120310     resultelement.obj
 0002:00002314       ?pmField@?$CVarTypeInfo@PAE@ATL@@2QQtagVARIANT@@PAEQ3@ 00120314     resultelement.obj
 0002:00002318       ?VT@?$CVarTypeInfo@F@ATL@@2GB 00120318     resultelement.obj
 0002:0000231c       ?pmField@?$CVarTypeInfo@F@ATL@@2QQtagVARIANT@@FQ3@ 0012031c     resultelement.obj
 0002:00002320       ?VT@?$CVarTypeInfo@PAF@ATL@@2GB 00120320     resultelement.obj
 0002:00002324       ?pmField@?$CVarTypeInfo@PAF@ATL@@2QQtagVARIANT@@PAFQ3@ 00120324     resultelement.obj
 0002:00002328       ?VT@?$CVarTypeInfo@G@ATL@@2GB 00120328     resultelement.obj
 0002:0000232c       ?pmField@?$CVarTypeInfo@G@ATL@@2QQtagVARIANT@@GQ3@ 0012032c     resultelement.obj
 0002:00002330       ?VT@?$CVarTypeInfo@H@ATL@@2GB 00120330     resultelement.obj
 0002:00002334       ?pmField@?$CVarTypeInfo@H@ATL@@2QQtagVARIANT@@HQ3@ 00120334     resultelement.obj
 0002:00002338       ?VT@?$CVarTypeInfo@PAH@ATL@@2GB 00120338     resultelement.obj
 0002:0000233c       ?pmField@?$CVarTypeInfo@PAH@ATL@@2QQtagVARIANT@@PAHQ3@ 0012033c     resultelement.obj
 0002:00002340       ?VT@?$CVarTypeInfo@I@ATL@@2GB 00120340     resultelement.obj
 0002:00002344       ?pmField@?$CVarTypeInfo@I@ATL@@2QQtagVARIANT@@IQ3@ 00120344     resultelement.obj
 0002:00002348       ?VT@?$CVarTypeInfo@PAI@ATL@@2GB 00120348     resultelement.obj
 0002:0000234c       ?pmField@?$CVarTypeInfo@PAI@ATL@@2QQtagVARIANT@@PAIQ3@ 0012034c     resultelement.obj
 0002:00002350       ?VT@?$CVarTypeInfo@J@ATL@@2GB 00120350     resultelement.obj
 0002:00002354       ?pmField@?$CVarTypeInfo@J@ATL@@2QQtagVARIANT@@JQ3@ 00120354     resultelement.obj
 0002:00002358       ?VT@?$CVarTypeInfo@PAJ@ATL@@2GB 00120358     resultelement.obj
 0002:0000235c       ?pmField@?$CVarTypeInfo@PAJ@ATL@@2QQtagVARIANT@@PAJQ3@ 0012035c     resultelement.obj
 0002:00002360       ?VT@?$CVarTypeInfo@K@ATL@@2GB 00120360     resultelement.obj
 0002:00002364       ?pmField@?$CVarTypeInfo@K@ATL@@2QQtagVARIANT@@KQ3@ 00120364     resultelement.obj
 0002:00002368       ?VT@?$CVarTypeInfo@PAK@ATL@@2GB 00120368     resultelement.obj
 0002:0000236c       ?pmField@?$CVarTypeInfo@PAK@ATL@@2QQtagVARIANT@@PAKQ3@ 0012036c     resultelement.obj
 0002:00002370       ?VT@?$CVarTypeInfo@M@ATL@@2GB 00120370     resultelement.obj
 0002:00002374       ?pmField@?$CVarTypeInfo@M@ATL@@2QQtagVARIANT@@MQ3@ 00120374     resultelement.obj
 0002:00002378       ?VT@?$CVarTypeInfo@PAM@ATL@@2GB 00120378     resultelement.obj
 0002:0000237c       ?pmField@?$CVarTypeInfo@PAM@ATL@@2QQtagVARIANT@@PAMQ3@ 0012037c     resultelement.obj
 0002:00002380       ?VT@?$CVarTypeInfo@N@ATL@@2GB 00120380     resultelement.obj
 0002:00002384       ?pmField@?$CVarTypeInfo@N@ATL@@2QQtagVARIANT@@NQ3@ 00120384     resultelement.obj
 0002:00002388       ?VT@?$CVarTypeInfo@PAN@ATL@@2GB 00120388     resultelement.obj
 0002:0000238c       ?pmField@?$CVarTypeInfo@PAN@ATL@@2QQtagVARIANT@@PANQ3@ 0012038c     resultelement.obj
 0002:00002390       ?VT@?$CVarTypeInfo@UtagVARIANT@@@ATL@@2GB 00120390     resultelement.obj
 0002:00002394       ?VT@?$CVarTypeInfo@PAG@ATL@@2GB 00120394     resultelement.obj
 0002:00002398       ?pmField@?$CVarTypeInfo@PAG@ATL@@2QQtagVARIANT@@PAGQ3@ 00120398     resultelement.obj
 0002:0000239c       ?VT@?$CVarTypeInfo@PAPAG@ATL@@2GB 0012039c     resultelement.obj
 0002:000023a0       ?pmField@?$CVarTypeInfo@PAPAG@ATL@@2QQtagVARIANT@@PAPAGQ3@ 001203a0     resultelement.obj
 0002:000023a4       ?VT@?$CVarTypeInfo@PAUIUnknown@@@ATL@@2GB 001203a4     resultelement.obj
 0002:000023a8       ?pmField@?$CVarTypeInfo@PAUIUnknown@@@ATL@@2QQtagVARIANT@@PAUIUnknown@@Q3@ 001203a8     resultelement.obj
 0002:000023ac       ?VT@?$CVarTypeInfo@PAPAUIUnknown@@@ATL@@2GB 001203ac     resultelement.obj
 0002:000023b0       ?pmField@?$CVarTypeInfo@PAPAUIUnknown@@@ATL@@2QQtagVARIANT@@PAPAUIUnknown@@Q3@ 001203b0     resultelement.obj
 0002:000023b4       ?VT@?$CVarTypeInfo@PAUIDispatch@@@ATL@@2GB 001203b4     resultelement.obj
 0002:000023b8       ?pmField@?$CVarTypeInfo@PAUIDispatch@@@ATL@@2QQtagVARIANT@@PAUIDispatch@@Q3@ 001203b8     resultelement.obj
 0002:000023bc       ?VT@?$CVarTypeInfo@PAPAUIDispatch@@@ATL@@2GB 001203bc     resultelement.obj
 0002:000023c0       ?pmField@?$CVarTypeInfo@PAPAUIDispatch@@@ATL@@2QQtagVARIANT@@PAPAUIDispatch@@Q3@ 001203c0     resultelement.obj
 0002:000023c4       ?VT@?$CVarTypeInfo@TtagCY@@@ATL@@2GB 001203c4     resultelement.obj
 0002:000023c8       ?pmField@?$CVarTypeInfo@TtagCY@@@ATL@@2QQtagVARIANT@@TtagCY@@Q3@ 001203c8     resultelement.obj
 0002:000023cc       ?VT@?$CVarTypeInfo@PATtagCY@@@ATL@@2GB 001203cc     resultelement.obj
 0002:000023d0       ?pmField@?$CVarTypeInfo@PATtagCY@@@ATL@@2QQtagVARIANT@@PATtagCY@@Q3@ 001203d0     resultelement.obj
 0002:000023d4       LIBID_ATLLib               001203d4     resultelement.obj
 0002:000023e4       CLSID_Registrar            001203e4     resultelement.obj
 0002:000023f4       IID_IRegistrar             001203f4     resultelement.obj
 0002:00002404       IID_IAxWinHostWindow       00120404     resultelement.obj
 0002:00002414       IID_IAxWinAmbientDispatch  00120414     resultelement.obj
 0002:00002424       IID_IInternalConnection    00120424     resultelement.obj
 0002:00002434       IID_IDocHostUIHandlerDispatch 00120434     resultelement.obj
 0002:00002444       IID_IAxWinHostWindowLic    00120444     resultelement.obj
 0002:00002454       IID_IAxWinAmbientDispatchEx 00120454     resultelement.obj
 0002:00002464       ?MAX_VALUE@CRegParser@ATL@@1HB 00120464     resultelement.obj
 0002:00002468       ?MAX_TYPE@CRegParser@ATL@@1HB 00120468     resultelement.obj
 0002:0000246c       ?rgszNeverDelete@CRegParser@ATL@@1QBQBGB 0012046c     resultelement.obj
 0002:0000249c       ?cbNeverDelete@CRegParser@ATL@@1HB 0012049c     resultelement.obj
 0002:000024a0       ??_7CResultListElement@@6B@ 001204a0     resultelement.obj
 0002:000024a8       ??_C@_1JE@NABCONDI@?$AAC?$AA?3?$AA?2?$AAP?$AAr?$AAo?$AAg?$AAr?$AAa?$AAm?$AA?5?$AAF?$AAi?$AAl?$AAe?$AAs?$AA?2?$AAM?$AAi?$AAc?$AAr?$AAo?$AAs?$AAo?$AAf?$AAt?$AA?5?$AAV?$AAi?$AAs?$AAu?$AAa@ 001204a8     resultelement.obj
 0002:0000253c       ??_C@_13COJANIEC@?$AA0?$AA?$AA@ 0012053c     resultelement.obj
 0002:000025f8       ??_C@_1JM@HGDAICHJ@?$AAC?$AA?3?$AA?2?$AAP?$AAr?$AAo?$AAg?$AAr?$AAa?$AAm?$AA?5?$AAF?$AAi?$AAl?$AAe?$AAs?$AA?2?$AAM?$AAi?$AAc?$AAr?$AAo?$AAs?$AAo?$AAf?$AAt?$AA?5?$AAV?$AAi?$AAs?$AAu?$AAa@ 001205f8     resultelement.obj
 0002:00002698       ??_C@_1EA@JHMKKLFC@?$AAn?$AAI?$AAn?$AAd?$AAe?$AAx?$AA?5?$AA?$DO?$AA?$DN?$AA?5?$AA0?$AA?5?$AA?$CG?$AA?$CG?$AA?5?$AAn?$AAI?$AAn?$AAd?$AAe?$AAx?$AA?5?$AA?$DM?$AA?5?$AAm?$AA_?$AAn?$AAS?$AAi?$AAz?$AAe?$AA?$AA@ 00120698     resultelement.obj
 0002:00005e8c       ??_7CModemStatus@@6B@      00123e8c     winmodemstat.obj
 0002:00005ecc       ??_C@_1DC@POOIKBAO@?$AAI?$AAT?$AAE?$AAR?$AAA?$AAT?$AAO?$AAR?$AA?5?$AAL?$AAI?$AAS?$AAT?$AA?5?$AAC?$AAO?$AAR?$AAR?$AAU?$AAP?$AAT?$AAE?$AAD?$AA?$CB?$AA?$AA@ 00123ecc     winmodemstat.obj
 0002:00005f00       ??_C@_1IE@BKKAAKCG@?$AAC?$AA?3?$AA?2?$AAP?$AAr?$AAo?$AAg?$AAr?$AAa?$AAm?$AA?5?$AAF?$AAi?$AAl?$AAe?$AAs?$AA?2?$AAM?$AAi?$AAc?$AAr?$AAo?$AAs?$AAo?$AAf?$AAt?$AA?5?$AAV?$AAi?$AAs?$AAu?$AAa@ 00123f00     winmodemstat.obj
 0002:00006050       ??_C@_1EE@BBMFLDOC@?$AAl?$AAi?$AAs?$AAt?$AA?5?$AAe?$AAr?$AAa?$AAs?$AAe?$AA?5?$AAi?$AAt?$AAe?$AAr?$AAa?$AAt?$AAo?$AAr?$AA?5?$AAo?$AAu?$AAt?$AAs?$AAi?$AAd?$AAe?$AA?5?$AAr?$AAa?$AAn?$AAg@ 00124050     winmodemstat.obj
 0002:00006098       ??_C@_1HM@HPOOGGJN@?$AAC?$AA?3?$AA?2?$AAP?$AAr?$AAo?$AAg?$AAr?$AAa?$AAm?$AA?5?$AAF?$AAi?$AAl?$AAe?$AAs?$AA?2?$AAM?$AAi?$AAc?$AAr?$AAo?$AAs?$AAo?$AAf?$AAt?$AA?5?$AAV?$AAi?$AAs?$AAu?$AAa@ 00124098     winmodemstat.obj
 0002:000061c0       ??_C@_1EG@BPNHNPIG@?$AAl?$AAi?$AAs?$AAt?$AA?5?$AAi?$AAn?$AAs?$AAe?$AAr?$AAt?$AA?5?$AAi?$AAt?$AAe?$AAr?$AAa?$AAt?$AAo?$AAr?$AA?5?$AAo?$AAu?$AAt?$AAs?$AAi?$AAd?$AAe?$AA?5?$AAr?$AAa?$AAn@ 001241c0     winmodemstat.obj
 0002:00006244       ??_C@_1BO@MEPPHOO@?$AA?$CC?$AAo?$AAu?$AAt?$AA?5?$AAo?$AAf?$AA?5?$AAr?$AAa?$AAn?$AAg?$AAe?$AA?$CC?$AA?$AA@ 00124244     winmodemstat.obj
 0002:00006268       ??_C@_1OI@CFPJBECN@?$AAs?$AAt?$AAd?$AA?3?$AA?3?$AAl?$AAi?$AAs?$AAt?$AA?$DM?$AAc?$AAl?$AAa?$AAs?$AAs?$AA?5?$AAC?$AAR?$AAe?$AAs?$AAu?$AAl?$AAt?$AAL?$AAi?$AAs?$AAt?$AAE?$AAl?$AAe?$AAm?$AAe@ 00124268     winmodemstat.obj
 0002:00006350       ??_C@_1FG@CMLDHNON@?$AA?$CI?$AA?$CC?$AAS?$AAt?$AAa?$AAn?$AAd?$AAa?$AAr?$AAd?$AA?5?$AAC?$AA?$CL?$AA?$CL?$AA?5?$AAL?$AAi?$AAb?$AAr?$AAa?$AAr?$AAi?$AAe?$AAs?$AA?5?$AAO?$AAu?$AAt?$AA?5?$AAo?$AAf?$AA?5@ 00124350     winmodemstat.obj
 0002:000063a8       ??_C@_1EC@HILJLMMC@?$AAl?$AAi?$AAs?$AAt?$AA?5?$AAi?$AAt?$AAe?$AAr?$AAa?$AAt?$AAo?$AAr?$AA?5?$AAn?$AAo?$AAt?$AA?5?$AAd?$AAe?$AAr?$AAe?$AAf?$AAe?$AAr?$AAe?$AAn?$AAc?$AAa?$AAb?$AAl?$AAe@ 001243a8     winmodemstat.obj
 0002:0000645c       ??_C@_0BB@MOGOBHAF@list?$DMT?$DO?5too?5long?$AA@ 0012445c     winmodemstat.obj
 0002:000064e4       ?npos@?$basic_string@DU?$char_traits@D@std@@V?$allocator@D@2@@std@@2IB 001244e4     winmodemstat.obj
 0002:00006598       ??_C@_1OK@IGJPFAPB@?$AAs?$AAt?$AAd?$AA?3?$AA?3?$AAl?$AAi?$AAs?$AAt?$AA?$DM?$AAc?$AAl?$AAa?$AAs?$AAs?$AA?5?$AAC?$AAR?$AAe?$AAs?$AAu?$AAl?$AAt?$AAL?$AAi?$AAs?$AAt?$AAE?$AAl?$AAe?$AAm?$AAe@ 00124598     winmodemstat.obj
 0002:00006688       ??_C@_1EA@DOGAGKDH@?$AAl?$AAi?$AAs?$AAt?$AA?5?$AAi?$AAt?$AAe?$AAr?$AAa?$AAt?$AAo?$AAr?$AA?5?$AAn?$AAo?$AAt?$AA?5?$AAi?$AAn?$AAc?$AAr?$AAe?$AAm?$AAe?$AAn?$AAt?$AAa?$AAb?$AAl?$AAe?$AA?$AA@ 00124688     winmodemstat.obj
 0002:000066c8       ??_C@_1OK@HFKNOMDA@?$AAs?$AAt?$AAd?$AA?3?$AA?3?$AAl?$AAi?$AAs?$AAt?$AA?$DM?$AAc?$AAl?$AAa?$AAs?$AAs?$AA?5?$AAC?$AAR?$AAe?$AAs?$AAu?$AAl?$AAt?$AAL?$AAi?$AAs?$AAt?$AAE?$AAl?$AAe?$AAm?$AAe@ 001246c8     winmodemstat.obj
 0002:000067b8       ??_C@_1EA@JDNDELPC@?$AAl?$AAi?$AAs?$AAt?$AA?5?$AAi?$AAt?$AAe?$AAr?$AAa?$AAt?$AAo?$AAr?$AA?5?$AAn?$AAo?$AAt?$AA?5?$AAd?$AAe?$AAc?$AAr?$AAe?$AAm?$AAe?$AAn?$AAt?$AAa?$AAb?$AAl?$AAe?$AA?$AA@ 001247b8     winmodemstat.obj
 0002:000067f8       ??_C@_1CG@JNLFBNGN@?$AA?$CC?$AAi?$AAn?$AAv?$AAa?$AAl?$AAi?$AAd?$AA?5?$AAa?$AAr?$AAg?$AAu?$AAm?$AAe?$AAn?$AAt?$AA?$CC?$AA?$AA@ 001247f8     winmodemstat.obj
 0002:00006820       ??_C@_1OC@OBKBLNGA@?$AAs?$AAt?$AAd?$AA?3?$AA?3?$AAl?$AAi?$AAs?$AAt?$AA?$DM?$AAc?$AAl?$AAa?$AAs?$AAs?$AA?5?$AAC?$AAR?$AAe?$AAs?$AAu?$AAl?$AAt?$AAL?$AAi?$AAs?$AAt?$AAE?$AAl?$AAe?$AAm?$AAe@ 00124820     winmodemstat.obj
 0002:00006908       ??_C@_1FO@OCPOOAIA@?$AA?$CI?$AA?$CC?$AAS?$AAt?$AAa?$AAn?$AAd?$AAa?$AAr?$AAd?$AA?5?$AAC?$AA?$CL?$AA?$CL?$AA?5?$AAL?$AAi?$AAb?$AAr?$AAa?$AAr?$AAi?$AAe?$AAs?$AA?5?$AAI?$AAn?$AAv?$AAa?$AAl?$AAi?$AAd@ 00124908     winmodemstat.obj
 0002:00006968       ??_C@_1DI@MDELDGPI@?$AAl?$AAi?$AAs?$AAt?$AA?5?$AAi?$AAt?$AAe?$AAr?$AAa?$AAt?$AAo?$AAr?$AAs?$AA?5?$AAi?$AAn?$AAc?$AAo?$AAm?$AAp?$AAa?$AAt?$AAi?$AAb?$AAl?$AAe?$AA?$AA@ 00124968     winmodemstat.obj
 0002:00006ac8       ??_C@_1IC@HKDJIJDA@?$AAC?$AA?3?$AA?2?$AAP?$AAr?$AAo?$AAg?$AAr?$AAa?$AAm?$AA?5?$AAF?$AAi?$AAl?$AAe?$AAs?$AA?2?$AAM?$AAi?$AAc?$AAr?$AAo?$AAs?$AAo?$AAf?$AAt?$AA?5?$AAV?$AAi?$AAs?$AAu?$AAa@ 00124ac8     winmodemstat.obj
 0002:00006b4c       ??_C@_1CK@EOPGIILJ@?$AAi?$AAn?$AAv?$AAa?$AAl?$AAi?$AAd?$AA?5?$AAn?$AAu?$AAl?$AAl?$AA?5?$AAp?$AAo?$AAi?$AAn?$AAt?$AAe?$AAr?$AA?$AA@ 00124b4c     winmodemstat.obj
 0002:00006c5c       IID_IClassFactory          00124c5c     uuid:unknwn_i_guid1.obj
 0002:00006c6c       IID_IUnknown               00124c6c     uuid:unknwn_i_guid0.obj
 0002:00006c7c       IID_IObjectWithSite        00124c7c     uuid:ocidl_i_guid34.obj
 0002:00006c8c       ??_C@_17LGKOMLJ@?$AA?4?$AA?4?$AA?4?$AA?$AA@ 00124c8c     LIBCMTD:dbgrpt.obj
 0002:00006c94       ??_C@_1CC@CGHMNGDG@?$AAA?$AAs?$AAs?$AAe?$AAr?$AAt?$AAi?$AAo?$AAn?$AA?5?$AAF?$AAa?$AAi?$AAl?$AAe?$AAd?$AA?$AA@ 00124c94     LIBCMTD:dbgrpt.obj
 0002:00006cb8       ??_C@_1M@ILHOPKA@?$AAE?$AAr?$AAr?$AAo?$AAr?$AA?$AA@ 00124cb8     LIBCMTD:dbgrpt.obj
 0002:00006cc4       ??_C@_1BA@GLMCNLEM@?$AAW?$AAa?$AAr?$AAn?$AAi?$AAn?$AAg?$AA?$AA@ 00124cc4     LIBCMTD:dbgrpt.obj
 0002:00006cd8       ??_C@_1FI@PHIAFFHM@?$AA?$CI?$AA?$CC?$AAT?$AAh?$AAe?$AA?5?$AAh?$AAo?$AAo?$AAk?$AA?5?$AAf?$AAu?$AAn?$AAc?$AAt?$AAi?$AAo?$AAn?$AA?5?$AAi?$AAs?$AA?5?$AAn?$AAo?$AAt?$AA?5?$AAi?$AAn?$AA?5?$AAt?$AAh@ 00124cd8     LIBCMTD:dbgrpt.obj
 0002:00006d30       ??_C@_1CG@JBJEFOCM@?$AAp?$AAf?$AAn?$AAN?$AAe?$AAw?$AAH?$AAo?$AAo?$AAk?$AA?5?$AA?$CB?$AA?$DN?$AA?5?$AAN?$AAU?$AAL?$AAL?$AA?$AA@ 00124d30     LIBCMTD:dbgrpt.obj
 0002:00006d58       ??_C@_1CI@OOAHIOG@?$AA_?$AAC?$AAr?$AAt?$AAS?$AAe?$AAt?$AAR?$AAe?$AAp?$AAo?$AAr?$AAt?$AAH?$AAo?$AAo?$AAk?$AAT?$AA2?$AA?$AA@ 00124d58     LIBCMTD:dbgrpt.obj
 0002:00006d80       ??_C@_1FC@DDJKODKC@?$AAf?$AA?3?$AA?2?$AAs?$AAp?$AA?2?$AAv?$AAc?$AAt?$AAo?$AAo?$AAl?$AAs?$AA?2?$AAc?$AAr?$AAt?$AAc?$AAe?$AA?2?$AAc?$AAr?$AAt?$AAw?$AA3?$AA2?$AA?2?$AAm?$AAi?$AAs?$AAc?$AA?2@ 00124d80     LIBCMTD:dbgrpt.obj
 0002:00006dd8       ??_C@_1HI@OFEHGPPC@?$AAm?$AAo?$AAd?$AAe?$AA?5?$AA?$DN?$AA?$DN?$AA?5?$AA_?$AAC?$AAR?$AAT?$AA_?$AAR?$AAP?$AAT?$AAH?$AAO?$AAO?$AAK?$AA_?$AAI?$AAN?$AAS?$AAT?$AAA?$AAL?$AAL?$AA?5?$AA?$HM?$AA?$HM?$AA?5@ 00124dd8     LIBCMTD:dbgrpt.obj
 0002:00006e50       ??_C@_1EG@PEOEAKBB@?$AAM?$AAi?$AAc?$AAr?$AAo?$AAs?$AAo?$AAf?$AAt?$AA?5?$AAV?$AAi?$AAs?$AAu?$AAa?$AAl?$AA?5?$AAC?$AA?$CL?$AA?$CL?$AA?5?$AAD?$AAe?$AAb?$AAu?$AAg?$AA?5?$AAL?$AAi?$AAb?$AAr?$AAa@ 00124e50     LIBCMTD:dbgrpt.obj
 0002:00006e98       ??_C@_1JI@EACPGHID@?$AAw?$AAc?$AAs?$AAc?$AAp?$AAy?$AA_?$AAs?$AA?$CI?$AAs?$AAz?$AAO?$AAu?$AAt?$AAM?$AAe?$AAs?$AAs?$AAa?$AAg?$AAe?$AA?0?$AA?5?$AA4?$AA0?$AA9?$AA6?$AA?0?$AA?5?$AAL?$AA?$CC?$AA_@ 00124e98     LIBCMTD:dbgrpt.obj
 0002:00006f30       ??_C@_1FG@BBOLDHGF@?$AA_?$AAC?$AAr?$AAt?$AAD?$AAb?$AAg?$AAR?$AAe?$AAp?$AAo?$AAr?$AAt?$AA?3?$AA?5?$AAS?$AAt?$AAr?$AAi?$AAn?$AAg?$AA?5?$AAt?$AAo?$AAo?$AA?5?$AAl?$AAo?$AAn?$AAg?$AA?5?$AAo@ 00124f30     LIBCMTD:dbgrpt.obj
 0002:00006f88       ??_C@_1KG@MFHGLLO@?$AAD?$AAe?$AAb?$AAu?$AAg?$AA?5?$AA?$CF?$AAs?$AA?$CB?$AA?6?$AA?6?$AAP?$AAr?$AAo?$AAg?$AAr?$AAa?$AAm?$AA?3?$AA?5?$AA?$CF?$AAs?$AA?$CF?$AAs?$AA?$CF?$AAs?$AA?$CF?$AAs?$AA?$CF?$AAs?$AA?$CF?$AAs@ 00124f88     LIBCMTD:dbgrpt.obj
 0002:00007030       ??_C@_1BE@CGCJKGHI@?$AA?6?$AAM?$AAo?$AAd?$AAu?$AAl?$AAe?$AA?3?$AA?5?$AA?$AA@ 00125030     LIBCMTD:dbgrpt.obj
 0002:00007044       ??_C@_1BA@LNHECFIM@?$AA?6?$AAF?$AAi?$AAl?$AAe?$AA?3?$AA?5?$AA?$AA@ 00125044     LIBCMTD:dbgrpt.obj
 0002:00007054       ??_C@_1BA@GLLGCPCK@?$AA?6?$AAL?$AAi?$AAn?$AAe?$AA?3?$AA?5?$AA?$AA@ 00125054     LIBCMTD:dbgrpt.obj
 0002:00007064       ??_C@_13LBAGMAIH@?$AA?6?$AA?$AA@ 00125064     LIBCMTD:dbgrpt.obj
 0002:00007068       ??_C@_1BK@PEDCIPMA@?$AAE?$AAx?$AAp?$AAr?$AAe?$AAs?$AAs?$AAi?$AAo?$AAn?$AA?3?$AA?5?$AA?$AA@ 00125068     LIBCMTD:dbgrpt.obj
 0002:00007084       ??_C@_11LOCGONAA@?$AA?$AA@ 00125084     LIBCMTD:dbgrpt.obj
 0002:00007088       ??_C@_1JM@GKDPCMEA@?$AAw?$AAc?$AAs?$AAn?$AAc?$AAp?$AAy?$AA_?$AAs?$AA?$CI?$AAs?$AAz?$AAS?$AAh?$AAo?$AAr?$AAt?$AAP?$AAr?$AAo?$AAg?$AAN?$AAa?$AAm?$AAe?$AA?0?$AA?5?$AA2?$AA6?$AA0?$AA?5?$AA?9@ 00125088     LIBCMTD:dbgrpt.obj
 0002:00007128       ??_C@_1GI@DEDNNLCI@?$AAw?$AAc?$AAs?$AAc?$AAp?$AAy?$AA_?$AAs?$AA?$CI?$AAs?$AAz?$AAE?$AAx?$AAe?$AAN?$AAa?$AAm?$AAe?$AA?0?$AA?5?$AA2?$AA6?$AA0?$AA?0?$AA?5?$AAL?$AA?$CC?$AA?$DM?$AAp?$AAr?$AAo?$AAg@ 00125128     LIBCMTD:dbgrpt.obj
 0002:00007190       ??_C@_1CI@PGJIFDEK@?$AA_?$AA_?$AAc?$AAr?$AAt?$AAM?$AAe?$AAs?$AAs?$AAa?$AAg?$AAe?$AAW?$AAi?$AAn?$AAd?$AAo?$AAw?$AAW?$AA?$AA@ 00125190     LIBCMTD:dbgrpt.obj
 0002:000071b8       ??_C@_1CO@EAEJAADC@?$AA?$DM?$AAp?$AAr?$AAo?$AAg?$AAr?$AAa?$AAm?$AA?5?$AAn?$AAa?$AAm?$AAe?$AA?5?$AAu?$AAn?$AAk?$AAn?$AAo?$AAw?$AAn?$AA?$DO?$AA?$AA@ 001251b8     LIBCMTD:dbgrpt.obj
 0002:000071e8       ??_C@_1CK@DDKKOLAN@?$AAs?$AAi?$AAz?$AAe?$AAI?$AAn?$AAB?$AAy?$AAt?$AAe?$AAs?$AA?5?$AA?$DO?$AA?$DN?$AA?5?$AAc?$AAo?$AAu?$AAn?$AAt?$AA?$AA@ 001251e8     LIBCMTD:memcpy_s.obj
 0002:00007214       ??_C@_1BI@DCHLDCPP@?$AAs?$AAr?$AAc?$AA?5?$AA?$CB?$AA?$DN?$AA?5?$AAN?$AAU?$AAL?$AAL?$AA?$AA@ 00125214     LIBCMTD:memcpy_s.obj
 0002:0000722c       ??_C@_1BC@GKHDJMGB@?$AAm?$AAe?$AAm?$AAc?$AAp?$AAy?$AA_?$AAs?$AA?$AA@ 0012522c     LIBCMTD:memcpy_s.obj
 0002:00007240       ??_C@_1FK@BOBCAACJ@?$AAf?$AA?3?$AA?2?$AAs?$AAp?$AA?2?$AAv?$AAc?$AAt?$AAo?$AAo?$AAl?$AAs?$AA?2?$AAc?$AAr?$AAt?$AAc?$AAe?$AA?2?$AAc?$AAr?$AAt?$AAw?$AA3?$AA2?$AA?2?$AAs?$AAt?$AAr?$AAi?$AAn@ 00125240     LIBCMTD:memcpy_s.obj
 0002:0000729c       ??_C@_1BI@GKKCBDMD@?$AAd?$AAs?$AAt?$AA?5?$AA?$CB?$AA?$DN?$AA?5?$AAN?$AAU?$AAL?$AAL?$AA?$AA@ 0012529c     LIBCMTD:memcpy_s.obj
 0002:000072b4       ??_C@_1BE@NMKKBGPA@?$AAm?$AAe?$AAm?$AAm?$AAo?$AAv?$AAe?$AA_?$AAs?$AA?$AA@ 001252b4     LIBCMTD:memmove_s.obj
 0002:000072c8       ??_C@_1FM@JMDLOEFB@?$AAf?$AA?3?$AA?2?$AAs?$AAp?$AA?2?$AAv?$AAc?$AAt?$AAo?$AAo?$AAl?$AAs?$AA?2?$AAc?$AAr?$AAt?$AAc?$AAe?$AA?2?$AAc?$AAr?$AAt?$AAw?$AA3?$AA2?$AA?2?$AAs?$AAt?$AAr?$AAi?$AAn@ 001252c8     LIBCMTD:memmove_s.obj
 0002:00007324       ??_C@_0BJ@IPHDMCNM@fatal?5error?5in?5_lock?5?$CD0?6?$AA@ 00125324     LIBCMTD:mlock.obj
 0002:00007340       ??_C@_1NK@LOFHIHFC@?$AAf?$AAM?$AAo?$AAd?$AAe?$AA?5?$AA?$DN?$AA?$DN?$AA?5?$AA_?$AAC?$AAR?$AAT?$AAD?$AAB?$AAG?$AA_?$AAR?$AAE?$AAP?$AAO?$AAR?$AAT?$AA_?$AAM?$AAO?$AAD?$AAE?$AA?5?$AA?$HM?$AA?$HM?$AA?5@ 00125340     LIBCMTD:dbgrptt.obj
 0002:0000741c       ??_C@_1CE@FIHIECNJ@?$AA_?$AAC?$AAr?$AAt?$AAS?$AAe?$AAt?$AAR?$AAe?$AAp?$AAo?$AAr?$AAt?$AAM?$AAo?$AAd?$AAe?$AA?$AA@ 0012541c     LIBCMTD:dbgrptt.obj
 0002:00007440       ??_C@_1FE@PLIBPAGC@?$AAf?$AA?3?$AA?2?$AAs?$AAp?$AA?2?$AAv?$AAc?$AAt?$AAo?$AAo?$AAl?$AAs?$AA?2?$AAc?$AAr?$AAt?$AAc?$AAe?$AA?2?$AAc?$AAr?$AAt?$AAw?$AA3?$AA2?$AA?2?$AAm?$AAi?$AAs?$AAc?$AA?2@ 00125440     LIBCMTD:dbgrptt.obj
 0002:00007498       ??_C@_1FA@IFFFOLDJ@?$AAn?$AAR?$AAp?$AAt?$AAT?$AAy?$AAp?$AAe?$AA?5?$AA?$DO?$AA?$DN?$AA?5?$AA0?$AA?5?$AA?$CG?$AA?$CG?$AA?5?$AAn?$AAR?$AAp?$AAt?$AAT?$AAy?$AAp?$AAe?$AA?5?$AA?$DM?$AA?5?$AA_?$AAC?$AAR?$AAT@ 00125498     LIBCMTD:dbgrptt.obj
 0002:000074e8       ??_C@_1CE@IKKEDCME@?$AA_?$AAC?$AAr?$AAt?$AAS?$AAe?$AAt?$AAR?$AAe?$AAp?$AAo?$AAr?$AAt?$AAF?$AAi?$AAl?$AAe?$AA?$AA@ 001254e8     LIBCMTD:dbgrptt.obj
 0002:00007510       ??_C@_1MA@LBAMNNOB@?$AAs?$AAt?$AAr?$AAc?$AAp?$AAy?$AA_?$AAs?$AA?$CI?$AAs?$AAz?$AAO?$AAu?$AAt?$AAM?$AAe?$AAs?$AAs?$AAa?$AAg?$AAe?$AA2?$AA?0?$AA?5?$AA4?$AA0?$AA9?$AA6?$AA?0?$AA?5?$AA?$CC?$AA_@ 00125510     LIBCMTD:dbgrptt.obj
 0002:000075d0       ??_C@_0DP@GNPEPHJD@_CrtDbgReport?3?5String?5too?5long?5o@ 001255d0     LIBCMTD:dbgrptt.obj
 0002:00007610       ??_C@_1FI@DBAIJPJE@?$AAw?$AAc?$AAs?$AAc?$AAp?$AAy?$AA_?$AAs?$AA?$CI?$AAs?$AAz?$AAO?$AAu?$AAt?$AAM?$AAe?$AAs?$AAs?$AAa?$AAg?$AAe?$AA?0?$AA?5?$AA4?$AA0?$AA9?$AA6?$AA?0?$AA?5?$AAs?$AAz?$AAL@ 00125610     LIBCMTD:dbgrptt.obj
 0002:00007668       ??_C@_1BI@JIDBEPIG@?$AA?$CF?$AAs?$AA?$CI?$AA?$CF?$AAd?$AA?$CJ?$AA?5?$AA?3?$AA?5?$AA?$CF?$AAs?$AA?$AA@ 00125668     LIBCMTD:dbgrptt.obj
 0002:00007680       ??_C@_1EK@PHCBEDKB@?$AAw?$AAc?$AAs?$AAc?$AAa?$AAt?$AA_?$AAs?$AA?$CI?$AAs?$AAz?$AAL?$AAi?$AAn?$AAe?$AAM?$AAe?$AAs?$AAs?$AAa?$AAg?$AAe?$AA?0?$AA?5?$AA4?$AA0?$AA9?$AA6?$AA?0?$AA?5?$AAL?$AA?$CC@ 00125680     LIBCMTD:dbgrptt.obj
 0002:000076d0       ??_C@_1EK@NMDFGHMF@?$AAw?$AAc?$AAs?$AAc?$AAa?$AAt?$AA_?$AAs?$AA?$CI?$AAs?$AAz?$AAL?$AAi?$AAn?$AAe?$AAM?$AAe?$AAs?$AAs?$AAa?$AAg?$AAe?$AA?0?$AA?5?$AA4?$AA0?$AA9?$AA6?$AA?0?$AA?5?$AAL?$AA?$CC@ 001256d0     LIBCMTD:dbgrptt.obj
 0002:0000771c       ??_C@_13CMNBPIDO@?$AA?$AN?$AA?$AA@ 0012571c     LIBCMTD:dbgrptt.obj
 0002:00007720       ??_C@_1FK@HPADHBBD@?$AAw?$AAc?$AAs?$AAc?$AAa?$AAt?$AA_?$AAs?$AA?$CI?$AAs?$AAz?$AAL?$AAi?$AAn?$AAe?$AAM?$AAe?$AAs?$AAs?$AAa?$AAg?$AAe?$AA?0?$AA?5?$AA4?$AA0?$AA9?$AA6?$AA?0?$AA?5?$AAs?$AAz@ 00125720     LIBCMTD:dbgrptt.obj
 0002:00007780       ??_C@_1KO@DGAHENCH@?$AAw?$AAc?$AAs?$AAc?$AAp?$AAy?$AA_?$AAs?$AA?$CI?$AAs?$AAz?$AAL?$AAi?$AAn?$AAe?$AAM?$AAe?$AAs?$AAs?$AAa?$AAg?$AAe?$AA?0?$AA?5?$AA4?$AA0?$AA9?$AA6?$AA?0?$AA?5?$AAs?$AAz@ 00125780     LIBCMTD:dbgrptt.obj
 0002:00007830       ??_C@_1CE@OJBNHDMO@?$AAA?$AAs?$AAs?$AAe?$AAr?$AAt?$AAi?$AAo?$AAn?$AA?5?$AAf?$AAa?$AAi?$AAl?$AAe?$AAd?$AA?$CB?$AA?$AA@ 00125830     LIBCMTD:dbgrptt.obj
 0002:00007854       ??_C@_1CG@FFFGGODN@?$AAA?$AAs?$AAs?$AAe?$AAr?$AAt?$AAi?$AAo?$AAn?$AA?5?$AAf?$AAa?$AAi?$AAl?$AAe?$AAd?$AA?3?$AA?5?$AA?$AA@ 00125854     LIBCMTD:dbgrptt.obj
 0002:00007880       ??_C@_1JK@KHFABAEO@?$AAw?$AAc?$AAs?$AAc?$AAp?$AAy?$AA_?$AAs?$AA?$CI?$AAs?$AAz?$AAU?$AAs?$AAe?$AAr?$AAM?$AAe?$AAs?$AAs?$AAa?$AAg?$AAe?$AA?0?$AA?5?$AA4?$AA0?$AA9?$AA6?$AA?0?$AA?5?$AAL?$AA?$CC@ 00125880     LIBCMTD:dbgrptt.obj
 0002:0000791c       ??_C@_1BA@ELMMDCFC@?$AA?0?$AA?5?$AAL?$AAi?$AAn?$AAe?$AA?5?$AA?$AA@ 0012591c     LIBCMTD:dbgrptt.obj
 0002:0000792c       ??_C@_1BO@OCHMLCAG@?$AA?$DM?$AAf?$AAi?$AAl?$AAe?$AA?5?$AAu?$AAn?$AAk?$AAn?$AAo?$AAw?$AAn?$AA?$DO?$AA?$AA@ 0012592c     LIBCMTD:dbgrptt.obj
 0002:00007950       ??_C@_1EM@MJFLEDMB@?$AAS?$AAe?$AAc?$AAo?$AAn?$AAd?$AA?5?$AAC?$AAh?$AAa?$AAn?$AAc?$AAe?$AA?5?$AAA?$AAs?$AAs?$AAe?$AAr?$AAt?$AAi?$AAo?$AAn?$AA?5?$AAF?$AAa?$AAi?$AAl?$AAe?$AAd?$AA?3?$AA?5@ 00125950     LIBCMTD:dbgrptt.obj
 0002:000079a0       ??_C@_1FA@CNLLOMHI@?$AA_?$AAi?$AAt?$AAo?$AAw?$AA_?$AAs?$AA?$CI?$AAn?$AAL?$AAi?$AAn?$AAe?$AA?0?$AA?5?$AAs?$AAz?$AAL?$AAi?$AAn?$AAe?$AAM?$AAe?$AAs?$AAs?$AAa?$AAg?$AAe?$AA?0?$AA?5?$AA4?$AA0@ 001259a0     LIBCMTD:dbgrptt.obj
 0002:000079f0       ??_C@_1CA@HPALHDOD@?$AA_?$AAV?$AAC?$AAr?$AAt?$AAD?$AAb?$AAg?$AAR?$AAe?$AAp?$AAo?$AAr?$AAt?$AAW?$AA?$AA@ 001259f0     LIBCMTD:dbgrptt.obj
 0002:00007a10       ??_C@_1CG@MKBKDNCP@?$AAG?$AAe?$AAt?$AAL?$AAa?$AAs?$AAt?$AAA?$AAc?$AAt?$AAi?$AAv?$AAe?$AAP?$AAo?$AAp?$AAu?$AAp?$AA?$AA@ 00125a10     LIBCMTD:crtmbox.obj
 0002:00007a38       ??_C@_1CA@HNKPMKAN@?$AAG?$AAe?$AAt?$AAA?$AAc?$AAt?$AAi?$AAv?$AAe?$AAW?$AAi?$AAn?$AAd?$AAo?$AAw?$AA?$AA@ 00125a38     LIBCMTD:crtmbox.obj
 0002:00007a58       ??_C@_1BI@OGPGOOGK@?$AAM?$AAe?$AAs?$AAs?$AAa?$AAg?$AAe?$AAB?$AAo?$AAx?$AAW?$AA?$AA@ 00125a58     LIBCMTD:crtmbox.obj
 0002:00007a70       ??_C@_1BI@IENOMFML@?$AAC?$AAO?$AAR?$AAE?$AAD?$AAL?$AAL?$AA?4?$AAD?$AAL?$AAL?$AA?$AA@ 00125a70     LIBCMTD:crtmbox.obj
 0002:00007a88       ??_C@_1DM@MADKGDLO@?$AA?$CI?$AAL?$AA?$CC?$AAB?$AAu?$AAf?$AAf?$AAe?$AAr?$AA?5?$AAi?$AAs?$AA?5?$AAt?$AAo?$AAo?$AA?5?$AAs?$AAm?$AAa?$AAl?$AAl?$AA?$CC?$AA?5?$AA?$CG?$AA?$CG?$AA?5?$AA0?$AA?$CJ?$AA?$AA@ 00125a88     LIBCMTD:wcsncpy_s.obj
 0002:00007ac4       ??_C@_1CI@HCPHDDLE@?$AAB?$AAu?$AAf?$AAf?$AAe?$AAr?$AA?5?$AAi?$AAs?$AA?5?$AAt?$AAo?$AAo?$AA?5?$AAs?$AAm?$AAa?$AAl?$AAl?$AA?$AA@ 00125ac4     LIBCMTD:wcsncpy_s.obj
 0002:00007aec       ??_C@_1CG@OFBJMIGJ@?$AA?$CI?$AA?$CI?$AA?$CI?$AA_?$AAS?$AAr?$AAc?$AA?$CJ?$AA?$CJ?$AA?$CJ?$AA?5?$AA?$CB?$AA?$DN?$AA?5?$AAN?$AAU?$AAL?$AAL?$AA?$AA@ 00125aec     LIBCMTD:wcsncpy_s.obj
 0002:00007b14       ??_C@_1BE@PMMBFFCC@?$AAw?$AAc?$AAs?$AAn?$AAc?$AAp?$AAy?$AA_?$AAs?$AA?$AA@ 00125b14     LIBCMTD:wcsncpy_s.obj
 0002:00007b28       ??_C@_1FG@OHHBDIEA@?$AAf?$AA?3?$AA?2?$AAs?$AAp?$AA?2?$AAv?$AAc?$AAt?$AAo?$AAo?$AAl?$AAs?$AA?2?$AAc?$AAr?$AAt?$AAc?$AAe?$AA?2?$AAc?$AAr?$AAt?$AAw?$AA3?$AA2?$AA?2?$AAh?$AA?2?$AAt?$AAc?$AAs@ 00125b28     LIBCMTD:wcsncpy_s.obj
 0002:00007b80       ??_C@_1FC@PFMLEHKI@?$AA?$CI?$AA?$CI?$AA_?$AAD?$AAs?$AAt?$AA?$CJ?$AA?$CJ?$AA?5?$AA?$CB?$AA?$DN?$AA?5?$AAN?$AAU?$AAL?$AAL?$AA?5?$AA?$CG?$AA?$CG?$AA?5?$AA?$CI?$AA?$CI?$AA_?$AAS?$AAi?$AAz?$AAe?$AAI?$AAn?$AAW?$AAo?$AAr@ 00125b80     LIBCMTD:wcsncpy_s.obj
 0002:00007bd4       ??_C@_1BC@KIONAFPO@?$AAw?$AAc?$AAs?$AAc?$AAp?$AAy?$AA_?$AAs?$AA?$AA@ 00125bd4     LIBCMTD:wcscpy_s.obj
 0002:00007be8       ??_C@_1FE@IPADLOPJ@?$AAf?$AA?3?$AA?2?$AAs?$AAp?$AA?2?$AAv?$AAc?$AAt?$AAo?$AAo?$AAl?$AAs?$AA?2?$AAc?$AAr?$AAt?$AAc?$AAe?$AA?2?$AAc?$AAr?$AAt?$AAw?$AA3?$AA2?$AA?2?$AAh?$AA?2?$AAt?$AAc?$AAs@ 00125be8     LIBCMTD:wcscpy_s.obj
 0002:00007c3c       ??_C@_1BC@CFJEPFGF@?$AAs?$AAt?$AAr?$AAc?$AAp?$AAy?$AA_?$AAs?$AA?$AA@ 00125c3c     LIBCMTD:strcpy_s.obj
 0002:00007c50       ??_C@_1FC@NCPEPIBI@?$AA?$CI?$AA?$CI?$AA_?$AAD?$AAs?$AAt?$AA?$CJ?$AA?$CJ?$AA?5?$AA?$CB?$AA?$DN?$AA?5?$AAN?$AAU?$AAL?$AAL?$AA?5?$AA?$CG?$AA?$CG?$AA?5?$AA?$CI?$AA?$CI?$AA_?$AAS?$AAi?$AAz?$AAe?$AAI?$AAn?$AAB?$AAy?$AAt@ 00125c50     LIBCMTD:strcpy_s.obj
 0002:00007ca8       ??_C@_1FA@MJKDNFFB@?$AA?$CI?$AAL?$AA?$CC?$AAS?$AAt?$AAr?$AAi?$AAn?$AAg?$AA?5?$AAi?$AAs?$AA?5?$AAn?$AAo?$AAt?$AA?5?$AAn?$AAu?$AAl?$AAl?$AA?5?$AAt?$AAe?$AAr?$AAm?$AAi?$AAn?$AAa?$AAt?$AAe?$AAd@ 00125ca8     LIBCMTD:wcscat_s.obj
 0002:00007cf8       ??_C@_1DM@FHLMIEG@?$AAS?$AAt?$AAr?$AAi?$AAn?$AAg?$AA?5?$AAi?$AAs?$AA?5?$AAn?$AAo?$AAt?$AA?5?$AAn?$AAu?$AAl?$AAl?$AA?5?$AAt?$AAe?$AAr?$AAm?$AAi?$AAn?$AAa?$AAt?$AAe?$AAd?$AA?$AA@ 00125cf8     LIBCMTD:wcscat_s.obj
 0002:00007d34       ??_C@_1BC@PLIEPKPJ@?$AAw?$AAc?$AAs?$AAc?$AAa?$AAt?$AA_?$AAs?$AA?$AA@ 00125d34     LIBCMTD:wcscat_s.obj
 0002:00007d48       ??_C@_1FE@EHLIBGFJ@?$AAf?$AA?3?$AA?2?$AAs?$AAp?$AA?2?$AAv?$AAc?$AAt?$AAo?$AAo?$AAl?$AAs?$AA?2?$AAc?$AAr?$AAt?$AAc?$AAe?$AA?2?$AAc?$AAr?$AAt?$AAw?$AA3?$AA2?$AA?2?$AAh?$AA?2?$AAt?$AAc?$AAs@ 00125d48     LIBCMTD:wcscat_s.obj
 0002:00007d9c       ??_C@_1CM@HABGDNLJ@?$AAl?$AAe?$AAn?$AAg?$AAt?$AAh?$AA?5?$AA?$DM?$AA?5?$AAs?$AAi?$AAz?$AAe?$AAI?$AAn?$AAT?$AAC?$AAh?$AAa?$AAr?$AAs?$AA?$AA@ 00125d9c     LIBCMTD:xtows.obj
 0002:00007dc8       ??_C@_1DE@PCJGDBBD@?$AA2?$AA?5?$AA?$DM?$AA?$DN?$AA?5?$AAr?$AAa?$AAd?$AAi?$AAx?$AA?5?$AA?$CG?$AA?$CG?$AA?5?$AAr?$AAa?$AAd?$AAi?$AAx?$AA?5?$AA?$DM?$AA?$DN?$AA?5?$AA3?$AA6?$AA?$AA@ 00125dc8     LIBCMTD:xtows.obj
 0002:00007e00       ??_C@_1FA@MKGGAGEI@?$AAs?$AAi?$AAz?$AAe?$AAI?$AAn?$AAT?$AAC?$AAh?$AAa?$AAr?$AAs?$AA?5?$AA?$DO?$AA?5?$AA?$CI?$AAs?$AAi?$AAz?$AAe?$AA_?$AAt?$AA?$CJ?$AA?$CI?$AAi?$AAs?$AA_?$AAn?$AAe?$AAg?$AA?5?$AA?$DP@ 00125e00     LIBCMTD:xtows.obj
 0002:00007e50       ??_C@_1CC@JNJFIMGE@?$AAs?$AAi?$AAz?$AAe?$AAI?$AAn?$AAT?$AAC?$AAh?$AAa?$AAr?$AAs?$AA?5?$AA?$DO?$AA?5?$AA0?$AA?$AA@ 00125e50     LIBCMTD:xtows.obj
 0002:00007e74       ??_C@_1O@NCBFODOE@?$AAx?$AAt?$AAo?$AAw?$AA_?$AAs?$AA?$AA@ 00125e74     LIBCMTD:xtows.obj
 0002:00007e88       ??_C@_1FE@LAGNOOBA@?$AAf?$AA?3?$AA?2?$AAs?$AAp?$AA?2?$AAv?$AAc?$AAt?$AAo?$AAo?$AAl?$AAs?$AA?2?$AAc?$AAr?$AAt?$AAc?$AAe?$AA?2?$AAc?$AAr?$AAt?$AAw?$AA3?$AA2?$AA?2?$AAc?$AAo?$AAn?$AAv?$AAe@ 00125e88     LIBCMTD:xtows.obj
 0002:00007edc       ??_C@_1BI@ICGGMGLK@?$AAb?$AAu?$AAf?$AA?5?$AA?$CB?$AA?$DN?$AA?5?$AAN?$AAU?$AAL?$AAL?$AA?$AA@ 00125edc     LIBCMTD:xtows.obj
 0002:00007ef4       ??_C@_0P@GHFPNOJB@bad?5allocation?$AA@ 00125ef4     libcpmtd:stdthrow.obj
 0002:00007f04       ??_C@_01EEMJAFIK@?6?$AA@   00125f04     libcpmtd:stdthrow.obj
 0002:00007f08       ??_C@_07CIFAGBMG@unknown?$AA@ 00125f08     libcpmtd:stdthrow.obj
 0002:00007f10       ??_C@_0M@LLHBPFNE@exception?3?5?$AA@ 00125f10     libcpmtd:stdthrow.obj
 0002:00007f1c       ?skipws@?$_Iosb@H@std@@2W4_Fmtflags@12@B 00125f1c     libcpmtd:string.obj
 0002:00007f20       ?unitbuf@?$_Iosb@H@std@@2W4_Fmtflags@12@B 00125f20     libcpmtd:string.obj
 0002:00007f24       ?uppercase@?$_Iosb@H@std@@2W4_Fmtflags@12@B 00125f24     libcpmtd:string.obj
 0002:00007f28       ?showbase@?$_Iosb@H@std@@2W4_Fmtflags@12@B 00125f28     libcpmtd:string.obj
 0002:00007f2c       ?showpoint@?$_Iosb@H@std@@2W4_Fmtflags@12@B 00125f2c     libcpmtd:string.obj
 0002:00007f30       ?showpos@?$_Iosb@H@std@@2W4_Fmtflags@12@B 00125f30     libcpmtd:string.obj
 0002:00007f34       ?left@?$_Iosb@H@std@@2W4_Fmtflags@12@B 00125f34     libcpmtd:string.obj
 0002:00007f38       ?right@?$_Iosb@H@std@@2W4_Fmtflags@12@B 00125f38     libcpmtd:string.obj
 0002:00007f3c       ?internal@?$_Iosb@H@std@@2W4_Fmtflags@12@B 00125f3c     libcpmtd:string.obj
 0002:00007f40       ?dec@?$_Iosb@H@std@@2W4_Fmtflags@12@B 00125f40     libcpmtd:string.obj
 0002:00007f44       ?oct@?$_Iosb@H@std@@2W4_Fmtflags@12@B 00125f44     libcpmtd:string.obj
 0002:00007f48       ?hex@?$_Iosb@H@std@@2W4_Fmtflags@12@B 00125f48     libcpmtd:string.obj
 0002:00007f4c       ?scientific@?$_Iosb@H@std@@2W4_Fmtflags@12@B 00125f4c     libcpmtd:string.obj
 0002:00007f50       ?fixed@?$_Iosb@H@std@@2W4_Fmtflags@12@B 00125f50     libcpmtd:string.obj
 0002:00007f54       ?boolalpha@?$_Iosb@H@std@@2W4_Fmtflags@12@B 00125f54     libcpmtd:string.obj
 0002:00007f58       ?_Stdio@?$_Iosb@H@std@@2W4_Fmtflags@12@B 00125f58     libcpmtd:string.obj
 0002:00007f5c       ?adjustfield@?$_Iosb@H@std@@2W4_Fmtflags@12@B 00125f5c     libcpmtd:string.obj
 0002:00007f60       ?basefield@?$_Iosb@H@std@@2W4_Fmtflags@12@B 00125f60     libcpmtd:string.obj
 0002:00007f64       ?floatfield@?$_Iosb@H@std@@2W4_Fmtflags@12@B 00125f64     libcpmtd:string.obj
 0002:00007f68       ?goodbit@?$_Iosb@H@std@@2W4_Iostate@12@B 00125f68     libcpmtd:string.obj
 0002:00007f6c       ?eofbit@?$_Iosb@H@std@@2W4_Iostate@12@B 00125f6c     libcpmtd:string.obj
 0002:00007f70       ?failbit@?$_Iosb@H@std@@2W4_Iostate@12@B 00125f70     libcpmtd:string.obj
 0002:00007f74       ?badbit@?$_Iosb@H@std@@2W4_Iostate@12@B 00125f74     libcpmtd:string.obj
 0002:00007f78       ?_Hardfail@?$_Iosb@H@std@@2W4_Iostate@12@B 00125f78     libcpmtd:string.obj
 0002:00007f7c       ?in@?$_Iosb@H@std@@2W4_Openmode@12@B 00125f7c     libcpmtd:string.obj
 0002:00007f80       ?out@?$_Iosb@H@std@@2W4_Openmode@12@B 00125f80     libcpmtd:string.obj
 0002:00007f84       ?ate@?$_Iosb@H@std@@2W4_Openmode@12@B 00125f84     libcpmtd:string.obj
 0002:00007f88       ?app@?$_Iosb@H@std@@2W4_Openmode@12@B 00125f88     libcpmtd:string.obj
 0002:00007f8c       ?trunc@?$_Iosb@H@std@@2W4_Openmode@12@B 00125f8c     libcpmtd:string.obj
 0002:00007f90       ?_Nocreate@?$_Iosb@H@std@@2W4_Openmode@12@B 00125f90     libcpmtd:string.obj
 0002:00007f94       ?_Noreplace@?$_Iosb@H@std@@2W4_Openmode@12@B 00125f94     libcpmtd:string.obj
 0002:00007f98       ?binary@?$_Iosb@H@std@@2W4_Openmode@12@B 00125f98     libcpmtd:string.obj
 0002:00007f9c       ?beg@?$_Iosb@H@std@@2W4_Seekdir@12@B 00125f9c     libcpmtd:string.obj
 0002:00007fa0       ?cur@?$_Iosb@H@std@@2W4_Seekdir@12@B 00125fa0     libcpmtd:string.obj
 0002:00007fa4       ?end@?$_Iosb@H@std@@2W4_Seekdir@12@B 00125fa4     libcpmtd:string.obj
 0002:00007fac       ??_7bad_alloc@std@@6B@     00125fac     libcpmtd:string.obj
 0002:00007fb8       ??_C@_1FE@OGIJMGPN@?$AAf?$AA?3?$AA?2?$AAs?$AAp?$AA?2?$AAv?$AAc?$AAt?$AAo?$AAo?$AAl?$AAs?$AA?2?$AAc?$AAr?$AAt?$AAc?$AAe?$AA?2?$AAc?$AAr?$AAt?$AAw?$AA3?$AA2?$AA?2?$AAs?$AAt?$AAd?$AAh?$AAp@ 00125fb8     libcpmtd:string.obj
 0002:00008010       ??_7logic_error@std@@6B@   00126010     libcpmtd:string.obj
 0002:0000801c       ??_7invalid_argument@std@@6B@ 0012601c     libcpmtd:string.obj
 0002:00008028       ??_7length_error@std@@6B@  00126028     libcpmtd:string.obj
 0002:00008034       ??_7out_of_range@std@@6B@  00126034     libcpmtd:string.obj
 0002:00008088       ??_C@_0BA@JFNIOLAK@string?5too?5long?$AA@ 00126088     libcpmtd:string.obj
 0002:000080e4       ??_C@_0BI@CFPLBAOH@invalid?5string?5position?$AA@ 001260e4     libcpmtd:string.obj
 0002:00008148       ??_C@_0BI@ILCMCLF@invalid?5string?5argument?$AA@ 00126148     libcpmtd:string.obj
 0002:00009144       _GUID_b196b284_bab4_101a_b69c_00aa00341d07 00127144     atlsd:atlfuncs.obj
 0002:00009154       _GUID_00000000_0000_0000_c000_000000000046 00127154     atlsd:atlfuncs.obj
 0002:00009168       ??_C@_1HA@FENMNPLO@?$AAf?$AA?3?$AA?2?$AAd?$AAd?$AA?2?$AAv?$AAc?$AAt?$AAo?$AAo?$AAl?$AAs?$AA?2?$AAv?$AAc?$AA7?$AAl?$AAi?$AAb?$AAs?$AAc?$AAe?$AA?2?$AAs?$AAh?$AAi?$AAp?$AA?2?$AAa?$AAt?$AAl@ 00127168     atlsd:atlfuncs.obj
 0002:000091d8       ??_C@_19LMDLLIGP@?$AAp?$AA?$DN?$AA?$DN?$AA0?$AA?$AA@ 001271d8     atlsd:atlfuncs.obj
 0002:000091e4       ??_C@_19JHCPJMAL@?$AAp?$AA?$CB?$AA?$DN?$AA0?$AA?$AA@ 001271e4     atlsd:atlfuncs.obj
 0002:000091f0       ??_C@_1HA@LPPEBACM@?$AAf?$AA?3?$AA?2?$AAd?$AAd?$AA?2?$AAv?$AAc?$AAt?$AAo?$AAo?$AAl?$AAs?$AA?2?$AAv?$AAc?$AA7?$AAl?$AAi?$AAb?$AAs?$AAc?$AAe?$AA?2?$AAs?$AAh?$AAi?$AAp?$AA?2?$AAa?$AAt?$AAl@ 001271f0     atlsd:atlfuncs.obj
 0002:00009260       ??_C@_1M@HLGKFCJM@?$AAf?$AAa?$AAl?$AAs?$AAe?$AA?$AA@ 00127260     atlsd:atlfuncs.obj
 0002:0000926c       ??_C@_1CK@DFMKPFAK@?$AAA?$AAt?$AAl?$AAT?$AAh?$AAr?$AAo?$AAw?$AA?3?$AA?5?$AAh?$AAr?$AA?5?$AA?$DN?$AA?5?$AA0?$AAx?$AA?$CF?$AAx?$AA?6?$AA?$AA@ 0012726c     atlsd:atlfuncs.obj
 0002:00009298       ??_C@_0DI@MHBOGIL@f?3?2dd?2vctools?2vc7libsce?2ship?2atl@ 00127298     atlsd:atlfuncs.obj
 0002:000092d0       ??_C@_1GM@IDLEHDFG@?$AAf?$AA?3?$AA?2?$AAd?$AAd?$AA?2?$AAv?$AAc?$AAt?$AAo?$AAo?$AAl?$AAs?$AA?2?$AAv?$AAc?$AA7?$AAl?$AAi?$AAb?$AAs?$AAc?$AAe?$AA?2?$AAs?$AAh?$AAi?$AAp?$AA?2?$AAa?$AAt?$AAl@ 001272d0     atlsd:atlfuncs.obj
 0002:0000933c       ??_C@_1BE@NPGJNKLA@?$AAm?$AA_?$AAb?$AAL?$AAo?$AAc?$AAk?$AAe?$AAd?$AA?$AA@ 0012733c     atlsd:atlfuncs.obj
 0002:00009350       ??_C@_1BG@OHCCAGNO@?$AA?$CB?$AAm?$AA_?$AAb?$AAL?$AAo?$AAc?$AAk?$AAe?$AAd?$AA?$AA@ 00127350     atlsd:atlfuncs.obj
 0002:00009368       ??_C@_1HE@LMFAHKHJ@?$AAf?$AA?3?$AA?2?$AAd?$AAd?$AA?2?$AAv?$AAc?$AAt?$AAo?$AAo?$AAl?$AAs?$AA?2?$AAv?$AAc?$AA7?$AAl?$AAi?$AAb?$AAs?$AAc?$AAe?$AA?2?$AAs?$AAh?$AAi?$AAp?$AA?2?$AAa?$AAt?$AAl@ 00127368     atlsd:atlfuncs.obj
 0002:00009550       GUID_ATLVer30              00127550     atlsd:atlbase.obj
 0002:00009560       GUID_ATLVer70              00127560     atlsd:atlbase.obj
 0002:0000c810       ??_C@_1JC@IHNNLNKC@?$AAf?$AA?3?$AA?2?$AAd?$AAd?$AA?2?$AAv?$AAc?$AAt?$AAo?$AAo?$AAl?$AAs?$AA?2?$AAv?$AAc?$AA7?$AAl?$AAi?$AAb?$AAs?$AAc?$AAe?$AA?2?$AAs?$AAh?$AAi?$AAp?$AA?2?$AAa?$AAt?$AAl@ 0012a810     atlsd:Allocate.obj
 0002:0000c8a4       ??_C@_1BK@GFEAMNLJ@?$AAn?$AAC?$AAo?$AAo?$AAk?$AAi?$AAe?$AA?5?$AA?$CB?$AA?$DN?$AA?5?$AA0?$AA?$AA@ 0012a8a4     atlsd:Allocate.obj
 0002:0000cca4       IID_IPersistStream         0012aca4     uuid:objidl_i_guid12.obj
 0002:0000cd30       ??_R4bad_alloc@std@@6B@    0012ad30     libcpmtd:string.obj
 0002:0000cd44       ??_R3bad_alloc@std@@8      0012ad44     libcpmtd:string.obj
 0002:0000cd54       ??_R2bad_alloc@std@@8      0012ad54     libcpmtd:string.obj
 0002:0000cd60       ??_R1A@?0A@EA@bad_alloc@std@@8 0012ad60     libcpmtd:string.obj
 0002:0000cd7c       ??_R1A@?0A@EA@exception@std@@8 0012ad7c     libcpmtd:string.obj
 0002:0000cd98       ??_R3exception@std@@8      0012ad98     libcpmtd:string.obj
 0002:0000cda8       ??_R2exception@std@@8      0012ada8     libcpmtd:string.obj
 0002:0000cdb0       ??_R4logic_error@std@@6B@  0012adb0     libcpmtd:string.obj
 0002:0000cdc4       ??_R3logic_error@std@@8    0012adc4     libcpmtd:string.obj
 0002:0000cdd4       ??_R2logic_error@std@@8    0012add4     libcpmtd:string.obj
 0002:0000cde0       ??_R1A@?0A@EA@logic_error@std@@8 0012ade0     libcpmtd:string.obj
 0002:0000cdfc       ??_R4invalid_argument@std@@6B@ 0012adfc     libcpmtd:string.obj
 0002:0000ce10       ??_R3invalid_argument@std@@8 0012ae10     libcpmtd:string.obj
 0002:0000ce20       ??_R2invalid_argument@std@@8 0012ae20     libcpmtd:string.obj
 0002:0000ce30       ??_R1A@?0A@EA@invalid_argument@std@@8 0012ae30     libcpmtd:string.obj
 0002:0000ce4c       ??_R4length_error@std@@6B@ 0012ae4c     libcpmtd:string.obj
 0002:0000ce60       ??_R3length_error@std@@8   0012ae60     libcpmtd:string.obj
 0002:0000ce70       ??_R2length_error@std@@8   0012ae70     libcpmtd:string.obj
 0002:0000ce80       ??_R1A@?0A@EA@length_error@std@@8 0012ae80     libcpmtd:string.obj
 0002:0000ce9c       ??_R4out_of_range@std@@6B@ 0012ae9c     libcpmtd:string.obj
 0002:0000ceb0       ??_R3out_of_range@std@@8   0012aeb0     libcpmtd:string.obj
 0002:0000cec0       ??_R2out_of_range@std@@8   0012aec0     libcpmtd:string.obj
 0002:0000ced0       ??_R1A@?0A@EA@out_of_range@std@@8 0012aed0     libcpmtd:string.obj
 0002:0000cfe4       _TI3?AVlength_error@std@@  0012afe4     winmodemstat.obj
 0002:0000cff4       _CTA3?AVlength_error@std@@ 0012aff4     winmodemstat.obj
 0002:0000d004       _CT??_R0?AVlength_error@std@@@8??0length_error@std@@QAA@ABV01@@Z44 0012b004     winmodemstat.obj
 0002:0000d020       _CT??_R0?AVlogic_error@std@@@8??0logic_error@std@@QAA@ABV01@@Z44 0012b020     winmodemstat.obj
 0002:0000d03c       _CT??_R0?AVexception@std@@@8??0exception@std@@QAA@ABV01@@Z12 0012b03c     winmodemstat.obj
 0002:0000d058       _TI2?AVbad_alloc@std@@     0012b058     winmodemstat.obj
 0002:0000d068       _CTA2?AVbad_alloc@std@@    0012b068     winmodemstat.obj
 0002:0000d074       _CT??_R0?AVbad_alloc@std@@@8??0bad_alloc@std@@QAA@ABV01@@Z12 0012b074     winmodemstat.obj
 0002:0000d090       _TI3?AVout_of_range@std@@  0012b090     libcpmtd:string.obj
 0002:0000d0a0       _CTA3?AVout_of_range@std@@ 0012b0a0     libcpmtd:string.obj
 0002:0000d0b0       _CT??_R0?AVout_of_range@std@@@8??0out_of_range@std@@QAA@ABV01@@Z44 0012b0b0     libcpmtd:string.obj
 0002:0000d0cc       _TI3?AVinvalid_argument@std@@ 0012b0cc     libcpmtd:string.obj
 0002:0000d0dc       _CTA3?AVinvalid_argument@std@@ 0012b0dc     libcpmtd:string.obj
 0002:0000d0ec       _CT??_R0?AVinvalid_argument@std@@@8??0invalid_argument@std@@QAA@ABV01@@Z44 0012b0ec     libcpmtd:string.obj
 0002:0000d108       _TI1?AVCAtlException@ATL@@ 0012b108     atlsd:Externs.obj
 0002:0000d118       _CTA1?AVCAtlException@ATL@@ 0012b118     atlsd:Externs.obj
 0002:0000d120       _CT??_R0?AVCAtlException@ATL@@@84 0012b120     atlsd:Externs.obj
 0002:0000d13c       __pobjMapEntryFirst        0012b13c     resultelement.obj
 0002:0000d140       __pobjMapEntryLast         0012b140     resultelement.obj
 0002:0000d144       __IMPORT_DESCRIPTOR_sw_utilityG 0012b144     sw_utilityG:sw_utilityG.dll
 0002:0000d158       __IMPORT_DESCRIPTOR_ril    0012b158     ril:ril.dll
 0002:0000d16c       __IMPORT_DESCRIPTOR_cellcore 0012b16c     Cellcore:cellcore.dll
 0002:0000d180       __IMPORT_DESCRIPTOR_AYGSHELL 0012b180     aygshell:AYGSHELL.dll
 0002:0000d194       __IMPORT_DESCRIPTOR_PHONE  0012b194     phone:PHONE.dll
 0002:0000d1a8       __IMPORT_DESCRIPTOR_COREDLL 0012b1a8     coredll:COREDLL.dll
 0002:0000d1bc       __IMPORT_DESCRIPTOR_ole32  0012b1bc     ole32:ole32.dll
 0002:0000d1d0       __NULL_IMPORT_DESCRIPTOR   0012b1d0     sw_utilityG:sw_utilityG.dll
 0003:00000000       __imp_SHGetEmergencyCallList 0012c000     aygshell:AYGSHELL.dll
 0003:00000004       \177AYGSHELL_NULL_THUNK_DATA 0012c004     aygshell:AYGSHELL.dll
 0003:00000008       __imp_InitializeCriticalSection 0012c008     coredll:COREDLL.dll
 0003:0000000c       __imp_SetLastError         0012c00c     coredll:COREDLL.dll
 0003:00000010       __imp_LoadLibraryW         0012c010     coredll:COREDLL.dll
 0003:00000014       __imp__wcsicmp             0012c014     coredll:COREDLL.dll
 0003:00000018       __imp_CreateFileMappingW   0012c018     coredll:COREDLL.dll
 0003:0000001c       __imp_MapViewOfFile        0012c01c     coredll:COREDLL.dll
 0003:00000020       __imp_GetSystemInfo        0012c020     coredll:COREDLL.dll
 0003:00000024       __imp_UnmapViewOfFile      0012c024     coredll:COREDLL.dll
 0003:00000028       __imp_VirtualAlloc         0012c028     coredll:COREDLL.dll
 0003:0000002c       __imp_OpenEventW           0012c02c     coredll:COREDLL.dll
 0003:00000030       __imp_CloseHandle          0012c030     coredll:COREDLL.dll
 0003:00000034       __imp_fputs                0012c034     coredll:COREDLL.dll
 0003:00000038       __imp_GetModuleHandleW     0012c038     coredll:COREDLL.dll
 0003:0000003c       __imp_MsgWaitForMultipleObjectsEx 0012c03c     coredll:COREDLL.dll
 0003:00000040       __imp_PeekMessageW         0012c040     coredll:COREDLL.dll
 0003:00000044       __imp_GetMessageW          0012c044     coredll:COREDLL.dll
 0003:00000048       __imp_TranslateMessage     0012c048     coredll:COREDLL.dll
 0003:0000004c       __imp_DispatchMessageW     0012c04c     coredll:COREDLL.dll
 0003:00000050       __imp_WaitForSingleObject  0012c050     coredll:COREDLL.dll
 0003:00000054       __imp_InterlockedExchange  0012c054     coredll:COREDLL.dll
 0003:00000058       __imp_fflush               0012c058     coredll:COREDLL.dll
 0003:0000005c       __imp_GetProcAddressW      0012c05c     coredll:COREDLL.dll
 0003:00000060       __imp_InterlockedIncrement 0012c060     coredll:COREDLL.dll
 0003:00000064       __imp_realloc              0012c064     coredll:COREDLL.dll
 0003:00000068       __imp_wcsncpy              0012c068     coredll:COREDLL.dll
 0003:0000006c       __imp_OutputDebugStringW   0012c06c     coredll:COREDLL.dll
 0003:00000070       __imp__vsnwprintf          0012c070     coredll:COREDLL.dll
 0003:00000074       __imp_NKDbgPrintfW         0012c074     coredll:COREDLL.dll
 0003:00000078       __imp_??3@YAXPAX@Z         0012c078     coredll:COREDLL.dll
 0003:0000007c       __imp_??2@YAPAXI@Z         0012c07c     coredll:COREDLL.dll
 0003:00000080       __imp_memcmp               0012c080     coredll:COREDLL.dll
 0003:00000084       __imp_CreateProcessW       0012c084     coredll:COREDLL.dll
 0003:00000088       __imp_CreateWindowExW      0012c088     coredll:COREDLL.dll
 0003:0000008c       __imp_GetLastError         0012c08c     coredll:COREDLL.dll
 0003:00000090       __imp_RegisterClassW       0012c090     coredll:COREDLL.dll
 0003:00000094       __imp_swprintf             0012c094     coredll:COREDLL.dll
 0003:00000098       __imp_GetStockObject       0012c098     coredll:COREDLL.dll
 0003:0000009c       __imp_memset               0012c09c     coredll:COREDLL.dll
 0003:000000a0       __imp_DestroyWindow        0012c0a0     coredll:COREDLL.dll
 0003:000000a4       __imp_wcscmp               0012c0a4     coredll:COREDLL.dll
 0003:000000a8       __imp_wcslen               0012c0a8     coredll:COREDLL.dll
 0003:000000ac       __imp_wcscpy               0012c0ac     coredll:COREDLL.dll
 0003:000000b0       __imp_wcsrchr              0012c0b0     coredll:COREDLL.dll
 0003:000000b4       __imp_MessageBoxW          0012c0b4     coredll:COREDLL.dll
 0003:000000b8       __imp_LoadStringW          0012c0b8     coredll:COREDLL.dll
 0003:000000bc       __imp_Sleep                0012c0bc     coredll:COREDLL.dll
 0003:000000c0       __imp__purecall            0012c0c0     coredll:COREDLL.dll
 0003:000000c4       __imp_InsertMenuW          0012c0c4     coredll:COREDLL.dll
 0003:000000c8       __imp_UnregisterClassW     0012c0c8     coredll:COREDLL.dll
 0003:000000cc       __imp_DeleteCriticalSection 0012c0cc     coredll:COREDLL.dll
 0003:000000d0       __imp_free                 0012c0d0     coredll:COREDLL.dll
 0003:000000d4       __imp_RaiseException       0012c0d4     coredll:COREDLL.dll
 0003:000000d8       __imp_CreateEventW         0012c0d8     coredll:COREDLL.dll
 0003:000000dc       __imp_??_U@YAPAXI@Z        0012c0dc     coredll:COREDLL.dll
 0003:000000e0       __imp_TerminateProcess     0012c0e0     coredll:COREDLL.dll
 0003:000000e4       __imp_PostMessageW         0012c0e4     coredll:COREDLL.dll
 0003:000000e8       __imp___rt_udiv            0012c0e8     coredll:COREDLL.dll
 0003:000000ec       __imp_EventModify          0012c0ec     coredll:COREDLL.dll
 0003:000000f0       __imp_??_V@YAXPAX@Z        0012c0f0     coredll:COREDLL.dll
 0003:000000f4       __imp_swscanf              0012c0f4     coredll:COREDLL.dll
 0003:000000f8       __imp_SendMessageTimeout   0012c0f8     coredll:COREDLL.dll
 0003:000000fc       __imp_CreateThread         0012c0fc     coredll:COREDLL.dll
 0003:00000100       __imp_wcstombs             0012c100     coredll:COREDLL.dll
 0003:00000104       __imp_memcpy               0012c104     coredll:COREDLL.dll
 0003:00000108       __imp___CxxThrowException  0012c108     coredll:COREDLL.dll
 0003:0000010c       __imp_??_7type_info@@6B@   0012c10c     coredll:COREDLL.dll
 0003:00000110       __imp_??0exception@std@@QAA@ABV01@@Z 0012c110     coredll:COREDLL.dll
 0003:00000114       __imp_??1exception@std@@UAA@XZ 0012c114     coredll:COREDLL.dll
 0003:00000118       __imp_??0exception@std@@QAA@XZ 0012c118     coredll:COREDLL.dll
 0003:0000011c       __imp_strlen               0012c11c     coredll:COREDLL.dll
 0003:00000120       __imp_??0exception@std@@QAA@PBD@Z 0012c120     coredll:COREDLL.dll
 0003:00000124       __imp_?what@exception@std@@UBAPBDXZ 0012c124     coredll:COREDLL.dll
 0003:00000128       __imp___report_gsfailure   0012c128     coredll:COREDLL.dll
 0003:0000012c       __imp_LocalReAlloc         0012c12c     coredll:COREDLL.dll
 0003:00000130       __imp_LocalAlloc           0012c130     coredll:COREDLL.dll
 0003:00000134       __imp_LocalSize            0012c134     coredll:COREDLL.dll
 0003:00000138       __imp_LocalFree            0012c138     coredll:COREDLL.dll
 0003:0000013c       __imp___security_gen_cookie 0012c13c     coredll:COREDLL.dll
 0003:00000140       __imp_strcmp               0012c140     coredll:COREDLL.dll
 0003:00000144       __imp___C_specific_handler 0012c144     coredll:COREDLL.dll
 0003:00000148       __imp_?terminate@std@@YAXXZ 0012c148     coredll:COREDLL.dll
 0003:0000014c       __imp_memmove              0012c14c     coredll:COREDLL.dll
 0003:00000150       __imp_malloc               0012c150     coredll:COREDLL.dll
 0003:00000154       __imp__snwprintf           0012c154     coredll:COREDLL.dll
 0003:00000158       __imp_GetModuleFileNameW   0012c158     coredll:COREDLL.dll
 0003:0000015c       __imp_TlsSetValue          0012c15c     coredll:COREDLL.dll
 0003:00000160       __imp_TlsGetValue          0012c160     coredll:COREDLL.dll
 0003:00000164       __imp_InterlockedCompareExchange 0012c164     coredll:COREDLL.dll
 0003:00000168       __imp_TlsCall              0012c168     coredll:COREDLL.dll
 0003:0000016c       __imp_EnterCriticalSection 0012c16c     coredll:COREDLL.dll
 0003:00000170       __imp_LeaveCriticalSection 0012c170     coredll:COREDLL.dll
 0003:00000174       __imp_InterlockedDecrement 0012c174     coredll:COREDLL.dll
 0003:00000178       __imp_WriteFile            0012c178     coredll:COREDLL.dll
 0003:0000017c       __imp__getstdfilex         0012c17c     coredll:COREDLL.dll
 0003:00000180       \177COREDLL_NULL_THUNK_DATA 0012c180     coredll:COREDLL.dll
 0003:00000184       __imp_PhoneMakeCall        0012c184     phone:PHONE.dll
 0003:00000188       \177PHONE_NULL_THUNK_DATA  0012c188     phone:PHONE.dll
 0003:0000018c       __imp_tapiRequestMakeCallW 0012c18c     Cellcore:cellcore.dll
 0003:00000190       \177cellcore_NULL_THUNK_DATA 0012c190     Cellcore:cellcore.dll
 0003:00000194       __imp_CreateStreamOnHGlobal 0012c194     ole32:ole32.dll
 0003:00000198       __imp_WriteClassStm        0012c198     ole32:ole32.dll
 0003:0000019c       __imp_CoCreateInstance     0012c19c     ole32:ole32.dll
 0003:000001a0       __imp_ReadClassStm         0012c1a0     ole32:ole32.dll
 0003:000001a4       \177ole32_NULL_THUNK_DATA  0012c1a4     ole32:ole32.dll
 0003:000001a8       __imp_RIL_Hangup           0012c1a8     ril:ril.dll
 0003:000001ac       __imp_RIL_SetEquipmentState 0012c1ac     ril:ril.dll
 0003:000001b0       __imp_RIL_GetSystemTime    0012c1b0     ril:ril.dll
 0003:000001b4       __imp_RIL_DevSpecific      0012c1b4     ril:ril.dll
 0003:000001b8       __imp_RIL_GetRegistrationStatus 0012c1b8     ril:ril.dll
 0003:000001bc       __imp_RIL_GetCallList      0012c1bc     ril:ril.dll
 0003:000001c0       __imp_RIL_GetEquipmentState 0012c1c0     ril:ril.dll
 0003:000001c4       __imp_RIL_CancelSupServiceDataSession 0012c1c4     ril:ril.dll
 0003:000001c8       __imp_RIL_SendSupServiceData 0012c1c8     ril:ril.dll
 0003:000001cc       __imp_RIL_GetSubscriberNumbers 0012c1cc     ril:ril.dll
 0003:000001d0       __imp_RIL_Deinitialize     0012c1d0     ril:ril.dll
 0003:000001d4       __imp_RIL_Initialize       0012c1d4     ril:ril.dll
 0003:000001d8       \177ril_NULL_THUNK_DATA    0012c1d8     ril:ril.dll
 0003:000001dc       __imp_?SWAI_GetRegValue@@YAJPAUHKEY__@@PBG1AAK@Z 0012c1dc     sw_utilityG:sw_utilityG.dll
 0003:000001e0       __imp_?LogW@@YAXPBGZZ      0012c1e0     sw_utilityG:sw_utilityG.dll
 0003:000001e4       __imp_?InitLog@@YAXPAUHINSTANCE__@@@Z 0012c1e4     sw_utilityG:sw_utilityG.dll
 0003:000001e8       __imp_?GetVerInfo@@YAPAGPAUHINSTANCE__@@@Z 0012c1e8     sw_utilityG:sw_utilityG.dll
 0003:000001ec       __imp_?LogStoreFileLine@@YAXPAGH@Z 0012c1ec     sw_utilityG:sw_utilityG.dll
 0003:000001f0       __imp_?LogV@@YAXPBGZZ      0012c1f0     sw_utilityG:sw_utilityG.dll
 0003:000001f4       __imp_?LogC@@YAXPBGZZ      0012c1f4     sw_utilityG:sw_utilityG.dll
 0003:000001f8       __imp_?WriteLog@@YAXKPBGZZ 0012c1f8     sw_utilityG:sw_utilityG.dll
 0003:000001fc       __imp_?GetCarrierIndex@@YAKXZ 0012c1fc     sw_utilityG:sw_utilityG.dll
 0003:00000200       \177sw_utilityG_NULL_THUNK_DATA 0012c200     sw_utilityG:sw_utilityG.dll
 0003:00000204       __xc_a                     0012c204     corelibc:crt0init.obj
 0003:00000284       __xc_z                     0012c284     corelibc:crt0init.obj
 0003:00000288       __xi_a                     0012c288     corelibc:crt0init.obj
 0003:0000028c       __xi_z                     0012c28c     corelibc:crt0init.obj
 0003:00000290       __xp_a                     0012c290     corelibc:crt0init.obj
 0003:00000294       __xp_z                     0012c294     corelibc:crt0init.obj
 0003:00000298       __xt_a                     0012c298     corelibc:crt0init.obj
 0003:0000029c       __xt_z                     0012c29c     corelibc:crt0init.obj
 0003:000002a4       ?gSrvState@@3KA            0012c2a4     DialParsExtOEM.obj
 0003:000002dc       ?m_SrvState@CModemStatus@@2KA 0012c2dc     winmodemstat.obj
 0003:000002e0       ??_R0?AVlength_error@std@@@8 0012c2e0     winmodemstat.obj
 0003:00000300       ??_R0?AVlogic_error@std@@@8 0012c300     winmodemstat.obj
 0003:00000320       ??_R0?AVexception@std@@@8  0012c320     winmodemstat.obj
 0003:0000033c       ??_R0?AVbad_alloc@std@@@8  0012c33c     winmodemstat.obj
 0003:00000358       __security_cookie_complement 0012c358     corelibc:seccook.obj
 0003:0000035c       __security_cookie          0012c35c     corelibc:seccook.obj
 0003:00000498       _crtAssertBusy             0012c498     LIBCMTD:dbgrptt.obj
 0003:0000049c       _CrtDbgMode                0012c49c     LIBCMTD:dbgrptt.obj
 0003:000004a8       _CrtDbgFile                0012c4a8     LIBCMTD:dbgrptt.obj
 0003:000004b4       _aexit_rtn                 0012c4b4     LIBCMTD:crt0dat.obj
 0003:000004c4       ??_R0?AVinvalid_argument@std@@@8 0012c4c4     libcpmtd:string.obj
 0003:000004e8       ??_R0?AVout_of_range@std@@@8 0012c4e8     libcpmtd:string.obj
 0003:00000508       ?rcDefault@CWindow@ATL@@2UtagRECT@@A 0012c508     atlsd:atlfuncs.obj
 0003:00000518       _pRawDllMain               0012c518     atlsd:atlbase.obj
 0003:0000051c       ?g_pszUpdateEventName@@3PB_WB 0012c51c     atlsd:Externs.obj
 0003:00000520       ?g_pszAllocFileMapName@@3PB_WB 0012c520     atlsd:Externs.obj
 0003:00000524       ?g_pszKernelObjFmt@@3PB_WB 0012c524     atlsd:Externs.obj
 0003:00000528       ??_R0?AVCAtlException@ATL@@@8 0012c528     atlsd:Externs.obj
 0003:00000548       ?gPwrState@@3W4ePowerState@CModemStatus@@A 0012c548     DialParsExtOEM.obj
 0003:0000054c       ?m_nCarrier@@3HA           0012c54c     DialParsExtOEM.obj
 0003:00000550       ?g_hmodThisDll@@3PAUHINSTANCE__@@A 0012c550     DialParsExtOEM.obj
 0003:00000554       ?bRequestMakeCall@@3HA     0012c554     DialParsExtOEM.obj
 0003:00000558       ?bEndCallWorkaround@@3HA   0012c558     DialParsExtOEM.obj
 0003:0000055c       ?bRoamMsgCheck@@3HA        0012c55c     DialParsExtOEM.obj
 0003:00000560       ?ghwndRilMessage@@3PAUHWND__@@A 0012c560     DialParsExtOEM.obj
 0003:00000564       ?g_PowerSaveMode@@3W4RIL_PWRSV_MODES@@A 0012c564     DialParsExtOEM.obj
 0003:00000568       ?g_cRefDLL@@3IA            0012c568     DialParsExtOEM.obj
 0003:0000056c       ?g_idCmdExternal@@3IA      0012c56c     DialParsExtOEM.obj
 0003:00000570       ?gModemstat@@3VCModemStatus@@A 0012c570     DialParsExtOEM.obj
 0003:00000574       ?m_bInitFailed@CAtlBaseModule@ATL@@2_NA 0012c574     resultelement.obj
 0003:00000578       ?_pPerfRegFunc@ATL@@3P6AJPAUHINSTANCE__@@@ZA 0012c578     resultelement.obj
 0003:0000057c       ?_pPerfUnRegFunc@ATL@@3P6AJXZA 0012c57c     resultelement.obj
 0003:00000580       ?_pAtlModule@ATL@@3PAVCAtlModule@1@A 0012c580     resultelement.obj
 0003:00000584       ?m_libid@CAtlModule@ATL@@2U_GUID@@A 0012c584     resultelement.obj
 0003:00000594       ?_pModule@ATL@@3PAVCComModule@1@A 0012c594     resultelement.obj
 0003:00000598       ?_AtlWinModule@ATL@@3VCAtlWinModule@1@A 0012c598     resultelement.obj
 0003:000005c0       ?m_MsgBoxBuffer@CModemStatus@@1UtagMsgBoxContent@@A 0012c5c0     winmodemstat.obj
 0003:000009d4       ?m_NonDataCallStatus@CModemStatus@@2KA 0012c9d4     winmodemstat.obj
 0003:000009d8       ?m_DataCallStatus@CModemStatus@@2KA 0012c9d8     winmodemstat.obj
 0003:000009dc       ?m_CallType@CModemStatus@@2KA 0012c9dc     winmodemstat.obj
 0003:000009e0       ?m_PwrState@CModemStatus@@2W4ePowerState@1@A 0012c9e0     winmodemstat.obj
 0003:000009e4       ?m_RoamState@CModemStatus@@2KA 0012c9e4     winmodemstat.obj
 0003:000009e8       ?m_IsOTASPCommited@CModemStatus@@2HA 0012c9e8     winmodemstat.obj
 0003:000009ec       ?m_LastCallEndStatus@CModemStatus@@2GA 0012c9ec     winmodemstat.obj
 0003:000009f0       ?m_hApi@CModemStatus@@1PAXA 0012c9f0     winmodemstat.obj
 0003:000009f4       ?m_hActiveWindow@CModemStatus@@2PAUHWND__@@A 0012c9f4     winmodemstat.obj
 0003:000009f8       ?m_MainWndH@CModemStatus@@1PAUHWND__@@A 0012c9f8     winmodemstat.obj
 0003:000009fc       ?m_hCurrModPowerState@CModemStatus@@2PAXA 0012c9fc     winmodemstat.obj
 0003:00000a00       ?m_hEquipmentStateOn@CModemStatus@@2PAXA 0012ca00     winmodemstat.obj
 0003:00000a04       ?m_bDMMode@CModemStatus@@1HA 0012ca04     winmodemstat.obj
 0003:00000a08       ?m_cFuncResultList@CModemStatus@@1V?$list@VCResultListElement@@V?$allocator@VCResultListElement@@@std@@@std@@A 0012ca08     winmodemstat.obj
 0003:00000bbc       ?_pAtlRawDllMain@@3P6AHPAXK0@ZA 0012cbbc     atlsd:atlbase.obj
 0003:00000bc0       ?_AtlModuleInstance@ATL@@3PAUHINSTANCE__@@A 0012cbc0     atlsd:atlbase.obj
 0003:00000bc4       ?_AtlBaseModule@ATL@@3VCAtlBaseModule@1@A 0012cbc4     atlsd:atlbase.obj
 0003:00000c48       ?atlTraceGeneral@ATL@@3VCTraceCategory@1@A 0012cc48     atlsd:atltrace.obj
 0003:00000c4c       ?atlTraceCOM@ATL@@3VCTraceCategory@1@A 0012cc4c     atlsd:atltrace.obj
 0003:00000c50       ?atlTraceQI@ATL@@3VCTraceCategory@1@A 0012cc50     atlsd:atltrace.obj
 0003:00000c54       ?atlTraceRegistrar@ATL@@3VCTraceCategory@1@A 0012cc54     atlsd:atltrace.obj
 0003:00000c58       ?atlTraceRefcount@ATL@@3VCTraceCategory@1@A 0012cc58     atlsd:atltrace.obj
 0003:00000c5c       ?atlTraceWindowing@ATL@@3VCTraceCategory@1@A 0012cc5c     atlsd:atltrace.obj
 0003:00000c60       ?atlTraceControls@ATL@@3VCTraceCategory@1@A 0012cc60     atlsd:atltrace.obj
 0003:00000c64       ?atlTraceHosting@ATL@@3VCTraceCategory@1@A 0012cc64     atlsd:atltrace.obj
 0003:00000c68       ?atlTraceNotImpl@ATL@@3VCTraceCategory@1@A 0012cc68     atlsd:atltrace.obj
 0003:00000c6c       ?atlTraceAllocation@ATL@@3VCTraceCategory@1@A 0012cc6c     atlsd:atltrace.obj
 0003:00000c70       ?atlTraceException@ATL@@3VCTraceCategory@1@A 0012cc70     atlsd:atltrace.obj
 0003:00000c74       ?atlTraceTime@ATL@@3VCTraceCategory@1@A 0012cc74     atlsd:atltrace.obj
 0003:00000c78       ?atlTraceCache@ATL@@3VCTraceCategory@1@A 0012cc78     atlsd:atltrace.obj
 0003:00000c7c       ?atlTraceStencil@ATL@@3VCTraceCategory@1@A 0012cc7c     atlsd:atltrace.obj
 0003:00000c80       ?atlTraceString@ATL@@3VCTraceCategory@1@A 0012cc80     atlsd:atltrace.obj
 0003:00000c84       ?atlTraceMap@ATL@@3VCTraceCategory@1@A 0012cc84     atlsd:atltrace.obj
 0003:00000c88       ?atlTraceUtil@ATL@@3VCTraceCategory@1@A 0012cc88     atlsd:atltrace.obj
 0003:00000c8c       ?atlTraceSync@ATL@@3VCTraceCategory@1@A 0012cc8c     atlsd:atltrace.obj
 0003:00000c90       ?atlTraceUser@ATL@@3VCTraceCategory@1@A 0012cc90     atlsd:atltrace.obj
 0003:00000c94       ?atlTraceUser2@ATL@@3VCTraceCategory@1@A 0012cc94     atlsd:atltrace.obj
 0003:00000c98       ?atlTraceUser3@ATL@@3VCTraceCategory@1@A 0012cc98     atlsd:atltrace.obj
 0003:00000c9c       ?atlTraceUser4@ATL@@3VCTraceCategory@1@A 0012cc9c     atlsd:atltrace.obj
 0003:00000ca0       ?g_Allocator@@3VCAtlAllocator@@A 0012cca0     atlsd:Externs.obj
 0003:00000cd4       ?s_trace@CTrace@ATL@@2V12@A 0012ccd4     atlsd:Externs.obj
 0003:00000cdc       __onexitend                0012ccdc     <common>
 0003:00000ce0       __onexitbegin              0012cce0     <common>
 0003:00000ce4       _exitflag                  0012cce4     <common>
 0003:00000ce8       _pfnReportHook             0012cce8     <common>
 0003:00000cec       _pReportHookListW          0012ccec     <common>
 0003:00000cf0       _pReportHookList           0012ccf0     <common>

 entry point at        0001:0000a8e4

 Static symbols

 0001:fffff030       __unwind$63208             00100030 f   winmodemstat.obj
 0001:fffff038       __unwind$63243             00100038 f   winmodemstat.obj
 0001:fffff050       __unwind$63013             00100050 f   winmodemstat.obj
 0001:fffff058       __unwind$18984             00100058 f   libcpmtd:string.obj
 0001:fffff058       __unwind$18609             00100058 f   libcpmtd:string.obj
 0001:fffff060       __unwind$19542             00100060 f   libcpmtd:string.obj
 0001:fffff068       __unwind$18537             00100068 f   libcpmtd:string.obj
 0001:fffff108       __catch$18380              00100108 f   libcpmtd:string.obj
 0001:fffff144       __catch$18378              00100144 f   libcpmtd:string.obj
 0001:000003e0       __unwind$39885             001013e0 f   clsfact.obj
 0001:000032c4       __unwind$48062             001042c4 f i resultelement.obj
 0001:000033a4       __unwind$48114             001043a4 f i resultelement.obj
 0001:00003454       __unwind$48149             00104454 f i resultelement.obj
 0001:00003910       __unwind$60975             00104910 f   winmodemstat.obj
 0001:00003928       __unwind$60976             00104928 f   winmodemstat.obj
 0001:00003d34       __catch$61118              00104d34 f   winmodemstat.obj
 0001:0000404c       __catch$61190              0010504c f   winmodemstat.obj
 0001:00004228       __catch$61224              00105228 f   winmodemstat.obj
 0001:00004b24       __unwind$61267             00105b24 f   winmodemstat.obj
 0001:00004b44       __unwind$61268             00105b44 f   winmodemstat.obj
 0001:00004b64       __unwind$61269             00105b64 f   winmodemstat.obj
 0001:00004b84       __unwind$61271             00105b84 f   winmodemstat.obj
 0001:00005618       __catch$61531              00106618 f   winmodemstat.obj
 0001:000058ac       __catch$61561              001068ac f   winmodemstat.obj
 0001:00006d5c       __catch$61796              00107d5c f   winmodemstat.obj
 0001:00006f7c       __catch$61827              00107f7c f   winmodemstat.obj
 0001:0000712c       __catch$61863              0010812c f   winmodemstat.obj
 0001:000073a8       __unwind$61046             001083a8 f i winmodemstat.obj
 0001:00007750       __unwind$61407             00108750 f i winmodemstat.obj
 0001:00007808       __unwind$61426             00108808 f i winmodemstat.obj
 0001:000079f0       __unwind$61918             001089f0 f i winmodemstat.obj
 0001:00007a08       __unwind$61920             00108a08 f i winmodemstat.obj
 0001:00007bec       __unwind$61946             00108bec f i winmodemstat.obj
 0001:00007c04       __unwind$61947             00108c04 f i winmodemstat.obj
 0001:00007c1c       __unwind$61948             00108c1c f i winmodemstat.obj
 0001:00007d2c       __unwind$61999             00108d2c f i winmodemstat.obj
 0001:00007d44       __unwind$62000             00108d44 f i winmodemstat.obj
 0001:00007f00       __unwind$62051             00108f00 f i winmodemstat.obj
 0001:000083d4       __catch$62190              001093d4 f i winmodemstat.obj
 0001:00008510       __unwind$62217             00109510 f i winmodemstat.obj
 0001:000085d4       __unwind$62253             001095d4 f i winmodemstat.obj
 0001:00008784       __unwind$62318             00109784 f i winmodemstat.obj
 0001:000087d8       __unwind$62338             001097d8 f i winmodemstat.obj
 0001:00008fdc       __unwind$62538             00109fdc f i winmodemstat.obj
 0001:00009344       __unwind$62617             0010a344 f i winmodemstat.obj
 0001:000093d0       __unwind$62640             0010a3d0 f i winmodemstat.obj
 0001:00009600       __catch$62671              0010a600 f i winmodemstat.obj
 0001:00009638       __catch$62669              0010a638 f i winmodemstat.obj
 0001:00009fb8       __unwind$63067             0010afb8 f i winmodemstat.obj
 0001:0000a0c4       __catch$63110              0010b0c4 f i winmodemstat.obj
 0001:0000a2dc       __unwind$63333             0010b2dc f i winmodemstat.obj
 0001:0000aaa0       _initterm                  0010baa0 f   corelibc:crt0dat.obj
 0001:0000ab40       doexit                     0010bb40 f   corelibc:crt0dat.obj
 0001:0000af84       ?FindHandler@@YAEPAUEHExceptionRecord@@PAKPAU_CONTEXT@@PAU_DISPATCHER_CONTEXT@@PBU_s_FuncInfo@@H@Z 0010bf84 f   LIBCMTD:frame_ce.obj
 0001:0000b578       ?TypeMatch@@YAHPBU_s_HandlerType@@PBU_s_CatchableType@@PBU_s_ThrowInfo@@@Z 0010c578 f   LIBCMTD:frame_ce.obj
 0001:0000b93c       ?FrameUnwindFilter@@YAHPAU_EXCEPTION_POINTERS@@@Z 0010c93c f   LIBCMTD:frame_ce.obj
 0001:0000b9c8       ?CallCatchBlock@@YAPAXPAUEHExceptionRecord@@PAKPAU_CONTEXT@@PBU_s_FuncInfo@@PAXHK@Z 0010c9c8 f   LIBCMTD:frame_ce.obj
 0001:0000bf64       ?CanThisExceptionObjectBeDestructed@@YAEPAUEHExceptionRecord@@E@Z 0010cf64 f   LIBCMTD:frame_ce.obj
 0001:0000c1f0       ?BuildCatchObject@@YAXPAUEHExceptionRecord@@PAKPBU_s_HandlerType@@PBU_s_CatchableType@@@Z 0010d1f0 f   LIBCMTD:frame_ce.obj
 0001:0000c540       ?AdjustPointer@@YAPAXPAXABUPMD@@@Z 0010d540 f   LIBCMTD:frame_ce.obj
 0001:000103c4       __crtInitCritSecNoSpinCount 001113c4 f   LIBCMTD:initcrit.obj
 0001:00010f5c       xtow_s                     00111f5c f   LIBCMTD:xtows.obj
 0001:00011c50       __unwind$18810             00112c50 f   libcpmtd:string.obj
 0001:00011ce0       __unwind$19010             00112ce0 f   libcpmtd:string.obj
 0001:00011da0       __unwind$19588             00112da0 f   libcpmtd:string.obj
 0001:00014744       ?_ATLLoadOle32API@ATL@@YAP6AHXZPB_W@Z 00115744 f   atlsd:atlbase.obj
 0001:00016788       ?Init@@YA_NXZ              00117788 f   atlsd:Externs.obj
 0001:000187d0       ?ShouldTraceOutput@ATL@@YA_NKKIPAPBVCAtlTraceCategory@@PAP6AHHPB_WH11ZZ@Z 001197d0 f   atlsd:AtlDebugAPI.obj
 0001:0001ba50       ??__EgModemstat@@YAXXZ     0011ca50 f   DialParsExtOEM.obj
 0001:0001ba70       ??__E_AtlWinModule@ATL@@YAXXZ 0011ca70 f   resultelement.obj
 0001:0001ba90       ??__E_AtlWinModule@ATL@@YAXXZ 0011ca90 f   winmodemstat.obj
 0001:0001bab0       ??__E?m_cFuncResultList@CModemStatus@@1V?$list@VCResultListElement@@V?$allocator@VCResultListElement@@@std@@@std@@A@@YAXXZ 0011cab0 f   winmodemstat.obj
 0001:0001bad0       ??__Einitlocks@std@@YAXXZ  0011cad0 f   libcpmtd:xlock.obj
 0001:0001bb0c       ??__E_AtlWinModule@ATL@@YAXXZ 0011cb0c f   atlsd:atlfuncs.obj
 0001:0001bb48       ??__E_AtlBaseModule@ATL@@YAXXZ 0011cb48 f   atlsd:atlbase.obj
 0001:0001bb84       ??__E_AtlWinModule@ATL@@YAXXZ 0011cb84 f   atlsd:atlbase.obj
 0001:0001bbc0       ??__EatlTraceGeneral@ATL@@YAXXZ 0011cbc0 f   atlsd:atltrace.obj
 0001:0001bbf0       ??__EatlTraceCOM@ATL@@YAXXZ 0011cbf0 f   atlsd:atltrace.obj
 0001:0001bc20       ??__EatlTraceQI@ATL@@YAXXZ 0011cc20 f   atlsd:atltrace.obj
 0001:0001bc50       ??__EatlTraceRegistrar@ATL@@YAXXZ 0011cc50 f   atlsd:atltrace.obj
 0001:0001bc80       ??__EatlTraceRefcount@ATL@@YAXXZ 0011cc80 f   atlsd:atltrace.obj
 0001:0001bcb0       ??__EatlTraceWindowing@ATL@@YAXXZ 0011ccb0 f   atlsd:atltrace.obj
 0001:0001bce0       ??__EatlTraceControls@ATL@@YAXXZ 0011cce0 f   atlsd:atltrace.obj
 0001:0001bd10       ??__EatlTraceHosting@ATL@@YAXXZ 0011cd10 f   atlsd:atltrace.obj
 0001:0001bd40       ??__EatlTraceNotImpl@ATL@@YAXXZ 0011cd40 f   atlsd:atltrace.obj
 0001:0001bd70       ??__EatlTraceAllocation@ATL@@YAXXZ 0011cd70 f   atlsd:atltrace.obj
 0001:0001bda0       ??__EatlTraceException@ATL@@YAXXZ 0011cda0 f   atlsd:atltrace.obj
 0001:0001bdd0       ??__EatlTraceTime@ATL@@YAXXZ 0011cdd0 f   atlsd:atltrace.obj
 0001:0001be00       ??__EatlTraceCache@ATL@@YAXXZ 0011ce00 f   atlsd:atltrace.obj
 0001:0001be30       ??__EatlTraceStencil@ATL@@YAXXZ 0011ce30 f   atlsd:atltrace.obj
 0001:0001be60       ??__EatlTraceString@ATL@@YAXXZ 0011ce60 f   atlsd:atltrace.obj
 0001:0001be90       ??__EatlTraceMap@ATL@@YAXXZ 0011ce90 f   atlsd:atltrace.obj
 0001:0001bec0       ??__EatlTraceUtil@ATL@@YAXXZ 0011cec0 f   atlsd:atltrace.obj
 0001:0001bef0       ??__EatlTraceSync@ATL@@YAXXZ 0011cef0 f   atlsd:atltrace.obj
 0001:0001bf20       ??__EatlTraceUser@ATL@@YAXXZ 0011cf20 f   atlsd:atltrace.obj
 0001:0001bf50       ??__EatlTraceUser2@ATL@@YAXXZ 0011cf50 f   atlsd:atltrace.obj
 0001:0001bf80       ??__EatlTraceUser3@ATL@@YAXXZ 0011cf80 f   atlsd:atltrace.obj
 0001:0001bfb0       ??__EatlTraceUser4@ATL@@YAXXZ 0011cfb0 f   atlsd:atltrace.obj
 0001:0001bfe0       ??__E_AtlWinModule@ATL@@YAXXZ 0011cfe0 f   atlsd:atltrace.obj
 0001:0001c01c       ??__Eg_Allocator@@YAXXZ    0011d01c f   atlsd:Externs.obj
 0001:0001c058       ??__Eg_bInitialized@@YAXXZ 0011d058 f   atlsd:Externs.obj
 0001:0001c090       ??__E?s_trace@CTrace@ATL@@2V12@A@@YAXXZ 0011d090 f   atlsd:Externs.obj
 0001:0001c0d4       ??__E_AtlWinModule@ATL@@YAXXZ 0011d0d4 f   atlsd:Externs.obj
 0001:0001c110       ??__E_AtlWinModule@ATL@@YAXXZ 0011d110 f   atlsd:AtlDebugAPI.obj
 0001:0001c14c       ??__E_AtlWinModule@ATL@@YAXXZ 0011d14c f   atlsd:Allocate.obj
 0001:0001c188       ??__E_AtlWinModule@ATL@@YAXXZ 0011d188 f   atlsd:AtlTraceModuleManager.obj
 0001:0001c1c4       ??__FgModemstat@@YAXXZ     0011d1c4 f   DialParsExtOEM.obj
 0001:0001c1d8       ??__F_AtlWinModule@ATL@@YAXXZ 0011d1d8 f   resultelement.obj
 0001:0001c1ec       ??__F_AtlWinModule@ATL@@YAXXZ 0011d1ec f   winmodemstat.obj
 0001:0001c200       ??__F?m_cFuncResultList@CModemStatus@@1V?$list@VCResultListElement@@V?$allocator@VCResultListElement@@@std@@@std@@A@@YAXXZ 0011d200 f   winmodemstat.obj
 0001:0001c214       ??__Finitlocks@std@@YAXXZ  0011d214 f   libcpmtd:xlock.obj
 0001:0001c238       ??__F_AtlWinModule@ATL@@YAXXZ 0011d238 f   atlsd:atlfuncs.obj
 0001:0001c25c       ??__F_AtlBaseModule@ATL@@YAXXZ 0011d25c f   atlsd:atlbase.obj
 0001:0001c280       ??__F_AtlWinModule@ATL@@YAXXZ 0011d280 f   atlsd:atlbase.obj
 0001:0001c2a4       ??__F_AtlWinModule@ATL@@YAXXZ 0011d2a4 f   atlsd:atltrace.obj
 0001:0001c2c8       ??__Fg_Allocator@@YAXXZ    0011d2c8 f   atlsd:Externs.obj
 0001:0001c2ec       ??__F?s_trace@CTrace@ATL@@2V12@A@@YAXXZ 0011d2ec f   atlsd:Externs.obj
 0001:0001c310       ??__F_AtlWinModule@ATL@@YAXXZ 0011d310 f   atlsd:Externs.obj
 0001:0001c334       ??__F_AtlWinModule@ATL@@YAXXZ 0011d334 f   atlsd:AtlDebugAPI.obj
 0001:0001c358       ??__F_AtlWinModule@ATL@@YAXXZ 0011d358 f   atlsd:Allocate.obj
 0001:0001c37c       ??__F_AtlWinModule@ATL@@YAXXZ 0011d37c f   atlsd:AtlTraceModuleManager.obj
